:100000000C94B9050C94E4050C94E4050C94E405F7
:100010000C94750D0C94E4050C94E4050C94E40523
:100020000C94E4050C94BC2D0C94E4050C94E405AC
:100030000C94E4050C9446380C94E4050C94E40507
:100040000C94E4050C94E4050C946B850C94E40585
:100050000C9467830C94B2830C94E4050C94E4052F
:100060000C94E4050C94E4050C94A0810C94E40534
:100070000C9431370C94F1830C94E4050C94E40552
:100080000C94E4050C94E4050C94E4052D33002D48
:1000900032002D31002030002B31002B32002B3369
:1000A000002B340020430020432300204400204440
:1000B0002300204500204600204623002047002042
:1000C000472300204100204123002042004D53548B
:1000D000004D494400434C4B00322F3100312F3149
:1000E00000312F3200312F34003132700032347041
:1000F000003438700053494E005452490053415760
:100100000053515500532F48004457320044573391
:100110000044573400445735004457360054573193
:100120000054573200545733005457340045585048
:1001300000485244005346540046555A0053504B11
:1001400000535450004F666600313A3200313A3362
:1001500000313A3400313A3500313A3600313A371D
:1001600000313A3800323A3300333A3400373A3803
:100170000031302500323525003530250037352552
:100180000039302500434852004D414A006D696EE8
:100190000050454E00444F5200504852004C5944C4
:1001A000004D4958004C4F4300464F52574152446E
:1001B0002020004241434B57415244200050494EB9
:1001C000472D504F4E470052414E444F4D20202066
:1001D0000053594E0042504D00545258004356525D
:1001E0005800434C4B004E430041430050545200D2
:1001F0004C454E0053434C0054524947004C464F27
:10020000005741560046525100414D500053545042
:10021000004E5445004F4354004C454E4700555442
:100220004D0050524F00525452470050554C00421E
:1002300041520043505900415554004D414E004F2A
:10024000464600204F4E0052535400504F53005327
:100250004E47004D555400524F4F00202020004281
:1002600044005344005331005332004C54004D5469
:10027000004854004350004348004F480043520098
:100280005244003576200031307600D101D5012B63
:1002900002E201330247025302E901EC01F001F4EA
:1002A00001F801FD010102050209022F02110215E8
:1002B000021902F401E601E601E6012F021E022204
:1002C0000226022F021E02220219022F02F001F45E
:1002D00001F8014F024B02EC01F001110215020D71
:1002E000021902F401570215025B02A901B301BD14
:1002F00001C701850189018D019101950199019D38
:1003000001A101A501450149014D015101550159C5
:10031000015D016101650169016D0171017501797D
:10032000017D018101F500F900FD000101050109D0
:10033000010D011101150119011D012101250129DD
:10034000012D013101350139013D014101D900DDA6
:1003500000E100E500E900ED00F100CD00D100D59D
:10036000008C008F009200950098009B009E00A1D9
:1003700000A400A700AB00AE00B200B500B800BCFE
:1003800000BF00C300C600CA005F026202650268C7
:10039000026B026E027102740277027A027D0280A1
:1003A000023B0237023F024302830287020102033B
:1003B0000405060708090A0B0C01010303050606DC
:1003C00008080A0A0C0101030304060608080909C3
:1003D0000B0101030303050508080A0A0A010103CA
:1003E0000304060608080A0A0B01010202040606B5
:1003F000080809090B0101030305070708080A0A91
:100400000C0101030305060608080A0A0B01010294
:1004100002040606070709090B00002B005500809F
:1004200000AB00D50000012B0155018001AB01D5C7
:1004300001807C797673706D6A6763605D5A57548A
:10044000514F4C494643403E3B383633312E2C2ADF
:10045000272523211F1D1B1917151312100F0D0C13
:100460000A09080706050403030201010000000051
:10047000000000000000000101020303040506075C
:1004800008090A0C0D0F1012131517191B1D1F2137
:100490002325272A2C2E313336383B3E404346490C
:1004A0004C4F5154575A5D6063676A6D707376792B
:1004B0007C808386898C8F9295989C9FA2A5A8ABFF
:1004C000AEB0B3B6B9BCBFC1C4C7C9CCCED1D3D509
:1004D000D8DADCDEE0E2E4E6E8EAECEDEFF0F2F3B5
:1004E000F5F6F7F8F9FAFBFCFCFDFEFEFFFFFFFF57
:1004F000FFFFFFFFFFFFFFFEFEFDFCFCFBFAF9F82C
:10050000F7F6F5F3F2F0EFEDECEAE8E6E4E2E0DE30
:10051000DCDAD8D5D3D1CECCC9C7C4C1BFBCB9B63B
:10052000B3B0AEABA8A5A29F9C9895928F8C8986FC
:10053000837C7A78767472706E6C6A6866646260C6
:100540005E5C5A58565452504E4C4A4846444240BB
:100550003E3C3A38363432302E2C2A2826242220AB
:100560001E1C1A18161412100E0C0A08060402019A
:100570000000020406080A0C0E10121416181A1CA9
:100580001E20222426282A2C2E30323436383A3C9B
:100590003E40424446484A4C4E50525456585A5C8B
:1005A0005E60626466686A6C6E70727476787A7C7B
:1005B0007E80828486888A8C8E90929496989A9C6B
:1005C0009EA0A2A4A6A8AAACAEB0B2B4B6B8BABC5B
:1005D000BEC0C2C4C6C8CACCCED0D2D4D6D8DADC4B
:1005E000DEE0E2E4E6E8EAECEEF0F2F4F6F8FAFC3B
:1005F000FEFEFCFAF8F6F4F2F0EEECEAE8E6E4E2ED
:10060000E0DEDCDAD8D6D4D2D0CECCCAC8C6C4C2DA
:10061000C0BEBCBAB8B6B4B2B0AEACAAA8A6A4A2CA
:10062000A09E9C9A98969492908E8C8A88868482BA
:10063000807E0102030405060708090A0B0C0D0E53
:100640000F101112131415161718191A1B1C1D1E42
:100650001F202122232425262728292A2B2C2D2E32
:100660002F303132333435363738393A3B3C3D3E22
:100670003F404142434445464748494A4B4C4D4E12
:100680004F505152535455565758595A5B5C5D5E02
:100690005F606162636465666768696A6B6C6D6EF2
:1006A0006F707172737475767778797A7B7C7D7EE2
:1006B0007F808182838485868788898A8B8C8D8ED2
:1006C0008F909192939495969798999A9B9C9D9EC2
:1006D0009FA0A1A2A3A4A5A6A7A8A9AAABACADAEB2
:1006E000AFB0B1B2B3B4B5B6B7B8B9BABBBCBDBEA2
:1006F000BFC0C1C2C3C4C5C6C7C8C9CACBCCCDCE92
:10070000CFD0D1D2D3D4D5D6D7D8D9DADBDCDDDE81
:10071000DFE0E1E2E3E4E5E6E7E8E9EAEBECEDEE71
:10072000EFF0F1F2F3F4F5F6F7F8F9FAFBFCFDFE61
:10073000FF000000000000000000000000000000BA
:1007400000000000000000000000000000000000A9
:100750000000000000000000000000000000000099
:100760000000000000000000000000000000000089
:100770000000000000000000000000000000000079
:100780000000000000000000000000000000000069
:100790000000000000000000000000000000000059
:1007A0000000000000000000000000000000000049
:1007B0000000FFFFFFFFFFFFFFFFFFFFFFFFFFFF47
:1007C000FFFFFFFFFFFFFFFFFFFFFFFFFFFFFFFF39
:1007D000FFFFFFFFFFFFFFFFFFFFFFFFFFFFFFFF29
:1007E000FFFFFFFFFFFFFFFFFFFFFFFFFFFFFFFF19
:1007F000FFFFFFFFFFFFFFFFFFFFFFFFFFFFFFFF09
:10080000FFFFFFFFFFFFFFFFFFFFFFFFFFFFFFFFF8
:10081000FFFFFFFFFFFFFFFFFFFFFFFFFFFFFFFFE8
:10082000FFFFFFFFFFFFFFFFFFFFFFFFFFFFFFFFD8
:10083000FFFF202837465564738291202020200036
:100840002E2E2E2E2E2E2E2E2E2E2E2E2E2E2E2EC8
:1008500000444143732063616C6962726174696F23
:100860006E0020696E697469616C697A6174696F80
:100870006E20002020202020454550524F4D202042
:10088000202020002B002D00546F74616C204163E8
:10089000632076616C756520005B506173746564DC
:1008A000215D005B436F70696564215D005B5341AE
:1008B000564544215D007832007831002020202008
:1008C0002020202020202020202020200020202048
:1008D0002000202020200020202020002020202078
:1008E0000010182030406080205374657020202054
:1008F0004163632F566F6C74006E7465206F637470
:1009000020737470206C656E67005074726E2000E6
:10091000506F73200020536F6E6720506C617920F8
:100920005300736E6720706F7320707472206C6553
:100930006E20004F6E004F6666004F6E004F666679
:100940000020204C464F73202043562F476174658A
:10095000200073006261722075746D2070726F20C8
:1009600072747267006261722075746D2070726FAC
:10097000206C656E67006C666F207761762066720A
:100980007120616D70200073636C20726F6F206F37
:1009900063742020202020007300626172206E7436
:1009A00065206F6374206C656E6700202020003125
:1009B0002F0046494C4C00626172206C656E2073BA
:1009C000636C20747269670073636C20726F6F20B0
:1009D0006F6374202020202000626172206C656E9D
:1009E0002073636C2074726967004558540020209E
:1009F0005061747465726E20506C61792020002003
:100A00002020426172202020205374657020200035
:100A1000200061630063707920727374206D7574B7
:100A20000073796E2062706D2070756C20636C6B42
:100A30002000205472636B20646972656374696F6F
:100A40006E2000205074726E206469726563746950
:100A50006F6E20002B002D00202053687566666C99
:100A6000652076616C756520000002040507090B9E
:100A7000000205070900030408121313111F0000E8
:100A800000000000000018040209191911100806DE
:100A900001000000000004001F0000000001020C23
:100AA00010000000001010111204081000000017C0
:100AB00014171517000000101810100C0000000E7D
:100AC0000A0E0A0E0000001B091B0A1B000101018F
:100AD00001010F1F0E00000A0A0E02020000000EA4
:100AE000020E080E0076312E30353600000021004F
:100AF000240027002A0000002200250028002B00E7
:100B00000000200023002600290002020202020247
:100B1000020204040404040404040303030303039F
:100B20000303010101010101010101020408102078
:100B300040800102040810204080010204081020B7
:100B400040800102040810204080000000010200E3
:100B50000809000000000403070600000000000070
:100B60000000000000000000000008273880D58445
:100B7000012711241FBECFEFD0E4DEBFCDBF11E0AF
:100B8000A0E0B1E0E4E3FEE101E00BBF02C00790AA
:100B90000D92AC3EB107D9F71BBE1BE3ACEEB1E042
:100BA00001C01D92A338B107E1F71BE0C0E7DBE00D
:100BB00004C02297FE010E94D28ECA36D107C9F71F
:100BC0000E9425870C940D8F0C940000CF93DF9327
:100BD000BC018230910510F462E070E0A091813B8D
:100BE000B091823BED01E0E0F0E040E050E021C058
:100BF000888199818617970769F48A819B8130974C
:100C000019F09383828304C09093823B8093813B4D
:100C1000FE0134C06817790738F44115510519F001
:100C20008417950708F4AC01FE018A819B819C0121
:100C3000E9012097E9F641155105A9F1CA01861B82
:100C4000970B049708F4BA01E0E0F0E02AC08D9118
:100C50009C91119784179507F9F46417750781F42F
:100C600012968D919C911397309719F093838283FC
:100C700004C09093823B8093813BFD0132964CC02F
:100C8000CA01861B970BFD01E80FF91F6193719351
:100C900002978D939C9340C0FD01828193819C01BA
:100CA000D9011097A1F680917F3B9091803B892BD1
:100CB00041F480912401909125019093803B809391
:100CC0007F3B40912601509127014115510541F488
:100CD0004DB75EB78091220190912301481B590BBB
:100CE00020917F3B3091803BCA01821B930B86177A
:100CF000970780F0AB014E5F5F4F8417950750F068
:100D0000420F531F5093803B40937F3BF901619307
:100D1000719302C0E0E0F0E0CF01DF91CF91089540
:100D2000CF93DF93009709F450C0EC0122971B8208
:100D30001A82A091813BB091823B109709F140E06B
:100D400050E0AC17BD0708F1BB83AA83FE012191D7
:100D50003191E20FF31FAE17BF0779F48D919C918B
:100D60001197280F391F2E5F3F4F39832883129622
:100D70008D919C9113979B838A834115510571F442
:100D8000D093823BC093813B20C012968D919C9161
:100D90001397AD01009711F0DC01D3CFFA01D38393
:100DA000C28321913191E20FF31FCE17DF0769F45F
:100DB00088819981280F391F2E5F3F4FFA013183B7
:100DC00020838A819B8193838283DF91CF910895D1
:100DD000A0E0B0E0EEEEF6E00C94DE8EEC01A88030
:100DE000B980CA80DB80A114B104C104D10441F4EC
:100DF00084E2A82E89EDB82E8BE5C82E87E0D82E88
:100E0000C601B5012DE133EF41E050E00E94B58EFF
:100E100027EA31E440E050E00E94418E7B018C01E2
:100E2000C601B5012DE133EF41E050E00E94B58EDF
:100E3000CA01B9012CEE34EF4FEF5FEF0E94418EF3
:100E40006E0D7F1D801F911F97FF04C06150704081
:100E500080409048688379838A839B839B01AC019F
:100E60005F77B901CA01CDB7DEB7EAE00C94FA8E1C
:100E70000E94E806089588E291E00E94E80608953D
:100E8000609328017093290180932A0190932B018C
:100E90000895A0E0B0E0EFE4F7E00C94D88E6C0188
:100EA000009729F4CB010E94E6056C01C1C08EEFCA
:100EB000882E8FEF982E8C0C9D1C8601060F171F15
:100EC0000815190508F4B2C0F401A081B181A61774
:100ED000B707B8F0A530B10508F4AAC0CD01049752
:100EE0008617970708F4A4C01297A61BB70BF80142
:100EF000A193B193D4016D937C93CF010E9490068E
:100F000097C07B01EA1AFB0AEEEFFFEFEE0EFF1E21
:100F100036016A0E7B1EC091813BD091823B4424F6
:100F20005524AA24BB244AC0C615D705E1F548813B
:100F300059814E155F05B8F1CA0104978E159F05BA
:100F4000B0F41296A40FB51FF401B183A0832A81D7
:100F50003B814114510431F0D20113963C932E93FE
:100F6000129766C03093823B2093813B61C08A8197
:100F70009B81F80193838283425050404E195F0950
:100F8000518340834114510431F0D20113961C93D4
:100F90000E93129704C01093823B0093813BF4019F
:100FA0007183608345C088819981A816B90608F4C9
:100FB0005C012E018A819B819C01E901209709F047
:100FC000B3CF80917F3B9091803B86159705E9F4E4
:100FD000A616B706D0F420912601309127012115DD
:100FE000310541F42DB73EB7809122019091230144
:100FF000281B390B02171307C8F41093803B00938A
:101000007F3BD4016D937C9313C0CB010E94E60516
:10101000EC01009759F0F40140815181B6010E9422
:101020002508C6010E9490066E0102C0CC24DD2472
:10103000C601CDB7DEB7E0E10C94F48EFB01DC0114
:1010400005900D920020E1F70895FB01DC0102C03C
:1010500001900D9241505040D8F70895FB01DC01FA
:101060008D91019080190110D9F3990B0895FB011E
:10107000DC0101900D920020E1F70895FB019F0132
:10108000E8944230C4F04532B4F44A3029F497FB76
:101090001EF4909581959F4F642F77270E946C8E48
:1010A000805D8A330CF0895D8193CB010097A1F7B5
:1010B00016F45DE251931082C9010C947508FB018E
:1010C0009F01423074F0453264F4642F77270E9408
:1010D0006C8E805D8A330CF0895D8193CB01009723
:1010E000A1F71082C9010C947508DC01FC01672F7F
:1010F00071917723E1F7329704C07C916D937083EF
:101100006291AE17BF07C8F30895CF92DF92EF92B6
:10111000FF920F931F93CF93DF93382F9091533605
:1011200080E020915236022F10E0082B192B332338
:1011300021F0313009F047C047C0C6E5D7E340E0B1
:1011400050E081E0C82ED12CE12CF12CC801042EF6
:1011500002C0969587950A94E2F7282F2170FA012C
:10116000EA59F84C20838881281731F1213021F584
:10117000CB01042E02C0969587950A94E2F780FF72
:101180000FC0D701C601042E04C0880F991FAA1FE3
:10119000BB1F0A94D2F780959095682379230CC0E1
:1011A000D701C601042E04C0880F991FAA1FBB1FB8
:1011B0000A94D2F7682B792B29934F5F5F4F403108
:1011C000510521F602C002C0B801CB01DF91CF91D9
:1011D0001F910F91FF90EF90DF90CF9008952F9285
:1011E0003F924F925F926F927F928F929F92AF92B7
:1011F000BF92CF92DF92EF92FF920F931F93DF93F4
:10120000CF9300D000D0CDB7DEB71C0180919736C8
:1012100085FF03C081E0809345378091B1028A83C6
:10122000482F50E0FA01E25BF44D6080629430EFA9
:1012300063222091352B30E09091B90399839090EF
:101240004C027090453706E417E360E070E084ECF0
:1012500090E0489F5001499FB00C589FB00C11245A
:1012600085E29DE0289F7001299FF00C389FF00CCB
:1012700011246A01CE0CDF1CA9ECB3E0CA0EDB1E00
:101280002BE3422E2BE2522E440E551E562D560FA6
:10129000E52FF0E0FC83EB83EE0FFF1F8B819C8139
:1012A000E80FF91FEA0DFB1DEE0DFF1DE452FC4F88
:1012B0008081382F3170282F26952170D6018C908F
:1012C000C101062E02C0969587950A94E2F7482F31
:1012D0004170DB01AA0FBB1FFD01E559F94C90815C
:1012E0009E7F942B9083892F86958170481711F4E7
:1012F000592D90C0969596959170913009F053C0F4
:10130000442309F061C0332309F45EC0222371F441
:10131000882009F4B2C0F8018081882309F0ADC0AB
:10132000772009F0AAC0592D21E04FC0F801808133
:10133000882309F0A4C0772009F0A1C0FD01E60FC1
:10134000F71F8A81803191F0EA0DFB1DEE0DFF1D24
:10135000DF01A452BC4F8C9183708C93E352FC4FFD
:1013600084E08083D2019C9330E08AC0EE0DFF1DA3
:10137000DF01AB5DBF4E8C918E7F8C93EA5DFF4E9B
:101380008081877080839C9111968C911197887FC2
:10139000846011968C931197917098619C9330E0C2
:1013A00021E0298311C0992379F4413069F4F201D5
:1013B0004083332331F4D8014C9320E0882009F492
:1013C00021E031E0772401C0592DEB81FC81EE0F43
:1013D000FF1F8B819C81E80FF91FEA0DFB1DEE0DAD
:1013E000FF1DE452FC4F80818C7F2170220F832BE4
:1013F000822B8083FB01EE0FFF1FE559F94C942FE0
:10140000990F990F80818B7F892B8083442311F45E
:10141000D8011C92FB01EE0FFF1FE559F94C8081AA
:10142000982F9170990F8D7F892B80836F5F7F4FED
:101430000F5F1F4F6031710511F0952E27CFB981D5
:10144000B093B90350934C02709245370F900F90B0
:101450000F900F90CF91DF911F910F91FF90EF9020
:10146000DF90CF90BF90AF909F908F907F906F90C4
:101470005F904F903F902F90089531E0A5CF31E0DD
:1014800021E0A2CF9F92AF92BF92CF92DF92EF92D4
:10149000FF920F931F93CF93DF935C010091B102F2
:1014A000402F50E02091352B30E0FA01E25BF44D03
:1014B00010811295107FA091B90360E070E085E281
:1014C0009DE0289FE001299FD00D389FD00D112469
:1014D0009924939484EC90E0489F6001499FD00C3C
:1014E000589FD00C11249BE3E92E9BE2F92EE40EC9
:1014F000F51EC501062E02C0969587950A94E2F75F
:10150000482F4170FB01EE0FFF1FE559F94C908108
:101510009E7F942B9083892F86958170481709F4BC
:1015200059C092FD4DC0413009F04AC0812F860F4D
:10153000282F30E090E0F901EE0FFF1FE20FF31FBC
:10154000EC0FFD1FEB5DFF4E808180FF91E0F90104
:10155000EE0FFF1FE20FF31F9F012C0F3D1FD9015C
:10156000AB5DBF4E8C918E7F892B8C93992339F57F
:10157000003189F0EC0DFD1DEC0FFD1FDF01A452C1
:10158000BC4F8C9183708C93E352FC4F84E080833A
:10159000F701908214C08E7F8C93F901EA5DFF4EB3
:1015A0008081877080839C9111968C911197887FA0
:1015B000846011968C931197917098619C93A1E02F
:1015C000FB01EE0FFF1FE559F94C440F80818D7F21
:1015D000842B80836F5F7F4F6031710509F089CF65
:1015E000A093B903DF91CF911F910F91FF90EF90DE
:1015F000DF90CF90BF90AF909F900895AF92BF9231
:10160000CF92DF92EF92FF920F931F93CF93DF93CE
:10161000EC01D0908B36D694D69481E0D822A0905D
:101620002C01C090392BB090F2024091F0335091D0
:10163000F13320E030E0E1E0EE2EF12C012D112D10
:10164000F901EE0FFF1FE559F94C6081CE01022E22
:1016500002C0969587950A94E2F7782F7170667F9D
:10166000962F972B9083892F86958170781709F490
:1016700053C092FD51C0713009F04EC06960608363
:10168000DD2031F1CC2081F0CA01022E02C09695F6
:1016900087950A94E2F780FD24C0AA24A394CC2461
:1016A000BB2440E050E038C0D801C701022E04C07E
:1016B000880F991FAA1FBB1F0A94D2F7AC0140954F
:1016C0005095AA24A394CC24C394BB24B39424C0DF
:1016D000CA01022E02C0969587950A94E2F780FF10
:1016E0000FC0D801C701022E04C0880F991FAA1F7E
:1016F000BB1F0A94D2F780959095482359230CC0BC
:10170000D801C701022E04C0880F991FAA1FBB1F52
:101710000A94D2F7482B592BF901EE0FFF1FE55918
:10172000F94C8081982F9170990F8D7F892B808340
:101730002F5F3F4F2031310509F082CFA0922C015D
:10174000C092392BB092F2025093F1334093F033B0
:10175000DF91CF911F910F91FF90EF90DF90CF908D
:10176000BF90AF90089581E060E070E00E9485082E
:10177000AC01909344378093433720E030E0CA01B6
:10178000022E02C0969587950A94E2F780FF02C068
:10179000822F08952F5F3F4F2031310581F78FEF62
:1017A000089581E060E070E00E948508AC019093AC
:1017B00042378093413760E020E030E0CA01022EDA
:1017C00002C0969587950A94E2F780FF05C06130C4
:1017D00011F4822F089561E02F5F3F4F20313105D2
:1017E00069F780E008953F924F925F926F927F92E7
:1017F0008F929F92AF92BF92CF92DF920F93DF931F
:10180000CF93CDB7DEB72C970FB6F894DEBF0FBEDF
:10181000CDBF382E462E8091352B90E0552425E201
:101820003DE0829FA001839F500D929F500D112497
:101830005C874B874F5D5F4E5A834983832D90E0D1
:10184000A0E0B0E08B839C83AD83BE83862F90E0C5
:10185000A0E0B0E08F839887A987BA8786C090E31D
:10186000491689F4852D90E0FC01EE0FFF1FE80F6B
:10187000F91FAB85BC85EA0FFB1FEB5DFF4E0081B6
:101880000E730E5F24C0852D90E0B0E64B1681F4F8
:10189000FC01EE0FFF1FE80FF91F4B855C85E40F7D
:1018A000F51FEB5DFF4E0081000F0C770C5F0FC042
:1018B000FC01EE0FFF1FE80FF91F8B859C85E80FD9
:1018C000F91FEB5DFF4E008106950F710F5F6B8175
:1018D0007C818D819E810E94288D5B016C016F81CE
:1018E000788589859A850E94288D3B014C01602F5F
:1018F00070E080E090E00E94288D9B01AC01C40163
:10190000B3010E948F8C9B01AC01C601B5010E94FE
:101910008F8C20E030E040E05FE30E94278C20E0E5
:1019200030E040E85FE30E94268C0E94FC8C90E34C
:10193000391611F4669505C0A0E63A1611F46695BD
:101940006695852D90E0FC01EE0FFF1FE80FF91F53
:101950004B855C85E40FF51FEB5DFF4E6F71660FE5
:101960008081817C862B80835394A981BA818C915C
:10197000851508F074CF1092B6031092B5032C961B
:101980000FB6F894DEBF0FBECDBFCF91DF910F91A0
:10199000DF90CF90BF90AF909F908F907F906F908F
:1019A0005F904F903F9008950F931F93CF93DF93D5
:1019B0009091352B092F10E0C82FD0E0FE01EE0FDB
:1019C000FF1FEC0FFD1F85E29DE0089FD001099FDE
:1019D000B00D189FB00D1124EA0FFB1FE95DFF4EFB
:1019E0008081482F429547708F70A15EBF4E2C9129
:1019F000680FE82FF0E0CF01861B91098130910537
:101A0000E1F430E0C901880F991F820F931F880FFE
:101A1000991F880F991FE80FF91FE355FC4F20E02D
:101A2000349102C0615021E0FC01E60FF11DE35545
:101A3000FC4FE4913E17B1F31DC08F5F9F4FC9F477
:101A400030E0C901880F991F820F931F880F991FDB
:101A5000880F991FE80FF91FE355FC4F249101C02F
:101A60006F5FFC01E60FF11DE355FC4FE4912E176B
:101A7000B9F320E06F3F19F4442319F412C06C301D
:101A800098F0473011F4222371F06F3F31F4442372
:101A900021F0415040F440E006C04F5F473008F06D
:101AA00047E060E001C06BE0FE01EE0FFF1FEC0FAE
:101AB000FD1F85E29DE09C01029FC001039F900DE8
:101AC000129F900D1124E80FF91FE95DFF4E6F7012
:101AD0008081807847704295407F862B842B80835D
:101AE000DF91CF911F910F9108951F920F920FB622
:101AF0000F920BB60F9211242F933F934F935F9346
:101B00008F939F93AF93BF93EF93FF9380B18170B7
:101B10008093333690913336809134369817B9F1EB
:101B200080913336882379F581E0809335361092A1
:101B30004E02ECE0F6E3819326E3ED31F207D9F7AC
:101B40002C9A2C9810924902109233011092320173
:101B500080E090E021E0FC01E05AFD4F1082FC01A2
:101B6000E752FD4F1082FC01EA54FD4F2083FC0137
:101B7000EE57FD4F1082FC01ED56FD4F208301967C
:101B80008131910541F780913336809334368091CD
:101B900048028370823009F0B8C080B190E095951A
:101BA00087958170809329369091293680917001B4
:101BB000981709F474C080917001882311F02C9A51
:101BC00001C02C9880912936882309F065C0809146
:101BD0001F3690912036A0912136B0912236209167
:101BE0002536309126364091273650912836821B73
:101BF000930BA40BB50B8093680190936901A0939C
:101C00006A01B0936B018091680190916901A09184
:101C10006A01B0916B01885E9340A040B04080F4AF
:101C20008091680190916901A0916A01B0916B0166
:101C300080936C0190936D01A0936E01B0936F013E
:101C400021E020932A3680911F3690912036A09172
:101C50002136B09122368093253690932636A09374
:101C60002736B09328368091AB028823C1F42093A5
:101C70002B362093710180916C0190916D01A091A0
:101C80006E01B0916F018093680190936901A093F8
:101C90006A01B0936B0103C081E080932D3680917F
:101CA0002936809370018091680190916901A0911B
:101CB0006A01B0916B01885E9340A040B04060F033
:101CC00088EE93E0A0E0B0E0809368019093690112
:101CD000A0936A01B0936B018091680190916901B2
:101CE000A0916A01B0916B01893C9105A105B105F4
:101CF00060F488EC90E0A0E0B0E0809368019093FD
:101D00006901A0936A01B0936B01FF91EF91BF91BC
:101D1000AF919F918F915F914F913F912F910F9034
:101D20000BBE0F900FBE0F901F901895E82F592FE4
:101D30004091F6353091F73520917A37222381F0A2
:101D4000213051F48DB380937C379DB380917B37E4
:101D5000809589238DBB04C08FB7F89480937C371E
:101D60004CBD3DBD5D985EBD00000DB407FEFDCFCE
:101D70008EB5EEBD00000DB407FEFDCF8EB57EBD65
:101D800000000DB407FEFDCF8EB56EBD00000DB492
:101D900007FEFDCF8EB55D9A222339F080917C3706
:101DA000213011F48DBB01C08FBF50935C36E0939E
:101DB0005B3670935A36609359360895682F592FC1
:101DC0004091F6353091F73520917A37222381F012
:101DD000213051F48DB380937C379DB380917B3754
:101DE000809589238DBB04C08FB7F89480937C378E
:101DF0004CBD3DBD5C985EBD00000DB407FEFDCF3F
:101E00008EB56EBD00000DB407FEFDCF8EB55C9A99
:101E1000222339F080917C37213011F48DBB01C031
:101E20008FBF509358366093573608954091F635DA
:101E30003091F73520917A37222381F0213051F407
:101E40008DB380937C379DB380917B3780958923B8
:101E50008DBB04C08FB7F89480937C374CBD3DBDDB
:101E60005C981EBC00000DB407FEFDCF8EB51EBCF5
:101E700000000DB407FEFDCF8EB55C9A222339F029
:101E800080917C37213011F48DBB08958FBF089568
:101E90009C013F7030616091F6355091F73540916B
:101EA0007A37442381F0413051F48DB380937C37ED
:101EB0009DB380917B37809589238DBB04C08FB7FC
:101EC000F89480937C376CBD5DBD12983EBD0000D8
:101ED0000DB407FEFDCF8EB52EBD00000DB407FE7C
:101EE000FDCF8EB5129A442339F080917C37413072
:101EF00011F48DBB08958FBF08958F3708F08FE7D9
:101F0000282F30E0F5E0220F331FFA95E1F73F70FC
:101F100030696091F6355091F73540917A37442316
:101F200081F0413051F48DB380937C379DB3809123
:101F30007B37809589238DBB04C08FB7F89480933D
:101F40007C376CBD5DBD12983EBD00000DB407FE30
:101F5000FDCF8EB52EBD00000DB407FEFDCF8EB5B2
:101F6000129A442339F080917C37413011F48DBBB3
:101F700008958FBF08959C013F7030616091F635E0
:101F80005091F73540917A37442381F0413051F434
:101F90008DB380937C379DB380917B378095892367
:101FA0008DBB04C08FB7F89480937C376CBD5DBD4A
:101FB00013983EBD00000DB407FEFDCF8EB52EBDBB
:101FC00000000DB407FEFDCF8EB5139A442339F0FF
:101FD00080917C37413011F48DBB08958FBF0895F7
:101FE0009C013F7030696091F6355091F735409112
:101FF0007A37442381F0413051F48DB380937C379C
:102000009DB380917B37809589238DBB04C08FB7AA
:10201000F89480937C376CBD5DBD13983EBD000085
:102020000DB407FEFDCF8EB52EBD00000DB407FE2A
:10203000FDCF8EB5139A442339F080917C3741301F
:1020400011F48DBB08958FBF08954091F6353091FE
:10205000F73520917A37222381F0213051F48DB366
:1020600080937C379DB380917B37809589238DBB8E
:1020700004C08FB7F89480937C374CBD3DBD5E9A09
:102080001EBC00000DB407FEFDCF8EB51EBC0000C7
:102090000DB407FEFDCF8EB580930A361EBC00003E
:1020A0000DB407FEFDCF8EB51EBC00000DB407FEBB
:1020B000FDCF8EB51EBC00000DB407FEFDCF8EB562
:1020C00080930836809309365E98222339F08091F8
:1020D0007C37213011F48DBB08958FBF08959C018A
:1020E00043B148704093F83593B194709093F935AB
:1020F000442311F58091FA358823F1F0992319F0E2
:10210000260F371F19C080918D3682FF10C0809135
:10211000EF01813041F0813010F0823069F42A30D3
:10212000310554F007C02031310534F003C02115CA
:10213000310511F0261B370B4093FA35C90108957C
:10214000482F53B152705093FE3593B191709093D4
:10215000FF355523D9F4809100368823B9F09923AF
:1021600069F08FEF90E0841B9109262F30E08217F1
:10217000930714F44FEF0AC0460F08C0461720F427
:10218000442321F0462F02C04111461B50930036D4
:10219000842F90E00895CF92DF92EF92FF920F93F9
:1021A0001F93CF93DF93EC01F42EE22E6801188188
:1021B00010931B37812F0E94A0108883F81608F017
:1021C000F88288818E1508F0E8828881811739F0BD
:1021D00080931B3781E0F601808380932C01DF918F
:1021E000CF911F910F91FF90EF90DF90CF900895C6
:1021F0000F931F93DF93CF930F92CDB7DEB78983F1
:102200008091352B90E025E23DE0829FF001839F95
:10221000F00D929FF00D1124E05EFF4E20812033DF
:1022200011F0203609F428E12150CE01019661E039
:1022300040E009EB13E00E94CB1069816093EB0250
:102240008091953683FF26C08091352B90E040E049
:1022500050E025E23DE0829FD001839FB00D929F28
:10226000B00D1124962F9F71990FFA01EE0FFF1FE9
:10227000E40FF51FEA0FFB1FEB5DFF4E8081817CB1
:10228000892B80834F5F5F4F4034510571F781E0A8
:102290008093B903862F0F90CF91DF911F910F91FB
:1022A00008951F93FC0113B112701093FE3593B182
:1022B00091709093FF35112361F58091003688234A
:1022C00041F19923D1F0CF01A0E0B0E02FEF3FEF33
:1022D00040E050E0281B390B4A0B5B0B862F90E047
:1022E000A0E0B0E0281739074A075B071CF4EFEFBE
:1022F000FFEF0FC0E60FF11D0CC070E0E617F70707
:1023000020F4309731F0FB0104C0309711F0E61B48
:10231000F70B10930036CF011F910895AF92BF9233
:10232000CF92DF92EF92FF920F931F93CF93DF93A1
:10233000EC01F42EE52EB22EA32E6801088119813E
:102340001093183700931737C8010E9451119C0150
:10235000998388838F2D9E2D8217930710F0998380
:1023600088832B2D3A2D888199818217930710F04D
:1023700039832883888199818017910749F0909348
:1023800018378093173781E0F601808380932C0102
:10239000DF91CF911F910F91FF90EF90DF90CF9041
:1023A000BF90AF9008959C0143B142704093FE35B9
:1023B00093B191709093FF35442309F580910036D5
:1023C0008823E9F070E0992369F08FEF9FE7821B83
:1023D000930B861797071CF42FEF3FE710C0260FCB
:1023E000371F0DC0261737072CF42115310539F09A
:1023F0009B0105C02115310511F0261B370B4093B9
:102400000036C9010895AF92BF92CF92DF92EF924A
:10241000FF920F931F93CF93DF93EC017A01690131
:1024200058010881198110931A3700931937C80190
:102430000E94D31199838883E816F90614F0F98273
:10244000E882888199818C159D0514F0D982C88213
:10245000888199818017910749F090931A3780936A
:10246000193781E0F501808380932C01DF91CF91B2
:102470001F910F91FF90EF90DF90CF90BF90AF90A2
:1024800008959F92AF92BF92CF92DF92EF92FF9208
:102490000F931F937B018C0159016A0193B082E075
:1024A00098229092FE3593B191709093FF359920C8
:1024B000D9F5809100368823B9F1992329F0C80114
:1024C000B7010E94278C2EC080918D3682FF1AC0E2
:1024D0008091EF01813059F0813010F0823021F588
:1024E000C801B70120E030E040E251E406C0C80175
:1024F000B70120E030E040E851E40E94DA8D882303
:102500009CF00AC0C801B70120E030E040E050E094
:102510000E948B8C882341F0C801B701A601950168
:102520000E94268C7B018C0190920036B701C80175
:102530001F910F91FF90EF90DF90CF90BF90AF90E1
:102540009F900895BF92CF92DF92EF92FF920F93E8
:102550001F93CF93DF93742F2091352B803109F097
:102560004EC030E0A0E0B0E085E29DE0289F700121
:10257000299FF00C389FF00C1124062F10E0C42F77
:10258000D0E0D42ED294DD0CDD0C30ECD322469575
:1025900046954770562F5295550F550F507C6695AE
:1025A00066956770FD01EE0FFF1FEA0FFB1FEE0D32
:1025B000FF1DEB5DFF4E2081922F9295969596958B
:1025C00093703181832F8770880F880F892B90E05B
:1025D0008017910734F42F73252B2083387F362BF7
:1025E00008C08C179D0734F02F732D292083387F66
:1025F000342B31831196A034B105A1F65CC0422F73
:1026000050E0A0E0B0E0282F30E084EC90E0289F7C
:102610006001299FD00C389FD00C112485E29DE0E9
:10262000489F7001499FF00C589FF00C1124062F11
:1026300010E0C72FD0E0B72EB294BB0CBB0C90ECCF
:10264000B922472F469546954770562F5295550FFC
:10265000550F507C669566956770FD01EE0FFF1F64
:10266000EA0FFB1FEC0DFD1DEE0DFF1DE452FC4FAC
:102670002081922F92959695969593703181832F14
:102680008770880F880F892B90E08017910734F4AA
:102690002F73252B2083387F362B08C08C179D077E
:1026A00034F02F732B292083387F342B31831196FC
:1026B000A034B10591F6DF91CF911F910F91FF905A
:1026C000EF90DF90CF90BF9008952F923F924F925E
:1026D0005F926F927F928F929F92AF92BF92CF92B2
:1026E000DF92EF92FF920F931F93DF93CF93CDB7BB
:1026F000DEB760970FB6F894DEBF0FBECDBFDE0128
:102700001196ECEAF1E080E101900D928150E1F741
:102710008091352B482F50E085E29DE0489FF001E5
:10272000499FF00D589FF00D1124E05EFF4ED080C0
:1027300080919B3683FF0DC080915E018F5F8093F7
:102740005E01883018F087E080935E0181E080931D
:102750002C018091993683FF0CC080915E018150DD
:1027600080935E01883010F010925E0181E08093CA
:102770002C0185E29DE0489FF001499FF00D589F94
:10278000F00D1124E15EFF4EE081E33018F4E130FA
:1027900048F405C0E33049F0E93048F403C0FCE0F8
:1027A0007F2E05C0E7E07E2E02C075E0772E809177
:1027B000AB02882309F44AC08091B002813009F04D
:1027C00045C08091B703882309F440C080918102FD
:1027D00090E0FC01EE0FFF1FE80FF91F85E29DE07E
:1027E000489F9001499F300D589F300D1124E20FF2
:1027F000F31FE95DFF4E909115379F708081807FB8
:10280000892B80838091810290E0FC01EE0FFF1FF5
:10281000E80FF91FE20FF31FE95DFF4E90915F0192
:1028200097709295907F80818F78892B808380919B
:10283000810290E0FC01EE0FFF1FE80FF91FE20F8D
:10284000F31FEB5DFF4E80818E7F8083C090163733
:1028500000911537EE24FF24472C552425E2822EC3
:102860002DE0922E91E0292E312C87E0682EF70181
:10287000EE0FFF1FE559F94C30818091B6369091EB
:10288000B7360E2C02C0969587950A94E2F7282F4A
:102890002170367F932F922B9083892F869581709C
:1028A000281709F404C192FDF6C0213009F0F3C0E5
:1028B00039603083E1E0F0E0EC0FFD1FEE0DFF1D0D
:1028C000E0818E2F90E0672D70E00E946C8E9B015E
:1028D00080915E01860F80935F01883010F06092D6
:1028E0005F01249DC001259D900D349D900D112404
:1028F0002E2F281B8091352B90E0889DF001899D1B
:10290000F00D989DF00D1124E15EFF4E8081833023
:1029100018F4813068F405C0833081F0893098F470
:1029200007C0E22FF0E0E355FC4FC490CA940BC0FF
:10293000E22FF0E0E759F54FC49005C0E22FF0E038
:10294000E059F54FC4904CE0849FF0011124EC0D48
:10295000F11DE355FC4F049101508091F53588231A
:1029600049F0080F0C3030F080915F018F5F809349
:102970005F010C50E02FF0E0EE0FFF1FE75EFB4F12
:102980008591949120915F01B22EBB0CAA248A0DEF
:102990009B1D0E94480F5F9A51E05093B7038091AE
:1029A000AB02882309F477C08091B002813009F02E
:1029B00072C08091352B482F50E08091700290E0DA
:1029C000FC01EE0FFF1FE80FF91F489D9001499D84
:1029D000300D589D300D1124E20FF31FE95DFF4EBD
:1029E000902F9F708081807F892B808380917002DF
:1029F00090E0FC01EE0FFF1FE80FF91FE20FF31F3D
:102A0000E95DFF4E90915F0197709295907F808174
:102A10008F78892B808388E1D816B9F08D1538F02E
:102A20009CE0D91671F0E0E1DE1691F40CC0F0E301
:102A3000DF1659F080E6D81651F090E2D91641F42D
:102A400006C01BE005C01FE003C017E101C01FE185
:102A50008091810290E0FC01EE0FFF1FE80FF91F4B
:102A6000489DC001499D900D589D900D1124E80F7F
:102A7000F91FEB5DFF4E912F9F71990F8081817C33
:102A8000892B8083E0918102F0E0EE0FFF1FE05977
:102A9000FC4C31822082F701EE0FFF1FE559F94C03
:102AA0008081982F9170990F8D7F892B8083089456
:102AB000E11CF11CE0E1EE16F10409F0D8CEC09261
:102AC0001637009315378091B6369091B736892B1B
:102AD00009F071C08091B703882309F46CC05F9836
:102AE0001092B7038091AB02882309F464C08091EF
:102AF000B002813009F05FC0F8E1DF16D9F0FD15B2
:102B000038F04CE0D41671F050E1D51651F50EC0F6
:102B100080E3D816D1F090E6D916F9F0E0E2DE169F
:102B200001F50FC080914E026CE007C010914E027B
:102B30001F7017C080914E0268E10E94608E192FAD
:102B400010C010914E021F710CC080914E0260E3C4
:102B50000E94608E192F169504C010914E02169592
:102B600016958091810290E02091352B30E0FC0198
:102B7000EE0FFF1FE80FF91F85E29DE0AC01249FD7
:102B8000C001259F900D349F900D1124E80FF91F6F
:102B9000EB5DFF4E1F71110F8081817C812B808343
:102BA000E0918102F0E0EE0FFF1FE059FC4C81E064
:102BB00090E091838083809170028823A9F5209111
:102BC000352B30E05091B90340E085E29DE0289F2D
:102BD000B001299F700D389F700D11248B010F5D7E
:102BE0001F4E1CC0242F30E0D901AA0FBB1FA059D3
:102BF000BC4C8D919C911197892B79F0F901EE0FC6
:102C0000FF1FE20FF31FE60FF71FEB5DFF4E808102
:102C1000816080831D921C9251E04F5FF80180819A
:102C2000481700F35093B90360960FB6F894DEBFCF
:102C30000FBECDBFCF91DF911F910F91FF90EF900D
:102C4000DF90CF90BF90AF909F908F907F906F90CC
:102C50005F904F903F902F900895CF93DF93C82FB0
:102C6000D0E060913E0270913F0280E090E00E94CF
:102C7000288DC854D94CEC89F0E0EE0FFF1FEE0F01
:102C8000FF1FE557FE4F20813181428153810E9411
:102C9000DE8D9B01AC0160E070E080E792E40E9471
:102CA0008F8C21E338E04CEA5CE30E948F8C0E9419
:102CB000FC8CCB016F3F710510F08EEF90E0819599
:102CC0008A83DF91CF9108953F924F925F926F92E6
:102CD0007F928F929F92AF92BF92CF92DF92EF92AC
:102CE000FF920F931F93CF93DF9390908B36969420
:102CF0009694AA24A3949A20992D990F80914B36EB
:102D00008C7FD0908D36D694D694DA20892B8D295D
:102D1000A090A336A694A694BB24B394AB202A2DEE
:102D2000220F220F837FB090A536B694B694CC24A0
:102D3000C394BC209B2D990F990F990F822B892B3F
:102D400040919136469546954170342F3295307FAB
:102D50008F7C20919936269526952170922F9295F9
:102D6000990F907E832B892B90919B369695969503
:102D70009170392F3295330F330F307C8F7B832B3B
:102D800080934B36022F10E0000F111F000F111F10
:102D9000692F70E093E0660F771F9A95E1F7C42FD3
:102DA000D0E085E0CC0FDD1F8A95E1F720914A360F
:102DB000922F96959270902B822F82958695817096
:102DC000982B962B269526952071292B2C2B20931A
:102DD0004336E0904602F090470221E0E216F1040B
:102DE00019F45091790109C0E114F10411F451E092
:102DF00005C050919536569556955170852F817026
:102E00008295880F807E90914A369F7D982B909373
:102E10004A36C7010397029720F04CE0E416F1040C
:102E200029F4C090790181E0C82207C0CC2492E047
:102E3000E916F10411F4CC24C3949C2D990F990F39
:102E400080914A368B7F892B80934A3624E0E216A4
:102E5000F10421F04CE0E416F10421F43091790101
:102E6000317007C03091AB3636953695317009F028
:102E700031E0932F9170990F990F990F80914A36F5
:102E8000877EB091A936B695B695B1702B2F229555
:102E9000207F892B822B80934A368091B002882331
:102EA00059F080914C36816080934C3690914C362D
:102EB0009170EBE3FBE220C08091382B882381F4F2
:102EC00080913702882361F48091B903882341F40B
:102ED0008091E736882321F48091F135882341F0F1
:102EE00090917901917080914C368E7F892BDCCF47
:102EF00080914C368E7FD8CF8081882319F09091B5
:102F00007901917031968BE2EB34F807A9F7809143
:102F10004C368E7F892B80934C3695E0E916F10470
:102F200021F480914A36806403C080914A368F7BB9
:102F300080934A36E091F033F091F133F0935136BB
:102F4000E093503628E0E216F104D9F48091F101C3
:102F5000823099F48091EF018250823070F481E0E8
:102F600090E00090B40202C0880F991F0A94E2F723
:102F700090933E3680933D3604C010923E361092B8
:102F80003D364091AB02A0E0442309F4A1E08091DA
:102F90004A368E7F8A2B80934A36442321F08091D3
:102FA0004B36806809C0909179019795992797953C
:102FB00080914B368F77892B80934B36602B712B0A
:102FC0006C2B7D2B80914A368295869586958170F3
:102FD00090E014E0880F991F1A95E1F7682B792B80
:102FE0008B2D90E026E0880F991F2A95E1F7682B3A
:102FF000792B8B2F90E09695982F8827979587951A
:10300000682B792B9A2D80E0682B792B992D990FBD
:10301000990F80E0682B792B9D2D990F990F990FAF
:1030200080E0682B792B20914B36221F2227221F0C
:10303000922F9295907F80E0682B792B20914C36CF
:103040002170922F9295990F990F907C80E0682BB8
:10305000792B9A2F9295990F907E80E0682B792B8F
:10306000852F90E0682B792B8C2D90E0880F991F8D
:10307000682B792B932F990F80E0682B792B709315
:103080004536609344363090B102C32DD0E021E044
:1030900030E0C901032C02C0880F991F0A94E2F79F
:1030A00090934E3680934D3655E0E516F10409F4C1
:1030B00065C266E0E616F104B4F472E0E716F104C6
:1030C00061F143E0E416F1041CF4F7FE4BC276C252
:1030D00053E0E516F10409F4EAC064E0E616F104F1
:1030E00009F06CC214C27CE0E716F10409F40FC2C7
:1030F0002DE0E216F1045CF447E0E416F10409F473
:10310000D6C059E0E516F10409F058C2D0C06FE00E
:10311000E616F1040CF052C2CAC08091953682FFC7
:1031200008C00090B20202C0220F331F0A94E2F7D7
:1031300020C2442309F46CC09091312B992309F4E7
:103140004BC08091322B482F50E04F70507060E0A0
:1031500070E020E030E0E92FF0E0B1E0EB2EF12C60
:10316000012D112D10C0C901840F951F5701680151
:1031700004C0AA0CBB1CCC1CDD1C8A95D2F76A29A2
:103180007B292F5F3F4FE217F3076CF7809179019E
:10319000FE01E658FE4FE081C15BDD4F288140E033
:1031A00050E0882311F441E050E08091B5028F7027
:1031B00002C0440F551F8A95E2F74095509564234D
:1031C00075238E2F90E02F7002C0880F991F2A95CB
:1031D000E2F7682779275AC040917901FE01E65845
:1031E000FE4F8081C15BDD4F288190E02F7002C0CF
:1031F000880F991F2A95E2F750E02091B5022F70B1
:1032000002C0440F551F2A95E2F784279527D2C1A3
:103210009091312B992309F43EC08091322B482F95
:1032200050E04F70507060E070E020E030E0E92F37
:10323000F0E0A1E0EA2EF12C012D112D10C0C90102
:10324000840F951F5701680104C0AA0CBB1CCC1C3D
:10325000DD1C8A95D2F76A297B292F5F3F4FE21741
:10326000F3076CF78091790120E030E0882311F4B6
:1032700021E030E08091B5028F7002C0220F331F31
:103280008A95E2F7209530956223732370933E363A
:1032900060933D3693C18091790190E02091B50211
:1032A0002F7002C0880F991F2A95E2F783C1DD2095
:1032B00009F080C1FE01E25BF44D9080892C82947C
:1032C00040EF84222091352B30E040E050E000E0D8
:1032D00010E060E070E084EC90E0C89F2001C99F9E
:1032E000500CD89F500C112485E29DE0289F30019E
:1032F000299F700C389F700C112431E0A32EB12C43
:10330000C12CD12C882D840F90E020E1321669F475
:10331000FC01EE0FFF1FE80FF91FE60DF71DEB5D37
:10332000FF4E808180FF3FC012C0FC01EE0FFF1FE7
:10333000E80FF91FE40DF51DE60DF71DE452FC4FF3
:103340008081982F917081FF0FC09923E1F0D60101
:10335000C501042E04C0880F991FAA1FBB1F0A9421
:10336000D2F7682B792B1FC0992369F0D601C501CC
:10337000042E04C0880F991FAA1FBB1F0A94D2F7FE
:10338000082B192B10C0D601C501042E04C0880FCC
:10339000991FAA1FBB1F0A94D2F7809590956823A6
:1033A0007923082319234F5F5F4F4034510509F0FB
:1033B000A9CF009341361093423660933F36709305
:1033C0004036FE01E15AF44D30819316B1F4FE010E
:1033D000E658FE4F8081FE01E15BFD4F208190E0C9
:1033E0002F7002C0880F991F2A95E2F7862797272A
:1033F00090933E3680933D3604C070933E36609382
:103400003D3680914F36883C08F19316B9F4FE01A1
:10341000E658FE4F8081C15BDD4F288190E02F7020
:1034200002C0880F991F2A95E2F780279127862BE3
:10343000972B90933E3680933D3606C0062B172B74
:1034400010933E3600933D3610924F3647E0E41617
:10345000F10429F059E0E516F10409F0AFC0992014
:10346000A1F480914C02803108F0A8C0209179012C
:1034700030E002C0220F331F8A95E2F780913D367B
:1034800090913E368227932795C061E0961679F495
:1034900020914C02203208F091C0203108F48EC0F7
:1034A0008091790190E030E02051304024C072E0FA
:1034B000971679F420914C02203308F07FC0203217
:1034C00008F47CC08091790190E030E020523040D7
:1034D00012C083E0981609F071C020914C0220348C
:1034E00008F06CC0203308F469C08091790190E045
:1034F00030E02053304002C0880F991F2A95E2F730
:1035000020913D3630913E362827392732C08091B0
:1035100048028370B9F081E060E070E00E948508A5
:103520002091A8023091A9024091473650E05901FC
:103530004A9D90014B9D300D5A9D300D1124282B32
:10354000392B17C0009148361091493681E060E070
:1035500070E00E948508082B192B10933E360093CB
:103560003D362CC00090F53302C0220F331F0A9461
:10357000E2F730933E3620933D3620C0809193365B
:1035800082FF12C08091790190E02091F233309156
:10359000F3336C01C29EC001C39E900DD29E900D6C
:1035A00011248E279F2706C0809148369091493676
:1035B0008E2B9F2B90933E3680933D366091443600
:1035C0007091453680913D3690913E36409143361C
:1035D0000E94960EDF91CF911F910F91FF90EF9077
:1035E000DF90CF90BF90AF909F908F907F906F9023
:1035F0005F904F903F900895EF92FF920F931F932B
:10360000CF93DF930091B10250E02091352BC62F6C
:10361000D0E0003109F073C030E0DA01AA0FBB1F1F
:10362000A40FB51F85E29DE0AC01249FC001259F3A
:10363000900D349F900D1124A80FB91FBD016B5D33
:103640007F4EFE01EE0FFF1FEC0FFD1FE80FF91F6D
:103650008F010B5D1F4EE80198819170EB0188810D
:103660008E7F892B8883AD01495D5F4E9F01295D67
:103670003F4EE90198819F70EA018881807F892B04
:103680008883E901988190778F78892BEA01888374
:10369000E901988190788F77892BEA018883E80186
:1036A00098819E73EB018881817C892B8883AA5D38
:1036B000BF4EEA5DFF4E9081987F8C918770892B79
:1036C0008C93F8018081829586958695837091818F
:1036D0009770990F990F982B292F2295220F220F5F
:1036E000207C88818F73822B88839695969589811B
:1036F000887F892B898381E08093B90375C010E0AE
:1037000030E0E82EFF24DA01AA0FBB1FA40FB51F7B
:1037100064EC70E0069FC001079F900D169F900D0E
:103720001124A80FB91F85E29DE0A901489F9001CF
:10373000499F300D589F300D1124A20FB31FAD01CA
:1037400044525C4FFE01EE0FFF1FEC0FFD1FE69E83
:10375000C001E79E900DF69E900D1124E80FF91F11
:10376000E20FF31FBF0164527C4FEB01988191700F
:10377000EA0188818E7F892B8883EB019881927082
:103780008D7F892BEA018883EB0198819C73837C70
:10379000892BEA018883EB012881229526952695BD
:1037A000237099819770990F990F922B292F229549
:1037B000220F220F207C8F73822BEA01888396953B
:1037C00096958981887F892B8983A352BC4FE352C8
:1037D000FC4F9081987F8C918770892B8C93055C2E
:1037E000144D81E0F8018083DF91CF911F910F91FB
:1037F000FF90EF900895DF92EF92FF920F931F9347
:10380000CF93DF932091352B803109F471C0422F83
:1038100050E0282F30E084EC90E0289FB001299FF1
:10382000700D389F700D112485E29DE0DA01A89F8C
:10383000A001A99F500DB89F500D1124DB01A40FCA
:10384000B51FAE53BC4FA652BF4F0D91FB01E45FB5
:10385000F14EE652FF4F01938C918083329612967F
:103860008C9180838E918293FA01EE53FC4FE20F8C
:10387000F31F8781245F314EF901878310E07B01BC
:10388000EA01812F90E0FC01EE0FFF1FE80FF91F06
:10389000EE0DFF1DBF016A5D714E9F012C0F3D1F94
:1038A000D901A452BC4F9C91492F4295469546950B
:1038B000437011968C918770880F880F842B482F46
:1038C0004295440F440F407C9F73942BDB019C93E3
:1038D00086958695E95DF14E23523C4FD9019C9126
:1038E000987F8770892B80831F5F011750F679C0FE
:1038F00030E085E29DE0F901E89F9001E99F300DFD
:10390000F89F300D1124F901EE53FC4FE15AF34FAB
:10391000D080D0926B2A829180936A2A32968191CC
:1039200080936C2A808180936D2A34978081809364
:10393000692A00E0E901802F90E0DC01AA0FBB1F9B
:10394000A80FB91F9D012159354DBD016C0F7D1F79
:10395000E5E2EE2EE0E1FE2EE60EF71EF701108105
:10396000912F9170F90180818E7F892B8083AD0129
:103970004F58554DFB01E95DFF4E8081FA01808370
:10398000912F9E73F9018081817C892B8083A059BE
:10399000B54D6A5D7F4EFB019081987F8C91877059
:1039A000892B8C931295169516951370D701119645
:1039B0009C919770990F990F912B492F4295440F25
:1039C000440F407CF90180818F73842B808396950E
:1039D00096958181887F892B81830F5FD01608F0AF
:1039E000AACFDF91CF911F910F91FF90EF90DF90C1
:1039F00008959F92AF92BF92CF92DF92EF92FF9283
:103A00000F931F93CF93DF932091352B803109F4CF
:103A100081C0422F50E0C82FD0E0262F30E084EC48
:103A200090E0289F7001299FF00C389FF00C112422
:103A3000D701A45FB14EA652BF4F9D90C89FB00161
:103A4000C99F700DD89F700D112485E29DE0FA0189
:103A5000E89FA001E99F500DF89F500D1124FB0134
:103A6000E40FF51FEE53FC4FE652FF4F91928C91FD
:103A70008083329612968C9180838E918293FA0184
:103A8000EE53FC4FEC0FFD1F245F314ED90117960A
:103A90008C91878300E05B016A01802F90E0FC013C
:103AA000EE0FFF1FE80FF91F9F012A0D3B1D2C0D84
:103AB0003D1DB90164527C4FEE0DFF1DDF01AA5D73
:103AC000B14E9C91492F429546954695437011966B
:103AD0008C918770880F880F842B482F4295440F54
:103AE000440F407C9F73942BDB019C9386958695B5
:103AF00023523C4FE95DF14E9081987F8770892B6E
:103B0000F90180830F5F901640F6C55CD44D81E0CB
:103B100088837EC030E0D0906B2A85E29DE0A901C9
:103B2000489F9001499F300D589F300D1124F90195
:103B3000EE53FC4FE15AF34FD08280916A2A829370
:103B4000329680916C2A819380916D2A808334977C
:103B50008091692A808300E0E901802F90E0DC01F8
:103B6000AA0FBB1FA80FB91FBD016C0F7D1F9B01C2
:103B70002B5D3F4E1FE6E12E1AE2F12EEA0EFB1EF0
:103B8000F7011081912F9170F90180818E7F892B2F
:103B90008083AB01495D5F4EFD01EF58F54D80819B
:103BA000FA018083912F9E73F9018081817C892B9A
:103BB00080836A5D7F4EA059B54D9C91987FDB0153
:103BC0008C918770892B8C9312951695169513708E
:103BD000F70191819770990F990F912B492F429579
:103BE000440F440F407CD9018C918F73842B8C93AC
:103BF0009695969511968C911197887F892B1196A1
:103C00008C930F5FD01608F0A8CF81E08093B903A2
:103C100081E080932C01DF91CF911F910F91FF9054
:103C2000EF90DF90CF90BF90AF909F900895CF938B
:103C3000DF932091352B30E0C82FD0E084EC90E06A
:103C4000C89FA001C99F500DD89F500D112485E237
:103C50009DE0B901689F9001699F300D789F300DFC
:103C60001124FA01E20FF31FEE53FC4FE652FF4F0F
:103C70008FE0819388E18083329681E08083129285
:103C800060E070E0FB01EE0FFF1FE60FF71FE40F8F
:103C9000F51FE20FF31FDF01A452BC4F82E08C93AB
:103CA000E352FC4F84E080836F5F7F4F6034710587
:103CB00049F7C55CD44D81E0888380932C01DF9166
:103CC000CF910895CF93DF938091352B90E025E23B
:103CD0003DE0A901849F9001859F300D949F300D98
:103CE0001124F901EE53FC4FE15AF34F8FE080832A
:103CF00088E18293329681E081931082349710821A
:103D000040E050E0B901FA01EE0FFF1FE40FF51F8C
:103D1000E60FF71FDF01AB5DBF4E8C918E7F8C935A
:103D2000CF01895D9F4E20E3EC0128838C91817C3B
:103D300088618C93EA5DFF4E8081877080838C91CF
:103D40008F738C9311968C911197887F8460119654
:103D50008C934F5F5F4F40345105A9F681E080930B
:103D6000B90380932C01DF91CF9108951F9310E048
:103D7000812F0E94FB1B1F5F1131D1F78091B83654
:103D80008093CF368091BA368093D1368091BC36FD
:103D90009091BD36A091BE36B091BF368093D33698
:103DA0009093D436A093D536B093D6368091CA3648
:103DB0008093E1368091CC368093E3368091B9369A
:103DC0008093D0368091BB368093D2368091C036B6
:103DD0009091C136A091C236B091C3368093D73648
:103DE0009093D836A093D936B093DA368091CB36FB
:103DF0008093E2368091CD368093E4361F9108950A
:103E00001F9310E0812F612F0E94F91C1F5F113159
:103E1000C9F78091CF368093B8368091D1368093A0
:103E2000BA368091D3369091D436A091D536B091E0
:103E3000D6368093BC369093BD36A093BE36B093F1
:103E4000BF368091E1368093CA368091E336809305
:103E5000CC368091D0368093B9368091D23680931B
:103E6000BB368091D7369091D836A091D936B09193
:103E7000DA368093C0369093C136A093C236B093A1
:103E8000C3368091E2368093CB368091E4368093BE
:103E9000CD3681E08093E7361F9108951F9310E09F
:103EA000812F0E94171E1F5F1031D1F70E94621EE2
:103EB0001F9108958F929F92BF92CF92DF92EF92BF
:103EC000FF920F931F93CF93DF93382FB42E20913F
:103ED000352B803161F430E0F62E85E29DE0289F9D
:103EE0006001299FD00C389FD00C1124E5C0822F8F
:103EF00090E0062F832E992424EC30E0829E60010E
:103F0000839ED00C929ED00C112425E23DE0829F2E
:103F10007001839FF00C929FF00C112458C0202F49
:103F200030E0802F8F7090E0D901AA0FBB1FA20F45
:103F3000B31FAC0DBD1DAE0DBF1DAD0144525C4F96
:103F4000FC01EE0FFF1FE80FF91FEC0DFD1DEE0D3C
:103F5000FF1DBF0164527C4FEB0198819170EA0113
:103F600088818E7F892B8883EB01988192708D7F69
:103F7000892BEA018883EB0198819C73837C892BD0
:103F8000EA018883EB0128812295269526952370E6
:103F900099819770990F990F922B292F2295220FB3
:103FA000220F207C8F73822BEA0188839695969549
:103FB0008981887F892B8983A352BC4FE352FC4FB0
:103FC0009081987F8C918770892B8C930F5FB016AE
:103FD00008F0A5CFEBE3FBE28E0E9F1E81E0E4012B
:103FE000888370C02F2D30E08F2D8F7090E0D90125
:103FF000AA0FBB1FA20FB31FAC0DBD1DBD016B5D92
:104000007F4EFC01EE0FFF1FE80FF91FEC0DFD1DA9
:104010008F010B5D1F4EE80198819170EB01888143
:104020008E7F892B8883AD01495D5F4E9F01295D9D
:104030003F4EE90198819F70EA018881807F892B3A
:104040008883E901988190778F78892BEA018883AA
:10405000E901988190788F77892BEA018883E801BC
:1040600098819E73EB018881817C892B8883AA5D6E
:10407000BF4EEA5DFF4E9081987F8C918770892BAF
:104080008C93F801808182958695869583709181C5
:104090009770990F990F982B292F2295220F220F95
:1040A000207C88818F73822B888396959695898151
:1040B000887F892B8983F394BF1408F093CF81E024
:1040C0008093B90381E080932C01DF91CF911F9100
:1040D0000F91FF90EF90DF90CF90BF909F908F90C7
:1040E00008952F923F925F926F927F928F929F924C
:1040F000AF92BF92CF92DF92EF92FF920F931F93F6
:10410000CF93DF932091352B803109F0EFC0822EC1
:10411000992485E29DE0889E9001899E300D989EAD
:10412000300D1124F901EF5DFF4E7080D901AB5DB8
:10413000BF4E9C91662463946922F901E95DFF4EAC
:104140008081EFE05E2E5822E82EE2947FE0E722A5
:1041500047E0E422A82EAA1CAA24AA1CD92ED69491
:104160008FE1D822F901EA5DFF4EB080B694B69493
:10417000B69492959695969593701196FC90F4222C
:10418000FF0CFF0CF92ACC24C394190166C02C2D16
:1041900030E0C9010197AC01440F551F480F591F6A
:1041A000420D531DBA016B5D7F4ED901AA0FBB1F93
:1041B000A20FB31FA20DB31D8D010B5D1F4EE801B1
:1041C00098819170FB0180818E7F892B80839A0179
:1041D000295D3F4EFD01E95DFF4E90819F70E90131
:1041E0008881807F892B8883908190778F78892B35
:1041F0008883908190788F77892B8883F8018081DC
:10420000829586958695837091819770990F990F05
:10421000982B292F2295220F220F207CEB018881D9
:104220008F73822B8883969596958981887F892BB9
:1042300089834A5D5F4EAA5DBF4E9C91987FFA01CB
:1042400080818770892B8083E80198819E73FB01B0
:104250008081817C892B8083C3947C1408F097CF64
:10426000872D90E0FC01EE0FFF1FE80FF91F85E29C
:104270009DE09C01829EC001839E900D929E900DB8
:104280001124E80FF91FDF01AB5DBF4E8C918E7FCB
:1042900086298C93CF01895D9F4E37E0E322E2941B
:1042A00010EFE122A794AA24A794E528EA28EC01BC
:1042B000E8829F2D9295990F990F907C8C918F7326
:1042C000892B8C93EA5DFF4EBB0CBB0CBB0CF694A8
:1042D000F694FB28F082EFE1DE22DD0C8C91817CEC
:1042E0008D298C9381E08093B903DCC0622E772402
:1042F000282E332484EC90E0289EA001299E500DA6
:10430000389E500D112485E29DE0689E9001699EC3
:10431000300D789E300D1124DA01A20FB31FFD017C
:10432000E456FB4FC080FD01E452FC4F80815524D0
:1043300053945822082F06950170F82EF694F6949F
:104340009FE0F9228295869586958370118117707A
:10435000110F110F182BA352BC4FDC90D694D6949A
:10436000D694EE24E3944A01590157C02E2D30E033
:10437000C9010197DC01AA0FBB1FA80FB91FA80D27
:10438000B91DAA0DBB1DAD0144525C4FF901EE0FE2
:10439000FF1FE20FF31FE80DF91DEA0DFB1DBF0122
:1043A00064527C4FEB0198819170EA0188818E7F85
:1043B000892B8883EB01988192708D7F892BEA018C
:1043C0008883EB0198819C73837C892BEA01888325
:1043D000EB01288122952695269523709981977067
:1043E000990F990F922B292F2295220F220F207CB3
:1043F0008F73822BEA018883969596958981887FB1
:10440000892B8983A352BC4FE352FC4F9081987F44
:104410008C918770892B8C93E394CE1408F0A6CFEF
:104420008C2D90E0FC01EE0FFF1FE80FF91F84ECCC
:1044300090E09C01229EC001239E900D329E900D23
:104440001124E80FF91F85E29DE0EC016C9EC0018C
:104450006D9E900D7C9E900D1124E80FF91FDF01D9
:10446000A452BC4F0170000F02702FE0F222FF0C2B
:10447000FF0C0529812F8295880F880F807C0F29DA
:10448000082B0C93E352FC4FDD0CDD0CDD0C169574
:1044900016951D2910838BE39BE2280E391E81E0BF
:1044A000E10188838091460290914702893091050D
:1044B00011F0079719F481E080932C01DF91CF91DF
:1044C0001F910F91FF90EF90DF90CF90BF90AF9032
:1044D0009F908F907F906F905F903F902F90089566
:1044E0002F923F924F925F926F927F928F929F9204
:1044F000AF92BF92CF92DF92EF92FF920F931F93F2
:10450000DF93CF93CDB7DEB728970FB6F894DEBF11
:104510000FBECDBF4091352B803109F009C1442E2B
:10452000552485E29DE0489EA001499E500D589E6D
:10453000500D1124FA01EF5DFF4E208130E0F901AA
:10454000EE0FFF1FE20FF31FE40FF51FBF016B5DBE
:104550007F4EDB019C91662463946922DF01A95D93
:10456000BF4E8C91B82FBF70BA83782E771C7724FA
:10457000771CE82EE294AFE0EA2217E0E122B92EA0
:10458000B6948FE1B822EA5DFF4EA080A694A6946F
:10459000A6949295969596959370DB011196FC9052
:1045A000F122FF0CFF0CF92A1C821B826901160103
:1045B0000894210831084A0174C0C601EB81FC81CE
:1045C0008E1B9F0B9C01220F331F280F391F280DB4
:1045D000391DB9016B5D7F4EDA01AA0FBB1FA40F15
:1045E000B51FA80DB91D8D010B5D1F4EF8019081FF
:1045F0009170FB0180818E7F892B8083A901495DA9
:104600005F4ECD01895D9F4E9E838D83FC0190811D
:104610009F70FA018081807F892B8083ED81FE81EC
:10462000908190778F78892BFA018083ED81FE81CC
:10463000908190788F77892BFA018083F8018081AF
:10464000829586958695837091819770990F990FC1
:10465000982B492F4295440F440F407CFB018081E9
:104660008F73842B8083969596958181887F892B83
:1046700081832A5D3F4EAA5DBF4E9C91987FD901F0
:104680008C918770892B8C93F80190819E73DB014C
:104690008C91817C892B8C93EB81FC813196FC83FE
:1046A000EB83A1012B813C81421B530B2C153D0553
:1046B00009F083CF85E29DE0489EA001499E500D00
:1046C000589E500D1124DA01AB5DBF4E8C918E7F48
:1046D00086298C93CA01895D9F4E37E0E322E294DC
:1046E00020EFE222779477247794EA81EE2AE72874
:1046F000FC01E0829F2D9295990F990F907C8C91EF
:104700008F73892B8C934A5D5F4EAA0CAA0CAA0C5E
:10471000F694F694FA28FA01F082FFE1BF22BB0C6E
:104720008C91817C8B298C9381E08093B903FBC0B1
:10473000242E3324A82EBB2484EC90E0A89EB00144
:10474000A99E700DB89E700D112485E29DE0289EF3
:10475000A001299E500D389E500D1124FB01E40F3D
:10476000F51FE456FB4F208130E0F901EE0FFF1FEB
:10477000E20FF31FE60FF71FE40FF51F1CEDC12E2C
:1047800013E0D12ECE0EDF1ED6018C91B82FB17062
:10479000B983082F06950170F82EF694F6941FE061
:1047A000F1228295869586958370D60111961C918B
:1047B0001770110F110F182BE352FC4FE080E69495
:1047C000E694E6941C821B82690126010894410844
:1047D00051083B014A0164C0C601EB81FC818E1B7C
:1047E0009F0B9C01220F331F280F391F260D371DE9
:1047F000280D391D38872F83A90144525C4FFB01D6
:10480000EE0FFF1FE60FF71FE60DF71DE80DF91D70
:10481000BF0164527C4FDB019C919170DA018C9155
:104820008E7F892B8C93DB019C9192708D7F892BDD
:10483000DA018C93DB019C919C73837C892BDA01D8
:104840008C93DB012C912295269526952370119649
:104850009C919770990F990F922B292F2295220FD7
:10486000220F207C8F73822BDA018C93969596957C
:1048700011968C911197887F892B11968C93AF811B
:10488000B885A352BC4FE352FC4F9081987F8C9126
:104890008770892B8C93EB81FC813196FC83EB83B1
:1048A000B2012B813C81621B730B2C153D0509F075
:1048B00093CF84EC90E0A89EF001A99EF00DB89EE5
:1048C000F00D112485E29DE0DC012A9EC0012B9EA3
:1048D000900D3A9E900D1124E80FF91F9F0124526C
:1048E0003C4F0170000F0270BFE0FB22FF0CFF0C79
:1048F0008981082B812F8295880F880F807C0F2952
:10490000082BD9010C93E352FC4FEE0CEE0CEE0C8D
:10491000169516951E291083EBE3FBE2AE0EBF1E23
:1049200081E0D5018C9380914602909147028930B5
:10493000910511F0079719F481E080932C012896D6
:104940000FB6F894DEBF0FBECDBFCF91DF911F91A0
:104950000F91FF90EF90DF90CF90BF90AF909F901E
:104960008F907F906F905F904F903F902F90089521
:10497000CF93DF936F5F2091352B8031B9F530E015
:1049800085E29DE0289FA001299F500D389F500D82
:10499000112429C0862F90E0FC01EE0FFF1FE80FC5
:1049A000F91FE40FF51FDF01AB5DBF4E8C918E7FC9
:1049B0008C93CF01895D9F4E20E3EC0128838C917D
:1049C000817C88618C93EA5DFF4E80818770808353
:1049D0008C918F738C9311968C911197887F846042
:1049E00011968C936F5F6034A8F22EC0422F50E076
:1049F000282F30E084EC90E0289FE001299FD00D23
:104A0000389FD00D112485E29DE0489F9001499F79
:104A1000300D589F300D112415C0862F90E0FC01F9
:104A2000EE0FFF1FE80FF91FEC0FFD1FE20FF31F42
:104A3000DF01A452BC4F82E08C93E352FC4F84E030
:104A400080836F5F603448F3DF91CF910895CF93F7
:104A5000DF938091352BC82FD0E085E29DE09C014B
:104A6000C29FC001C39F900DD29F900D1124FC01E5
:104A7000EE53FC4F108270914D2BDC01A456BB4FBE
:104A800020E030E060E09C918081891708F49083F9
:104A900011969C9111978C91989FA0011124241735
:104AA000350710F0A90101C0762F6F5FAC53BF4FDF
:104AB000603111F09A01E7CF70934D2B85E29DE0B4
:104AC000C89FF001C99FF00DD89FF00D1124EE533F
:104AD000FC4FE15AF34F9081EF55FC4080818917DC
:104AE00008F4908385E29DE0C89FF001C99FF00D16
:104AF000D89FF00D1124EE53FC4FDF01A15AB34FA4
:104B0000E25AF34F80812C91829FC00111244817F3
:104B1000590718F480E180934D2BDF91CF910895D0
:104B2000DF92EF92FF920F931F93CF93DF938091C9
:104B3000352B90E025E23DE0829FF001839FF00D50
:104B4000929FF00D1124EE53FC4F1182C0E0D0E093
:104B5000E4ECEE2EF12C05E21DE0DD24D3944C2F85
:104B60008091352B282F30E0CE9DF001CF9DF00DA8
:104B7000DE9DF00D1124209FC001219F900D309FDC
:104B8000900D1124E80FF91FE356FB4FE081DC0183
:104B9000AE53BC4F11968C9111978E1710F411964D
:104BA000EC93FE01EA54FD4FD082CE9DF001CF9DE3
:104BB000F00DDE9DF00D1124209FC001219F900D6E
:104BC000309F900D1124E80FF91FE456FB4F842FFE
:104BD00060810E94B8242196C031D10509F0BFCF71
:104BE0008091352B282F30E085E29DE0289FF00151
:104BF000299FF00D389FF00D1124EE53FC4FE25A1F
:104C0000F34F9081EE55FC408181891708F4918320
:104C100081E08093C60285E29DE0289FF001299FF4
:104C2000F00D389FF00D1124EF5DFF4E80E16081A3
:104C30000E94B8240E9427255F981092EA02DF9113
:104C4000CF911F910F91FF90EF90DF9008951F93E8
:104C50008091973683FF0FC01091F5331093003782
:104C60000E94B30B8093F533811729F081E0809384
:104C7000F03580932C011F91089580914802837034
:104C800090E0009719F0039754F523C060913E021D
:104C900070913F0280E090E00E94288D20E030E09B
:104CA00040EC52E40E94DE8D20E030E040E752E428
:104CB0000E948F8C9B01AC0160E074E284EF99E468
:104CC0000E948F8C0E94FC8C7093890060938800F6
:104CD000089584EF91E0909389008093880008956F
:104CE000E1E8F0E0108280818093800080818A601A
:104CF00080830E943D26EFE6F0E080818260808321
:104D00000895CF92EF920F938130910509F04CC036
:104D10006F5F7F4F09F071C086EF91E060E071E056
:104D20000E94DA8A8DEF91E060E071E00E94DA8AF9
:104D300084E092E060E071E00E94DA8A8BE092E029
:104D400060E071E00E94DA8A82E192E060E071E066
:104D50000E94DA8A89E192E060E071E00E94DA8ADA
:104D600080E292E060E071E00E94DA8A87E292E0FD
:104D700060E071E00E94DA8A8EE292E060E071E029
:104D80000E94DA8A80E58093F6351092F7358BEE33
:104D900096E362E143E124E105E1A6E1EA2EF7E1D1
:104DA000CF2E0E94BB7F29C0892B39F56F5F7F4FC3
:104DB00021F58EE292E00E941A8C87E292E00E9436
:104DC0001A8C80E292E00E941A8C89E192E00E94A3
:104DD0001A8C82E192E00E941A8C8BE092E00E9491
:104DE0001A8C84E092E00E941A8C8DEF91E00E9470
:104DF0001A8C86EF91E00E941A8C0F91EF90CF9061
:104E0000089580E090E06FEF7FEF0E948126089583
:104E100081E090E06FEF7FEF0E94812608950E946D
:104E2000B38520916736309168364091693650914C
:104E30006A36621B730B840B950B66307105810516
:104E4000910508F470C00E94B38560936736709333
:104E500068368093693690936A364091F635309182
:104E6000F73520917A37222381F0213051F48DB328
:104E700080937C379DB380917B37809589238DBB50
:104E800004C08FB7F89480937C374CBD3DBD5E9ACB
:104E90001EBC00000DB407FEFDCF8EB580935D36BD
:104EA0001EBC00000DB407FEFDCF8EB580935F36AB
:104EB0001EBC00000DB407FEFDCF8EB58093613699
:104EC0001EBC00000DB407FEFDCF8EB58093633687
:104ED0001EBC00000DB407FEFDCF8EB58093653675
:104EE0005E98222339F080917C37213011F48DBBFC
:104EF00001C08FBF93B190729093FB35EDE5F6E35F
:104F0000A2E5B6E320818181281709F42C9332961B
:104F1000119686E3E736F807A9F78091FC359817D4
:104F200011F49093FD354091F6353091F73520918D
:104F30007A37222381F0213051F48DB380937C376E
:104F40009DB380917B37809589238DBB04C08FB73B
:104F5000F89480937C374CBD3DBD5E9A1EBC00002A
:104F60000DB407FEFDCF8EB580935E361EBC0000EB
:104F70000DB407FEFDCF8EB5809360361EBC0000D9
:104F80000DB407FEFDCF8EB5809362361EBC0000C7
:104F90000DB407FEFDCF8EB5809364361EBC0000B5
:104FA0000DB407FEFDCF8EB5809366365E98222342
:104FB00039F080917C37213011F48DBB01C08FBF57
:104FC00083B180728093FC350895CF93DF93EC0119
:104FD0008881877E888320E0672B09F021E0988113
:104FE0009E7F922B9883892F86958170281701F1D7
:104FF00092FD0EC0213061F4986098830E94B385C1
:1050000060937637709377378093783790937937BA
:10501000888182FF05C080FD03C080618F7D888309
:105020008881982F9170990F990F8B7F892B888396
:10503000888182FF18C080FF16C00E94B38520912E
:105040007637309177374091783750917937621BB6
:10505000730B840B950B695E73408040904018F091
:105060008881806288838881982F9170990F8D7FC5
:10507000892B8883DF91CF910895DF92EF92FF9281
:105080000F931F93CF93DF930E940F27E090543626
:10509000D09056360091553610E0B80164707070AB
:1050A0008BE896E30E94E527B801687070708DE880
:1050B00096E30E94E527B8016170707083EA96E379
:1050C0000E94E527FF24B7016270707081EA96E3C1
:1050D0000E94E527027010708BEA96E3B8010E94E7
:1050E000E527B7016470707089E996E30E94E527AF
:1050F000B701687070708BE996E30E94E527B701ED
:105100006078707089EA96E30E94E527CD2DD0E0A3
:10511000BE01617070708DEA96E30E94E527BE01C2
:10512000627070708FEA96E30E94E527B7016072A3
:10513000707081E996E30E94E527B7016074707092
:1051400085EA96E30E94E527B7016071707083E9F4
:1051500096E30E94E52721E0E222FF2485E996E319
:10516000B7010E94E527BE01607270708DE996E379
:105170000E94E527BE01607170708FE996E30E947E
:10518000E5277091533660E08091523690E0682BAD
:10519000792B87E996E30E94E52720918F36D695F3
:1051A000C795D695C795CE018170682F267E922F20
:1051B000982B90938F36892F86958170681729F1E7
:1051C00092FD0FC0613069F4296020938F360E94F0
:1051D000B3856093B1367093B2368093B3369093B3
:1051E000B43680918F3682FF06C080FD04C0806196
:1051F0008F7D80938F3680918F36982F9170990F85
:10520000990F8B7F892B80938F3680918F36982FC3
:105210009170990F8D7F892B80938F3682FF18C0F4
:105220000E94B3852091B1363091B2364091B336A9
:105230005091B436621B730B840B950B695E7340FF
:105240008040904028F080918F36806280938F3626
:1052500020E030E0F901EE0FFF1FE559F94C8081A5
:10526000877E80832F5F3F4F2031310599F7DF9193
:10527000CF911F910F91FF90EF90DF9008951F93B2
:10528000CF93DF93182F883038F1599AC82FD0E088
:105290008091352B90E025E23DE0829FF001839FD5
:1052A000F00D929FF00D1124EE53FC4FEC0FFD1FFB
:1052B0008781882311F48FE301C084E10E947D0F70
:1052C00082B1C85ADE4F8F719881892B82B988E2EA
:1052D00090E00E941A86599888E290E00E941A860F
:1052E000599A183038F5149AC12FD0E08091352B97
:1052F00090E025E23DE0829FF001839FF00D929FB8
:10530000F00D1124EE53FC4FEC0FFD1F8781882315
:1053100011F48FE301C084E10E947D0F82B1C05A75
:10532000DE4F8F719881892B82B988E290E00E94CC
:105330001A86149888E290E00E941A86149ADF91E7
:10534000CF911F9108950F931F93CF93DF93C8E0E0
:10535000D0E005E21DE0599A8091352B90E0809FC6
:10536000F001819FF00D909FF00D1124EE53FC4F42
:10537000EC0FFD1F8781882311F48FE301C084E1C6
:105380000E947D0F82B18F71FE01E85AFE4F90811D
:10539000892B82B988E290E00E941A86599821965A
:1053A000CC30D105C1F688E290E00E941A86599A65
:1053B000C0E0D0E005E21DE0149A8091352B90E02A
:1053C000809FF001819FF00D909FF00D1124EE530E
:1053D000FC4FEC0FFD1F8781882311F48FE301C080
:1053E00084E10E947D0F82B18F71FE01E05AFE4F71
:1053F0009081892B82B988E290E00E941A861498E5
:105400002196C830D105C1F688E290E00E941A8644
:10541000149ADF91CF911F910F910895CF92DF924F
:10542000EF92FF920F931F93CF93DF938C01C8E00D
:10543000D0E0F4ECCF2ED12CE5E2EE2EEDE0FE2E06
:10544000C8010C2E02C0969587950A94E2F780FF5A
:105450005EC0599AFE01E15BFD4F808190E0209192
:10546000352B30E0FC01EE0FFF1FE80FF91FCC9D3C
:10547000C001CD9D900DDC9D900D1124E80FF91F0A
:105480002E9DC0012F9D900D3E9D900D1124E80F83
:10549000F91FE452FC4F808181FD02C024E10FC05E
:1054A00080914202909143020C2E02C096958795FE
:1054B0000A94E2F780FD02C02FE301C02FE780913C
:1054C000F0339091F1330C2E02C0969587950A9493
:1054D000E2F780FF0CC080914402909145020C2EAF
:1054E00002C0969587950A94E2F780FD20E0822F0E
:1054F0000E947D0F82B18F71FE01E85AFE4F9081AC
:10550000892B82B988E290E00E941A8659982196E8
:10551000CC30D10509F094CF88E290E00E941A8641
:10552000599AC0E0D0E064ECC62ED12C55E2E52EAD
:105530005DE0F52EC8010C2E02C0969587950A9461
:10554000E2F780FF5EC0149AFE01E15BFD4F8081AF
:1055500090E02091352B30E0FC01EE0FFF1FE80FAB
:10556000F91FCC9DC001CD9D900DDC9D900D1124A7
:10557000E80FF91F2E9DC0012F9D900D3E9D900DAF
:105580001124E80FF91FE452FC4F808181FD02C015
:1055900024E10FC080914202909143020C2E02C080
:1055A000969587950A94E2F780FD02C02FE301C02B
:1055B0002FE78091F0339091F1330C2E02C0969535
:1055C00087950A94E2F780FF0CC080914402909185
:1055D00045020C2E02C0969587950A94E2F780FD4D
:1055E00020E0822F0E947D0F82B18F71FE01E05A70
:1055F000FE4F9081892B82B988E290E00E941A8642
:1056000014982196C830D10509F094CF88E290E033
:105610000E941A86149ADF91CF911F910F91FF90EB
:10562000EF90DF90CF9008951F93CF93DF9310E01A
:10563000C0E0D0E087E29AE3BE0140E00E945A83D6
:10564000219687E29AE3BE0143E60E945A8321969F
:1056500087E29AE3BE0144E60E945A83219687E2DC
:105660009AE3BE0141E00E945A83219687E29AE3C1
:10567000BE0143E00E945A832196CA30D105D1F67B
:105680001F5F1038A9F6DF91CF911F910895EF9217
:10569000FF920F931F93CF93DF939AE0899FE001CE
:1056A000112408EB16E3A4E0EA2EF12CE00EF11E23
:1056B00087E29AE3BE01F80140810E945A83219655
:1056C00087E29AE3BE01F80142810E945A83219643
:1056D000F70161917191819191917F0120E030E01A
:1056E00048EC52E40E94DE8D0E94FC8C9B01AC01D0
:1056F00087E29AE3BE01422F0E945A83219687E2F5
:105700009AE3BE01F80142890E945A83219687E2FA
:105710009AE3BE01F80144890E945A830F5F1F4F2C
:105720002196F6E30A3B1F0719F6DF91CF911F91EF
:105730000F91FF90EF90089587E29AE360EA7FE08F
:1057400040E00E945A83089587E29AE360EA7FE08E
:1057500040910B360E945A830895EF92FF920F9367
:105760001F93CF93DF939AE0899F80011124C8EBA8
:10577000D6E3B4E0EB2EF12CEC0EFD1E87E29AE3AB
:10578000B8010E945383853008F084E08883B80113
:105790006F5F7F4F87E29AE30E9453838F3F09F444
:1057A0008EEF8A83B8016E5F7F4F87E29AE30E9493
:1057B0005383853608F084E6682F70E0882777FDEC
:1057C0008095982F0E942A8D20E030E048EC52E42A
:1057D0000E948F8CF7016083718382839383B80169
:1057E0006D5F7F4F87E29AE30E945383811181E0CE
:1057F0008A8BB8016C5F7F4F87E29AE30E945383E4
:10580000883008F087E08C8B1C861E86188A0B5F18
:105810001F4F219684E090E0E80EF91E96E3CA3B04
:10582000D90709F0ABCFDF91CF911F910F91FF9076
:10583000EF9008951092E6361092CE3680E00E94E6
:10584000AD2B80E00E942D1681E00E942D16089558
:1058500087E29AE360EA7FE00E94538380930B36ED
:10586000823020F010920B360E94A42B0895AF9244
:10587000BF92CF92DF92EF92FF920F931F9390917E
:10588000C4369F5F9093C4368091C5368F5F8093F6
:10589000C5368091CE36882349F080E098E00E949A
:1058A000BB0F80E098E00E94F00F2FC1892F90E09D
:1058B0004091BA3620E031E0241B3109821793076A
:1058C0000CF48BC01092C4368091B8368430D9F570
:1058D0008091C636882309F075C060E070E080E0F2
:1058E00090E02FEF30E040E050E00E948A89E090A5
:1058F000BC36F090BD360091BE361091BF360E9486
:105900002A8DA80197010E94DE8D5B016C01C80100
:10591000B70120E030E040E053EC0E94DE8D20E053
:1059200030E040E053E40E94278C9B01AC01C601AB
:10593000B5010E94278C0E94FC8C04E0660F771F43
:105940000A95E1F73BC0F82FE0E08091C636E80FFA
:10595000F11DEF5CFB4FE491E090BC36F090BD365A
:105960000091BE361091BF366E2F70E0882777FD0C
:105970008095982F0E942A8DA80197010E94DE8DA4
:105980005B016C01C801B70120E030E040E053EC5E
:105990000E94DE8D20E030E040E053E40E94278C3E
:1059A0009B01AC01C601B5010E94278C20E030E0CC
:1059B00040E851E40E94DE8D0E94FC8C70930E370B
:1059C00060930D3780910D3790910E370E94BB0F79
:1059D0008091C6368F5F8093C6368091C53690E041
:1059E0004091BB3620E031E0241B31098217930738
:1059F0000CF48BC01092C5368091B9368430D9F53D
:105A00008091C736882309F075C060E070E080E0BF
:105A100090E02FEF30E040E050E00E948A89E09073
:105A2000C036F090C1360091C2361091C3360E9444
:105A30002A8DA80197010E94DE8D5B016C01C801CF
:105A4000B70120E030E040E053EC0E94DE8D20E022
:105A500030E040E053E40E94278C9B01AC01C6017A
:105A6000B5010E94278C0E94FC8C14E0660F771F02
:105A70001A95E1F73BC0F82FE0E08091C736E80FB8
:105A8000F11DEF5CFB4FE491E090C036F090C13621
:105A90000091C2361091C3366E2F70E0882777FDD3
:105AA0008095982F0E942A8DA80197010E94DE8D73
:105AB0005B016C01C801B70120E030E040E053EC2D
:105AC0000E94DE8D20E030E040E053E40E94278C0D
:105AD0009B01AC01C601B5010E94278C20E030E09B
:105AE00040E851E40E94DE8D0E94FC8C70930C37DC
:105AF00060930B3780910B3790910C370E94F00F19
:105B00008091C7368F5F8093C73680914A02882381
:105B100029F190914B02809148028370813041F4C9
:105B2000E0913D02F0E0E05DF74FE491E69506C0BC
:105B3000E0913D02F0E0E05DF74FE491F0E09F5F1F
:105B400090934B029150892F90E08E179F0734F06D
:105B50000E94160F10924B0210924A0280914F360B
:105B60008F5F80934F361F910F91FF90EF90DF90E2
:105B7000CF90BF90AF9008951F920F920FB60F92E3
:105B80000BB60F9211242F933F934F935F936F9314
:105B90007F938F939F93AF93BF93EF93FF930E9455
:105BA000372CFF91EF91BF91AF919F918F917F9192
:105BB0006F915F914F913F912F910F900BBE0F907E
:105BC0000FBE0F901F9018952F923F924F925F92A9
:105BD0006F927F928F929F92AF92BF92CF92DF92FD
:105BE000EF92FF920F931F93DF93CF93CDB7DEB762
:105BF00028970FB6F894DEBF0FBECDBF8091EA02A2
:105C00008823D1F08091B7038823B1F42091B303A6
:105C10003091B4038091B5039091B6038217930736
:105C200058F48091B803882339F45F981092EA02FF
:105C30001092B4031092B3038091463690E088230B
:105C400009F491E09093463680914E0260E30E9401
:105C5000608E943041F48091790190E0882309F4BA
:105C600091E09093790180914E026CE00E94608EE9
:105C7000943051F4E091B102F0E0E658FE4F10820A
:105C800010924936109248368091AB02882311F465
:105C90000C948436EAEBF6E34FEF50E030E880896D
:105CA000882309F4A1C082898330F1F1843028F47B
:105CB000813069F18230A0F50CC0853009F454C000
:105CC0008530B8F1863009F457C0873009F067C0D5
:105CD0005EC08091AA0290E083709070892B09F0D9
:105CE0005EC080914E02813009F059C08091E83643
:105CF000882311F0348704C084858093E9361486A4
:105D000090E08091E836882309F591E01FC08091EA
:105D1000AA0290E083709070892B09F040C004C003
:105D20008091AA0280FD3BC080914E028130B9F57E
:105D30002AC090914E02913011F00C94FB36809164
:105D4000E836882311F00C94FB3634879093E836BC
:105D500026C08091E836882311F184858093E93646
:105D600014861092E8361BC080914E0260E30E94B8
:105D7000608E9923A1F407C080914E0290E08F714C
:105D80009070892B61F484858093E93607C08091F7
:105D90004E0268E10E94608E992309F414862081E6
:105DA000233000F19091E936892F80588F3768F4BD
:105DB000BA01691B7109653171052CF08289833044
:105DC00010F42B5F0EC02F5F0CC0892F815087FD10
:105DD00009C0953128F08289833010F4255001C024
:105DE000215020831092E936319676E3EC3BF70799
:105DF00009F055CF809148028370E1F580913A0215
:105E00008330D1F0843028F4813071F0823080F416
:105E100007C0853019F18530C8F0863059F522C0A9
:105E200080914E0260E60BC080914E0260E307C095
:105E300080914E0268E103C080914E026CE00E94A6
:105E4000608E9923B9F4809149020FC080914E026F
:105E500090E083709070892B69F404C080914E02A9
:105E600080FD08C08091490290E0882309F491E008
:105E7000909349021092A5021092A4021092BA03C4
:105E80008CE096E39A838983AFE5BBE2BC83AB8366
:105E900036EB432E32E0532E27EC622E22E0722E98
:105EA0009E838D8318861F8285E2282E8DE0382EF2
:105EB00001E0802E912CA12CB12CDF802091352B7C
:105EC000B0E1DB1681F4822F90E0829DF001839D8A
:105ED000F00D929DF00D1124EE53FC4FE25AF34F5A
:105EE000C190F0801DC0822F90E02F81388544EC56
:105EF00050E0249FF001259FF00D349FF00D1124F8
:105F0000BC01629DC001639D900D729D900D112496
:105F1000E80FF91FEE53FC4FE552FF4FC080F2909F
:105F20003296E08080914E029C2D9695292F30E08C
:105F300090E06C2D70E00E946C8E8217930731F414
:105F4000EF81F885ED56FD4F71E0708380914E0230
:105F500090E06C2D70E00E946C8E8217930709F020
:105F600068C0EF81F885EE57FD4F80818F5F808399
:105F70008081F81608F4108281E0E81681F0E816B6
:105F800040F092E0E916C9F0A3E0EA1609F051C02A
:105F90003DC0EF81F885EE57FD4F808108C0EF814D
:105FA000F885EE57FD4F8081BF2DB81B8B2FEF81F9
:105FB000F885EF58FD4F80833CC0EF81F885EF589E
:105FC000FD4F80818F1509F01EC7F301808181305C
:105FD00009F019C7108206C0D3018C91882311F4EF
:105FE000E1E0EC93D3018C91EF81F885EE57FD4F02
:105FF000AF81B885AF58BD4F882311F0808104C0B0
:106000008081EF2DE81B8E2F8C9313C02F2D30E055
:106010002F5F3F4F442737FD4095542F60E070E0DD
:1060200080E090E00E948A89EF81F885EF58FD4F6B
:1060300060832091352B4F2D50E0F0E1DF1679F58C
:1060400030E080915F0290E0841795071CF080E0BB
:1060500090E004C080915F0290E00196FC01EE0F99
:10606000FF1FE80FF91F229DD001239DB00D329D27
:10607000B00D1124EA0FFB1FEB5DFF4E908192954E
:1060800096959695937081818770880F880F892BDC
:10609000482F50E040515040AE5DBF4E40C0622F8F
:1060A00070E0EF81F885E15BFD4F808190E084171F
:1060B00095071CF080E090E003C0808190E001969D
:1060C000FC01EE0FFF1FE80FF91F2F81388544EC0C
:1060D00050E0249FD001259FB00D349FB00D1124B6
:1060E000EA0FFB1F629D9001639D300D729D300D84
:1060F0001124E20FF31FE452FC4F90819295969584
:106100009695937081818770880F880F892B482F0F
:1061100050E040515040A20FB31FA156BB4FAC916D
:10612000A15020914E020F81188507521D4FF80192
:106130008081EA2FF0E0EE0FFF1FE80FF11DEE0F58
:10614000FF1FEE5BFE4F80819181820F911D841BAA
:10615000950B6C2D70E00E94808E892B09F09CC2FB
:10616000EF81F885ED56FD4F8081882309F494C2B4
:106170001082D8018C9190E0882309F491E0EF819E
:10618000F885E752FD4F9083EF81F885E658FE4F82
:10619000B1E0B083EB16A1F0EB1640F0E2E0EE16B2
:1061A000D1F0F3E0EF1609F051C03DC0EF81F88562
:1061B000E05AFD4F8081EF81F885E15BFD4F2DC0F6
:1061C000EF81F885E05AFD4F8081F81AEF81F8855C
:1061D000E15BFD4F26C0EF81F885E15BFD4F8081DB
:1061E0008F1508F419C6D2018C91813009F014C6BC
:1061F0001C9206C0F2018081882311F421E02083E3
:10620000D2018C91EF81F885E15BFD4FAF81B885BC
:10621000A05ABD4F882319F08C91808317C08C91B0
:10622000F81AF08213C02F2D30E02F5F3F4F442724
:1062300037FD4095542F60E070E080E090E00E94D0
:106240008A89EF81F885E15BFD4F60832091352BD2
:10625000EF81F885E15BFD4FB0E1DB16C1F4808191
:1062600090E030E0FC01EE0FFF1FE80FF91F229DC8
:10627000C001239D900D329D900D1124E80FF91F50
:10628000EA5DFF4E608166956695669524C08081C3
:1062900090E030E0FC01EE0FFF1FE80FF91F4F8187
:1062A000588564EC70E0469FC001479F900D569F53
:1062B000900D1124E80FF91F229DC001239D900D20
:1062C000329D900D1124E80FF91FE452FC4F6081BC
:1062D000669566956F70EF81F885E15BFD4F808173
:1062E00082958F70AB81BC819C918917F9F0908168
:1062F00092959F709C9380913A2B882329F0EF818F
:10630000F885E25BF44D90838091460290914702BC
:106310008330910541F08730910529F0893091054E
:1063200011F0049719F4B1E0B0932C012091352BB2
:10633000E0E1DE16C9F480915F0290E030E0FC01FC
:10634000EE0FFF1FE80FF91F229DC001239D900D46
:10635000329D900D1124E80FF91FEB5DFF4E8081F7
:1063600081708093BA0339C0EF81F885E15BFD4FFE
:10637000808190E030E0FC01EE0FFF1FE80FF91F75
:106380004F815885A4ECB0E04A9FC0014B9F900D0F
:106390005A9F900D1124E80FF91F229DC001239DE3
:1063A000900D329D900D1124E80FF91FE452FC4F1F
:1063B000808180FF12C02091A4023091A50281E06B
:1063C00090E00F8002C0880F991F0A94E2F7822B99
:1063D000932B9093A5028093A402EF81F885E15B53
:1063E000FD4F808190E08F709070892B09F048C03C
:1063F000808190E02091352B30E0FC01EE0FFF1FF3
:10640000E80FF91F4F815885A4ECB0E04A9FC00106
:106410004B9F900D5A9F900D1124E80FF91F229D5C
:10642000C001239D900D329D900D1124E80FF91F9E
:10643000E452FC4F8081209102363091033680FD7A
:106440000DC0D501C4010F8004C0880F991FAA1F79
:10645000BB1F0A94D2F7282B392B0EC0D501C401DB
:106460000F8004C0880F991FAA1FBB1F0A94D2F780
:106470008095909528233923309303362093023654
:10648000EF81F885E05AFD4F80818F5F80836B300C
:1064900008F4AAC0B0E1DB16B9F02091A402309153
:1064A000A502D501C4010F8004C0880F991FAA1F3F
:1064B000BB1F0A94D2F780959095822393239093E3
:1064C000A5028093A40202C01092BA036D3091F12C
:1064D0006E3030F46B3059F06C3009F0D5C010C01C
:1064E0006E3009F440C06F3009F0CEC055C060E096
:1064F00070E080E090E029E030E040E050E054C0FF
:1065000060E070E080E090E027E030E040E050E0C4
:106510000E948A899B01AC0161307105810591055A
:1065200009F0B2C060E1D61609F04BC071E070937B
:10653000BA03AAC060E070E080E090E024E030E0C0
:1065400040E050E00E948A899B01AC0161307105F6
:106550008105910509F098C080E1D81691F591E088
:106560009093BA0391C060E070E080E090E023E097
:1065700030E040E050E00E948A899B01AC0161302C
:1065800071058105910509F07FC0A0E1DA16C9F413
:10659000B1E0B093BA0378C060E070E080E090E0D2
:1065A00022E030E040E050E00E948A899B01AC018B
:1065B000613071058105910509F066C0E0E1DE16E4
:1065C00079F08091A4029091A5020F8004C0220F5F
:1065D000331F441F551F0A94D2F7822B932B4DC0B3
:1065E000F1E0F093BA0350C0862F8150873068F4F1
:1065F00070E06F5F7F4FAD81BE818C9190E00E9413
:10660000808E892B09F440C015C0683049F4ED81B3
:10661000FE81808163E00E94608E9923A9F518C0F5
:10662000693061F4AD81BE818C9190E0837090708F
:10663000892B51F5B0E1DB1671F424C06A3021F5E5
:10664000ED81FE81808190E087709070892BE1F46C
:10665000F0E1DF16B9F02091A4023091A502D50136
:10666000C4010F8004C0880F991FAA1FBB1F0A9482
:10667000D2F780959095822393239093A5028093DF
:10668000A40202C01092BA038091A4029091A502C4
:106690009093A7028093A60220E1D21609F47DC050
:1066A0004091352B50E0BFE4EB2EB2E0FB2E6F8122
:1066B0007885E60EF71ED7012C9180914E0230E0CE
:1066C000F901EE0FFF1FE20FF31F24EC30E0629F91
:1066D0008001639F100D729F100D1124E00FF11FB8
:1066E000429D9001439D300D529D300D1124E20FCB
:1066F000F31FE352FC4FE081E695E695E695F0E066
:10670000EC5CFE4FE08190E06E2F70E00E946C8E9A
:10671000892B09F042C0EE2309F43FC08091A60204
:106720009091A7020F8002C0969587950A94E2F790
:1067300080FF33C0D7018C9190E0FC01EE0FFF1F6A
:10674000E80FF91FE00FF11FE20FF31FE452FC4FB7
:10675000808180FF22C04091A4025091A502209127
:10676000A4023091A502D501C4010F8004C0880F96
:10677000991FAA1FBB1F0A94D2F7282B392B3093DD
:10678000A5022093A4028091A4029091A502842BDB
:10679000952B9093A5028093A402EF81F885319602
:1067A000F887EF832D813E812F5F3F4F3E832D83FE
:1067B0004B815C814F5F5F4F5C834B830894411C2E
:1067C000511C0894611C711C719709F076CB809163
:1067D0004802837039F480914902882311F02C9A81
:1067E00001C02C988091BA03882309F40AC18091D2
:1067F000F202882309F005C18091B703882309F0CC
:1068000000C18091352BE82EFF2480915F022091FA
:106810005F0290E0FC01EE0FFF1FE80FF91F85E219
:106820009DE0E89EB001E99E700DF89E700D112468
:10683000E60FF71FE95DFF4E90819F70DB01AE53BD
:10684000BC4FA35AB34FEC918CE0E89FF0011124A8
:10685000E90FF11DE355FC4FE491E150F0E0EE0F3C
:10686000FF1FE75EFB4F4591549130E0F901EE0FB9
:10687000FF1FE20FF31FE60FF71FE95DFF4E2081B8
:10688000269526952695922F9E7080E0480F591FD9
:106890005093BD034093BC0380915F0212962C91EC
:1068A00030E090E0821793071CF080E090E004C095
:1068B00080915F0290E00196FC01EE0FFF1FE80F50
:1068C000F91F85E29DE0BC01E69EC001E79E900DA8
:1068D000F69E900D1124E80FF91FE95DFF4EE0814F
:1068E000EF7080915F0290E0821793071CF020E028
:1068F00030E006C080915F02282F30E02F5F3F4FCD
:10690000F0E0E355FC4FE491F0E0EE0FFF1FE75E8F
:10691000FB4F85919491F901EE0FFF1FE20FF31FDA
:1069200005E21DE0E09ED001E19EB00DF09EB00DAD
:106930001124EA0FFB1FE95DFF4E40814695469505
:106940004695342F3E7020E0820F931F9093BF0333
:106950008093BE032091BC033091BD03A05EBF4E67
:106960006C91821B930B70E00E94808E7093C10328
:106970006093C003C9010E94480F5F9A81E0809331
:10698000EA022091352B30E080915F0290E0FC011B
:10699000EE0FFF1FE80FF91F209FD001219FB00DC0
:1069A000309FB00D1124EA0FFB1FEB5DFF4E80817D
:1069B00086958F71A05EBF4EAC91A03639F490E001
:1069C0000196880F991F880F991F08C090E0A03387
:1069D00021F40196880F991F01C001969093B60388
:1069E0008093B5032091B5033091B6038A2F90E0D0
:1069F0002817390720F081E08093B80302C0109275
:106A0000B80380915F0290E02091352B30E0FC01CB
:106A1000EE0FFF1FE80FF91F85E29DE0DC012A9FC2
:106A2000C0012B9F900D3A9F900D1124E80FF91F84
:106A3000E95DFF4E808187FF14C08091B7038823F2
:106A400081F48091C0039091C1032091BC033091E7
:106A5000BD03820F931F9093BD038093BC030E94DC
:106A6000480F209137363091383621153105C1F065
:106A700080914E02E0913636F0E0EE58FE4F608194
:106A800090E070E00E946C8E892B51F48091A402FA
:106A90009091A502822B932B9093A5028093A40240
:106AA0008091A4029091A502892B61F18091A402AA
:106AB0009091A50290934936809348368091A40224
:106AC0009091A5020E940E2A80913502882349F0F8
:106AD0008091A4029091A5029F779093A502809344
:106AE000A4022091A4023091A5028091F0339091EC
:106AF000F13380959095822393230E94DE0E81E0EE
:106B000080934A02E0914D2BF0E0E05AFD4F8081E6
:106B100090E090933301809332011091352B612FD7
:106B200070E085E29DE0689FF001699FF00D789F1D
:106B3000F00D1124E456FB4F20E030E041E0D90194
:106B4000A05ABD4F9C918081891750F41C92A98155
:106B5000BA818C918F5F8C938150833D08F04C9368
:106B60002F5F3F4FEC53FF4F89819A8101969A83A3
:106B700089832031310519F72091700285E29DE06B
:106B8000689FF001699FF00D789FF00D1124EF5D73
:106B9000FF4E8081821768F41092700280911C363B
:106BA0008F5F80931C368150833D18F081E0809385
:106BB0001C3640914D2B403161F485E29DE0689F89
:106BC000F001699FF00D789FF00D1124E05EFF4EFB
:106BD00019C0242F30E084EC90E0289FF001299F19
:106BE000F00D389FF00D112485E29DE0DC016A9FD5
:106BF000C0016B9F900D7A9F900D1124E80FF91F33
:106C0000E356FB4F2081E42FF0E0E05AFD4F8081F6
:106C1000882309F056C080914E0290E0622F70E008
:106C20000E946C8E30E0215030408217930709F0AB
:106C300048C0109233011092320110924037809177
:106C4000372B8823F1F180914602909147028230E0
:106C5000910541F08530910529F08130910511F0C1
:106C6000892B79F51092372B1092352B112319F4BB
:106C700081E08093352B8091B5028093B3020E940E
:106C8000902581E08093EA3680932C0180E090E0AB
:106C900021E0FC01E05AFD4F1082FC01E752FD4F5C
:106CA0001082FC01EE57FD4F1082FC01E45FF94CAD
:106CB0002083FC01ED56FD4F208301968131910523
:106CC00041F740913201509133018091352B90E092
:106CD00025E23DE0829FF001839FF00D929FF00D31
:106CE0001124EE53FC4F808190E00197481759071B
:106CF00009F09BC080914037882309F096C081E05D
:106D00008093D802809340378091AB02882349F466
:106D100080914E026CE00E94608E992311F40E94D3
:106D2000A3298091AB02882309F520913736309151
:106D3000383621153105D1F080914E02E09136367A
:106D4000F0E0EE58FE4F608190E070E00E946C8EA3
:106D5000892B61F4C9010E940E2A809137369091E7
:106D600038360E94DE0E81E080934A0280914E0206
:106D70008F5F80934E028150803658F181E080937E
:106D80004E028091AA028F5F8093AA028091AA028C
:106D9000803110F01092AA028091AA0290E08370D4
:106DA0009070892BB1F400E010E080910236909150
:106DB0000336002E02C0969587950A94E2F780FF6D
:106DC00003C0802F0E943F290F5F1F4F0C30110519
:106DD00061F78091EA02882359F18091B8038823F2
:106DE00039F58091B3039091B40301969093B40365
:106DF0008093B3031DC080914E02813011F00C943A
:106E0000CF2E0C94A92EEF81F885EF58FD4F80818D
:106E1000882309F0E7C8E0C8EF81F885E15BFD4F02
:106E20008081882309F0ECC9E5C91092D8026CCFA3
:106E300028960FB6F894DEBF0FBECDBFCF91DF917D
:106E40001F910F91FF90EF90DF90CF90BF90AF9088
:106E50009F908F907F906F905F904F903F902F907A
:106E600008951F920F920FB60F920BB60F92112436
:106E70002F933F934F935F936F937F938F939F9342
:106E8000AF93BF93EF93FF939091CE008091480210
:106E90008370813009F0E7C0983F08F4E4C09A3F5E
:106EA00039F09C3F09F454C0983F09F0DCC053C04E
:106EB0008093AB0210924E021092B4031092B3036F
:106EC0001092AA021092E8362C982C9A90E08091A9
:106ED0003A02843009F091E0909349021092B03662
:106EE00010923301109232018FEF9FEF909307368B
:106EF0008093063680E090E021E0FC01E05AFD4FEF
:106F00001082FC01E752FD4F1082FC01EA54FD4F54
:106F10002083FC01EE57FD4F1082FC01E45FF94C29
:106F20002083FC01ED56FD4F2083019681319105B0
:106F300021F78091CA36882311F01092C6368091CD
:106F4000CB36882311F01092C7360E94E42D8BC0F7
:106F50008093053687C080911F3690912036A0918E
:106F60002136B09122368093680190936901A093F5
:106F70006A01B0936B0110921F3610922036109266
:106F80002136109222368091680190916901A0917A
:106F90006A01B0916B010A97A105B10560F48AE01E
:106FA00090E0A0E0B0E08093680190936901A09325
:106FB0006A01B0936B0180914E028370813029F495
:106FC00080914E02815080934E0280914E028370D8
:106FD000833029F480914E028F5F80934E0280911E
:106FE00006369091073601969093073680930636C1
:106FF00020913A02223091F0233028F4222341F0EC
:10700000213031F508C0233061F0243009F518C073
:107010004897F1F408C00C97D9F405C00697C1F45D
:1070200002C00397A9F48091490290E0882309F4F3
:1070300091E090934902109207361092063608C0EC
:107040008091490290E0882309F491E090934902ED
:107050008091AB02882339F080914902882311F096
:107060002C9A01C02C98FF91EF91BF91AF919F9105
:107070008F917F916F915F914F913F912F910F90E1
:107080000BBE0F900FBE0F901F9018951F920F927E
:107090000FB60F920BB60F921124AF92BF92CF9200
:1070A000DF92EF92FF920F931F932F933F934F9393
:1070B0005F936F937F938F939F93AF93BF93EF9360
:1070C000FF9380914802837090E08130910549F0F0
:1070D0008230910581F1892B09F09FC00E94E42D37
:1070E0009CC06091233670912436E0906801F09046
:1070F000690100916A0110916B0180E090E00E94AB
:10710000288D5B016C01C801B7010E94288D20E029
:1071100030E040E85EE30E94DE8D9B01AC01C601D9
:10712000B5010E94DA8D88230CF45BC010922436DE
:107130001092233654C080912A36882389F1109208
:1071400024361092233610922A3680914E028435CE
:1071500020F480914E028C3010F410924E028091F7
:107160004E028C3038F080914E02843218F488E15F
:1071700080934E0280914E02843238F080914E020C
:107180008C3318F480E380934E0280914E028C334E
:1071900038F080914E02843518F488E480934E02D2
:1071A0000091233610912436609168017091690135
:1071B00080916A0190916B0128E130E040E050E05D
:1071C0000E94938E0217130720F01092243610921B
:1071D00023368091233690912436892B11F40E9416
:1071E000E42D80911F3690912036A0912136B091E8
:1071F00022360196A11DB11D80931F369093203633
:10720000A0932136B0932236809123369091243674
:1072100001969093243680932336FF91EF91BF918E
:10722000AF919F918F917F916F915F914F913F911E
:107230002F911F910F91FF90EF90DF90CF90BF9013
:10724000AF900F900BBE0F900FBE0F901F90189530
:10725000FF920F931F93F82E0BEE16E3C8016F2DCC
:1072600041E00E94987EC8016BE378E00E946C8741
:10727000C8016F2D41E00E94987E1F910F91FF90F1
:1072800008950F931F930BEE16E3C80164E040E0EE
:107290000E94987EC80169E978E00E946C8781E0CD
:1072A0008093EC011F910F9108950F931F930BEEA4
:1072B00016E3C80164E040E00E94987EC80163EADA
:1072C00078E00E946C8781E08093EC011F910F9120
:1072D00008950F931F930BEE16E3C80164E040E09E
:1072E0000E94987EC8016DEA78E00E946C8781E078
:1072F0008093EC011F910F9108958BEE96E36CEB58
:1073000078E00E946C8708950F931F930BEE16E3AD
:10731000C80160E040E00E94987EC80161E578E025
:107320000E946C87C80160E041E00E94987E0E9444
:107330007D39C80160E041E00E94987EC80160E4A8
:1073400078E00E946C871F910F9108950F931F930F
:107350000BEE16E3C80160E040E00E94987EC80191
:1073600063E778E00E946C87C80160E041E00E941A
:10737000987E0E947D39C80160E041E00E94987EBD
:10738000C80162E678E00E946C871F910F91089512
:107390000F931F93CF93DF93C0E0D0E0082F10E04E
:1073A00006C08BEE96E361EA0E948F872196C01794
:1073B000D107BCF3DF91CF911F910F91089588E021
:1073C0000E942839E091E636F0E0E854F94C8489CF
:1073D0008330D1F1843030F4813009F449C08230F7
:1073E000E0F54DC08530C9F0853000F1863061F0A0
:1073F000873009F04AC08BEE96E360E00E948E7EF3
:107400008BEE96E361E031C08BEE96E360E00E9484
:107410008E7E8BEE96E361E011C08BEE96E360E02A
:107420000E948E7E8BEE96E363E01FC08BEE96E3A8
:1074300060E00E948E7E8BEE96E363E00E948E7E7B
:107440008BEE96E362E011C08BEE96E360E00E9463
:107450008E7E8BEE96E366E008C08BEE96E360E0EE
:107460000E948E7E8BEE96E367E00E948E7E0895EA
:107470008BEE96E369EB78E00E946C8708958BEEC3
:1074800096E366EB78E00E946C8708951F93209145
:10749000B1024091352B203171F4242F30E085E288
:1074A0009DE0289FF001299FF00D389FF00D1124D9
:1074B000E05EFF4E19C030E050E084EC90E0289F81
:1074C000F001299FF00D389FF00D112485E29DE019
:1074D0009C01429FC001439F900D529F900D11242B
:1074E000E80FF91FE356FB4F108188E00E9428390E
:1074F000183109F1193130F41C3059F0103109F00C
:1075000044C010C0103371F11036A9F11032E9F502
:107510001BC08BEE96E360E00E948E7E8BEE96E3BE
:1075200064E031C08BEE96E360E00E948E7E8BEECD
:1075300096E361E011C08BEE96E360E00E948E7EE0
:107540008BEE96E361E01FC08BEE96E360E00E9455
:107550008E7E8BEE96E363E00E948E7E8BEE96E34A
:1075600062E011C08BEE96E360E00E948E7E8BEEAF
:1075700096E363E008C08BEE96E360E00E948E7EA7
:107580008BEE96E366E00E948E7E1F910895CF9267
:10759000DF92EF92FF920F931F93CF93DF93EC0153
:1075A0008B017A01690166EF71E00E94F4898823FA
:1075B00021F58BEE96E360E041E00E94987E8BEE31
:1075C00096E36CED78E00E946C878C819D81029738
:1075D00020F48BEE96E361E003C08BEE96E360E06F
:1075E00041E00E94987E8BEE96E3BE010E943589B1
:1075F00086EF91E0BE010E94ED8BC8016DEF71E056
:107600000E94F4898823E1F48BEE96E364E041E084
:107610000E94987E8BEE96E367ED78E00E946C877F
:107620008BEE96E364E041E00E94987E8BEE96E359
:10763000B8010E9435898DEF91E0B8010E94ED8B71
:10764000C70164E072E00E94F489882329F58BEE7B
:1076500096E368E041E00E94987E8BEE96E362ED4F
:1076600078E00E946C87F70184819581029720F46D
:107670008BEE96E369E003C08BEE96E368E041E0B1
:107680000E94987E8BEE96E3B7010E94358984E0D4
:1076900092E0B7010E94ED8BC6016BE072E00E94A0
:1076A000F489882329F58BEE96E36CE041E00E9493
:1076B000987E8BEE96E36DEC78E00E946C87F60185
:1076C00084819581029720F48BEE96E36DE003C0F0
:1076D0008BEE96E36CE041E00E94987E8BEE96E3A1
:1076E000B6010E9435898BE092E0B6010E94ED8BD5
:1076F000DF91CF911F910F91FF90EF90DF90CF908E
:1077000008958F929F92AF92BF92CF92DF92EF92A5
:10771000FF920F931F93DF93CF93CDB7DEB7CF5771
:10772000D3400FB6F894DEBF0FBECDBF8091ED0100
:107730008823A1F08BEE96E36091F00141E00E9476
:10774000987E809179018823F1F48BEE96E361E0D5
:1077500071E00E949488109212371EC080911237F7
:107760008823D1F48091EE0190E02091460230917F
:1077700047028217930781F48BEE96E36091F00144
:1077800041E00E94987E8BEE96E36EE272E00E94EA
:10779000358981E0809312378091EE0190E020914D
:1077A0004602309147028217930711F01092ED01C3
:1077B00080912C01882311F40C94495110922C01D2
:1077C0008091F501882309F472C08BEE96E360E0A6
:1077D00040E00E94987E8BEE96E368E57AE00E9496
:1077E0006C878BEE96E360E041E00E94987E0E94F9
:1077F0007D398BEE96E362E041E00E94987E8BEE4D
:1078000096E366E57AE00E946C878BEE96E365E08E
:1078100041E00E94987E87E00E94C8398BEE96E393
:107820006EE041E00E94987E8BEE96E364E57AE09C
:107830000E946C872091B1024091352B203171F468
:10784000242F30E085E29DE0289FF001299FF00D74
:10785000389FF00D1124EE5DFF4E19C030E050E06E
:1078600084EC90E0289FF001299FF00D389FF00DE7
:10787000112485E29DE09C01429FC001439F900D31
:10788000529F900D1124E80FF91FE156FB4F6081C4
:107890006C5F8BEE96E341E00E94987E8BEE96E360
:1078A0006BED0E948F878BE090E00C9445518091A6
:1078B000F401882309F475C08BEE96E360E040E0A4
:1078C0000E94987E8091460290914702029729F487
:1078D0008BEE96E363E47AE004C08BEE96E362E31A
:1078E0007AE00E946C878BEE96E360E041E00E94B4
:1078F000987E0E947D398BEE96E363E041E00E9422
:10790000987E2091B1024091352BDE01A958BC4FE1
:107910002031B9F4242F30E085E29DE0289FF0016A
:10792000299FF00D389FF00D1124ED5DFF4E8081F1
:10793000E82FF0E0EE0FFF1FE551FD4F65917491C8
:1079400022C030E050E084EC90E0289FF001299FB5
:10795000F00D389FF00D112485E29DE0BC01469F9B
:10796000C001479F900D569F900D1124E80FF91FFD
:10797000E256FB4F8081E82FF0E0EE0FFF1FE5514C
:10798000FD4F65917491CD010E941E088BEE96E328
:10799000BE0169587C4F0E9494888AE090E00C9464
:1079A000455180914602909147028630910511F42D
:1079B0000C94124987309105D4F48230910509F472
:1079C0002FC28330910554F4009711F40C948A4E21
:1079D000019711F00C9449510C94614D843091053C
:1079E00009F458C5059714F00C941C4D2EC389302A
:1079F000910511F40C94544A8A30910554F487305F
:107A0000910511F40C941446089711F00C94495107
:107A100010C08D30910511F40C945B4F8E309105A0
:107A200011F40C9436500C9711F00C9449510C94AD
:107A300081458091AE029091AF020897A9F08BE04A
:107A400092E066E071E00E940E8BBC0184E092E05F
:107A50000E94ED8BBC018DEF91E00E94ED8BBC018B
:107A600086EF91E00E94ED8B8091F101813029F049
:107A7000823011F00C944951BBC08091AE029091BC
:107A8000AF02089761F480914101813041F4809107
:107A90002D01882321F48091EC018823D1F188E025
:107AA00090E09093AF028093AE028091F1018093B9
:107AB000410110922D011092EC018BEE96E360E0F3
:107AC00040E00E94987E8BEE96E361E27AE00E94AD
:107AD0006C878091EF01E82FF0E0EE0FFF1FE55774
:107AE000FD4F659174918E010F5F1F4FC8010E9479
:107AF0001E08E091EF01F0E0E25DFE4F8BEE96E3B1
:107B0000608140E00E94987E8BEE96E3B8010E946F
:107B10009488809148028370E82FF0E0EE0FFF1FF9
:107B2000E55AFC4F659174917E010894E11CF11CAB
:107B3000C7010E941E0882E192E0B7010E940E8BED
:107B40008E010B5F1F4F6091400270914102C8018E
:107B50004AE00E94278B89E192E0B8010E94ED8BF8
:107B6000C8010E941A8C8E01045F1F4FC8016091EA
:107B70003D024AE00E94898B80E292E0B8010E94B7
:107B8000ED8BC8010E941A8C80913A02E82FF0E038
:107B9000EE0FFF1FE35BFC4F65917491C7010E94DC
:107BA0001E0887E292E0B7010E940E8BF3E1AF2E30
:107BB000B12CAC0EBD1EC50162E172E00E94048CC6
:107BC000EAE1CE2ED12CCC0EDD1EC60169E172E0B9
:107BD0000E94048C71E2E72EF12CEC0EFD1EC70111
:107BE00060E272E00E94048C8E01085D1F4FFFC0AE
:107BF00080914101823049F480912D01882329F43C
:107C00008091EC01882309F44DC082E0809341010A
:107C100010922D011092EC018BEE96E360E040E0B3
:107C20000E94987E8BEE96E365E17AE00E946C8775
:107C30008091B402809314378BEE96E36FE70E9435
:107C40008F878BEE96E362E17AE00E946C87609109
:107C5000B40270E06F5F7F4F8BEE96E34AE050E036
:107C60000E9481888091EF01E82FF0E0EE0FFF1F66
:107C7000ED56FD4F659174918E010F5F1F4FC80146
:107C80000E941E08E091EF01F0E0E25DFE4F8BEEF6
:107C900096E3608140E00E94987E8BEE96E3B80107
:107CA0000E949488909114378091B402981709F13A
:107CB0008BEE96E36FE040E00E94987E8BEE96E3B9
:107CC00060E17AE00E946C878BEE96E36EE040E024
:107CD0000E94987E6091B40270E06F5F7F4F8BEEE0
:107CE00096E34AE050E00E9481888091B40280933C
:107CF000143780913602E82FF0E0EE0FFF1FEF55AA
:107D0000FC4F659174918E010F5F1F4FC8010E9457
:107D10001E0882E192E0B8010E940E8B809135022C
:107D2000E82FF0E0EE0FFF1FEB55FC4F65917491CB
:107D3000C8010E941E0889E192E0B8010E940E8BE2
:107D4000E0914402F09145020090B40202C0F69521
:107D5000E7950A94E2F7E170F070EE0FFF1FEB5524
:107D6000FC4F65917491C8010E941E0880E292E068
:107D7000B8010E940E8BE0914202F0914302009004
:107D8000B40202C0F695E7950A94E2F7E170F0704C
:107D9000EE0FFF1FE755FC4F65917491C8010E94DB
:107DA0001E0887E292E0B8010E940E8B9FE2A92E86
:107DB000B12CAC0EBD1EC50162E172E00E94048CC4
:107DC00086E3C82ED12CCC0EDD1EC60169E172E01F
:107DD0000E94048C0DE3E02EF12CEC0EFD1EC70179
:107DE00060E272E00E94048C8E010C5B1F4FC801A0
:107DF00067E272E00E94048CC501B601A7019801F8
:107E00000E94C73AC8010E941A8CC7010E941A8CAE
:107E1000C6010E941A8CC5010E941A8C0C9449510B
:107E20008BEE96E360E040E00E94987E8091F20144
:107E3000882309F445C08BEE96E36FEF79E00E944A
:107E40006C878BEE96E360E041E00E94987E0E9492
:107E50007D398BEE96E364E041E00E94987EE091EC
:107E6000B102F0E0E25BF44D608170E06F5F7F4F44
:107E70008BEE96E34AE050E00E9481888BEE96E319
:107E80006BE041E00E94987E8091352B90E025E2E6
:107E90003DE0829FF001839FF00D929FF00D112431
:107EA000EE53FC4F608170E06F5F7F4F8BEE96E387
:107EB0004AE050E00E94818881E08093F30177C01E
:107EC0008091AE029091AF02029749F48091F30144
:107ED000882329F48091EC01882309F468C082E0AA
:107EE00090E09093AF028093AE021092F301109253
:107EF000EC018BEE96E36EEE79E00E946C878BEEE0
:107F000096E360E041E00E94987E0E947D398BEE0E
:107F100096E362E041E00E94987E6091B2026F5B5E
:107F20008BEE96E30E948F876091B30270E06F5FE3
:107F30007F4F8091B20290E014E0880F991F1A954C
:107F4000E1F7681B790B8BEE96E34AE050E00E9464
:107F500081888091B302809314378BEE96E369E0B9
:107F600041E00E94987E8BEE96E365E00E948E7E53
:107F70008BEE96E368E071E00E949488809148025D
:107F8000837039F08BEE96E36AEE79E00E946C879D
:107F90000AC060913E0270913F028BEE96E34AE088
:107FA00050E00E941E8880913E028093133790918A
:107FB000B30280911437981719F182E00E94283992
:107FC0006091B2026F5B8BEE96E30E948F876091A7
:107FD000B30270E06F5F7F4F8091B20290E0B4E037
:107FE000880F991FBA95E1F7681B790B8BEE96E322
:107FF0004AE050E00E9481888091B3028093143758
:108000008091133790E020913E0230913F02821719
:10801000930711F40C94495180914802837011F038
:108020000C9449518BE00E94283960913E02709176
:108030003F028BEE96E34AE050E00E941E8880915A
:108040003E02809313370C9449518091AE02909177
:10805000AF020397C1F08BE092E066E071E00E940E
:108060000E8BBC0184E092E00E94ED8BBC018DEF91
:1080700091E00E94ED8BBC0186EF91E00E94ED8BB8
:1080800081E00E94463A8091AE029091AF02039740
:1080900041F480912D01882321F48091EC01882303
:1080A00081F18BEE96E360E040E00E94987E8BEEDB
:1080B00096E369ED79E00E946C878091EF01E82FEB
:1080C000F0E0EE0FFF1FE553FD4F659174918E01B7
:1080D0000F5F1F4FC8010E941E08E091EF01F0E002
:1080E000E25DFE4F8BEE96E3608140E00E94987E59
:1080F0008BEE96E3B8010E94948810922D011092A5
:10810000EC018E01055B1F4FE091B102F0E0E15AF6
:10811000F44D608170E06F5F7F4FC8014AE00E94BC
:10812000588BCE018E5A9F4FB8010E940F8C8091C0
:108130003A2B882311F460E201C06EE7E2E5CE2E0F
:10814000D12CCC0EDD1EC6010E94928A8C0179E5ED
:10815000E72EF12CEC0EFD1EE091B102F0E0E25BA7
:10816000F44D608170E06F5F7F4FC7014AE00E946D
:10817000588BC801B7010E94A38ABC018E01005A26
:108180001F4FC8010E94048C82E192E0B8010E9456
:10819000ED8BC8010E941A8CC7010E941A8CC6017F
:1081A0000E94208CCE01855B9F4F0E941A8C2091EB
:1081B000B1024091352B203171F4242F30E085E25B
:1081C0009DE0289FF001299FF00D389FF00D1124AC
:1081D000EF5DFF4E19C030E050E084EC90E0289F46
:1081E000F001299FF00D389FF00D112485E29DE0EC
:1081F0009C01429FC001439F900D529F900D1124FE
:10820000E80FF91FE456FB4F8081682F70E06F5F25
:108210007F4F8E0109591F4FC8014AE00E94588BB9
:1082200089E192E0B8010E94ED8BC8010E941A8C8E
:1082300080E292E060E070E00E940E8B4091B1021B
:10824000403139F48E0102591F4FC8016AE071E0D4
:1082500092C080910B36882309F481C0E42FF0E0AE
:10826000EE0FFF1FE757FC4F65917491CE01019609
:108270000E941E084091B1024C3090F58091352B40
:1082800090E025E23DE0829FF001839FF00D929FF8
:10829000F00D1124EE53FC4FE40FF11D878188236C
:1082A00011F460E201C06BE25CE7C52ED12CCC0E6C
:1082B000DD1EC6010E94D48B45E7E42EF12CEC0EA6
:1082C000FD1EC701BE016F5F7F4F0E94DA8AC601A3
:1082D000B7010E94A38ABC018E010D571F4F8AC0AF
:1082E0004F3041F480913502882321F08E010657EA
:1082F0001F4F3EC08091352B90E025E23DE0829FEC
:10830000F001839FF00D929FF00D1124EE53FC4F6E
:10831000E40FF11D8781882311F460E201C06BE254
:1083200038E9C32ED12CCC0EDD1EC6010E94D48BA1
:1083300021E9E22EF12CEC0EFD1E6091B10270E0FD
:108340006F5F7F4FC7014AE00E94588BC601B7019B
:108350000E94A38ABC018E0101561F4F4BC04F30B3
:10836000A9F480913502882389F08E010A551F4FA8
:10837000C8016DE071E00E94DA8A87E292E0B801FC
:108380000E94ED8BC8010E941A8C45C08091352B4C
:1083900090E025E23DE0829FF001839FF00D929FE7
:1083A000F00D1124EE53FC4FE40FF11D878188235B
:1083B00011F460E201C06BE294EBC92ED12CCC0E1B
:1083C000DD1EC6010E94D48B8DEAE82EF12CEC0E46
:1083D000FD1E6091B10270E06F5F7F4FC7014AE000
:1083E0000E94588BC601B7010E94A38ABC018E016E
:1083F00005541F4FC8010E94048C87E292E0B80127
:108400000E94ED8BC8010E941A8CC7010E941A8C31
:10841000C6010E94208C02ECA02EB12CAC0EBD1E19
:10842000C50162E172E00E94048C19ECC12ED12CCE
:10843000CC0EDD1EC60169E172E00E94048CB0ED35
:10844000EB2EF12CEC0EFD1EC70160E272E00E94E3
:10845000048C8E0109521F4FC80167E272E00E942E
:10846000048CC501B601A70198010E94C73AC80152
:108470000E941A8CC7010E941A8CC6010E941A8C95
:10848000C5010E941A8C80E00E94463A83E090E089
:108490000C9445518091B1022091AE023091AF020F
:1084A000803109F001C124303105A9F08BE092E060
:1084B00066E071E00E940E8BBC0184E092E00E94B5
:1084C000ED8BBC018DEF91E00E94ED8BBC0186EF3E
:1084D00091E00E94ED8B8091AE029091AF020497E3
:1084E00041F480912D01882321F48091EC018823AF
:1084F000A1F18BEE96E360E040E00E94987E8BEE67
:1085000096E368EC79E00E946C878091EF01E82F98
:10851000F0E0EE0FFF1FED51FD4F659174918E015C
:108520000F5F1F4FC8010E941E08E091EF01F0E0AD
:10853000E25DFE4F8BEE96E3608140E00E94987E04
:108540008BEE96E3B8010E9494888091BB038093E0
:10855000410110922D011092EC018091352B90E099
:1085600025E23DE0829FF001839FF00D929FF00D88
:108570001124E15EFF4E8081E82FF0E0EE0FFF1F37
:10858000ED50FD4F659174917E010894E11CF11C42
:10859000C7010E941E088E0102521F4FC801B70179
:1085A0000E94DA8A82E192E0B8010E94ED8BC80154
:1085B0000E941A8C8091F535E82FF0E0EE0FFF1F36
:1085C000EF58FC4F65917491C7010E941E088E01FF
:1085D0000B511F4FC801B7010E94DA8A89E192E06E
:1085E000B8010E94ED8BC8010E941A8C8E010451C3
:1085F0001F4F60915E0170E063507040C8014AE017
:108600000E94588B80E292E0B8010E94ED8BC80175
:108610000E941A8C8E010D501F4FC80160E071E05E
:108620000E94DA8A87E292E0B8010E94ED8BC801CD
:108630000E941A8C5AEFA52EB12CAC0EBD1EC5019E
:1086400062E172E00E94048C41E0C42ED42ECC0E74
:10865000DD1EC60169E172E00E94048C38E0E32E61
:1086600031E0F32EEC0EFD1EC70160E272E00E94C5
:10867000048C8E01015F1E4FC80167E272E00E9408
:10868000048CC501B601A70198010E94C73AC80130
:108690000E941A8CC7010E941A8CC6010E941A8C73
:1086A000C5010E941A8C29C224303105C1F08BE02B
:1086B00092E066E071E00E940E8BBC0184E092E0E3
:1086C0000E94ED8BBC018DEF91E00E94ED8BBC010F
:1086D00086EF91E00E94ED8B81E00E94463A809106
:1086E000AE029091AF02049741F480912D0188234E
:1086F00021F48091EC01882381F18BEE96E360E018
:1087000040E00E94987E8BEE96E367EB79E00E9452
:108710006C878091EF01E82FF0E0EE0FFF1FE5532B
:10872000FD4F659174918E010F5F1F4FC8010E942C
:108730001E08E091EF01F0E0E25DFE4F8BEE96E364
:10874000608140E00E94987E8BEE96E3B8010E9423
:10875000948810922D011092EC018E010A5E1E4F3A
:10876000E091B102F0E0E15AF44D608170E06F5F9A
:108770007F4FC8014AE00E94588BCE01835E9E4F16
:10878000B8010E940F8C80913A2B882311F460E28B
:1087900001C06EE79DE1C92E91E0D92ECC0EDD1E01
:1087A000C6010E94928A8C0184E2E82E81E0F82EB4
:1087B000EC0EFD1EE091B102F0E0E25BF44D608151
:1087C00070E06F5F7F4FC7014AE00E94588BC8017D
:1087D000B7010E94A38ABC018E01055D1E4FC8012E
:1087E0000E94048C82E192E0B8010E94ED8BC801E6
:1087F0000E941A8CC7010E941A8CC6010E94208C0C
:10880000CE018A5E9E4F0E941A8C2091B102409147
:10881000352B203171F4242F30E085E29DE0289F34
:10882000F001299FF00D389FF00D1124EF5DFF4EF0
:1088300019C030E050E084EC90E0289FF001299FBF
:10884000F00D389FF00D112485E29DE0BC01469F9C
:10885000C001479F900D569F900D1124E80FF91FFE
:10886000E456FB4F8081682F70E06F5F7F4F8E0171
:108870000E5C1E4FC8014AE00E94588B89E192E0CD
:10888000B8010E94ED8BC8010E941A8C80E292E030
:1088900060E070E00E940E8B4091B102403139F4EB
:1088A0008E01075C1E4FC8016AE071E096C080919E
:1088B0000B36882309F485C0E42FF0E0EE0FFF1F8C
:1088C000E757FC4F65917491CE0101960E941E08F6
:1088D0004091B1024C30A0F58091352B90E025E21B
:1088E0003DE0829FF001839FF00D929FF00D1124D7
:1088F000EE53FC4FE40FF11D8781882311F460E2F1
:1089000001C06BE2B7E4CB2EB1E0DB2ECC0EDD1E56
:10891000C6010E94D48BA0E4EA2EA1E0FA2EEC0E50
:10892000FD1EC701BE016F5F7F4F0E94DA8AC6013C
:10893000B7010E94A38ABC018E01025B1E4F8EC04C
:108940004F3041F480913502882321F08E010B5A7B
:108950001E4F40C08091352B90E025E23DE0829F84
:10896000F001839FF00D929FF00D1124EE53FC4F08
:10897000E40FF11D8781882311F460E201C06BE2EE
:10898000F3E6CF2EF1E0DF2ECC0EDD1EC6010E94F5
:10899000D48BECE5EE2EE1E0FE2EEC0EFD1E609198
:1089A000B10270E06F5F7F4FC7014AE00E94588BB1
:1089B000C601B7010E94A38ABC018E0106591E4F51
:1089C0004DC04F30A9F480913502882389F08E0183
:1089D0000F581E4FC8016DE071E00E94DA8A87E2ED
:1089E00092E0B8010E94ED8BC8010E941A8C47C02A
:1089F0008091352B90E025E23DE0829FF001839F3E
:108A0000F00D929FF00D1124EE53FC4FE40FF11D79
:108A10008781882311F460E201C06BE27FE7C72EF3
:108A200071E0D72ECC0EDD1EC6010E94D48B68E704
:108A3000E62E61E0F62EEC0EFD1E6091B10270E0B4
:108A40006F5F7F4FC7014AE00E94588BC601B70194
:108A50000E94A38ABC018E010A571E4FC8010E94C2
:108A6000048C87E292E0B8010E94ED8BC8010E945D
:108A70001A8CC7010E941A8CC6010E94208C5DE8E6
:108A8000A52E51E0B52EAC0EBD1EC50162E172E00F
:108A90000E94048C44E9C42E41E0D42ECC0EDD1E8D
:108AA000C60169E172E00E94048C3BE9E32E31E0EB
:108AB000F32EEC0EFD1EC70160E272E00E94048CF2
:108AC0008E010E551E4FC80167E272E00E94048CB1
:108AD000C501B601A70198010E94C73AC8010E94CA
:108AE0001A8CC7010E941A8CC6010E941A8CC501FB
:108AF0000E941A8C80E00E94463A84E090E00C9438
:108B000045518091AE029091AF020C9721F4809173
:108B1000EC018823B9F18BEE96E360E040E00E941F
:108B2000987E0E947D398BEE96E362E040E00E94E1
:108B3000987E8BEE96E362EB79E00E946C878BEE79
:108B400096E360E041E00E94987E0E947D398BEEC2
:108B500096E362E041E00E94987E8BEE96E36FEA36
:108B600079E00E946C87E0913636F0E0EF51F74FE4
:108B7000E4918BEE96E36E2F4AE050E00E942F883E
:108B80001092EC01E0913636F0E0EF51F74FE491AE
:108B90008E0107551E4FC8016E2F4AE00E94898B37
:108BA00086EF91E0B8010E94F489F82EC8010E9476
:108BB0001A8CFF20A9F58BEE96E364E041E00E9459
:108BC000987E8BEE96E36BEA79E00E946C878BEEE1
:108BD00096E364E041E00E94987EE0913636F0E052
:108BE000EF51F74FE4918BEE96E36E2F4AE050E0A1
:108BF0000E942F88E0913636F0E0EF51F74FE49174
:108C00008E0100551E4FC8016E2F4AE00E94898BCD
:108C100086EF91E0B8010E94ED8BC8010E941A8C8A
:108C20008CE090E00C9445518091BB03882321F0A7
:108C3000813009F0F3C2E3C18091AE029091AF029E
:108C4000079721F4809141018823A9F08BE092E0FD
:108C500066E071E00E940E8BBC0184E092E00E940D
:108C6000ED8BBC018DEF91E00E94ED8BBC0186EF96
:108C700091E00E94ED8B8091AE029091AF02079738
:108C800071F49091BB0380914101981741F4809158
:108C90002D01882321F48091EC018823A1F18BEE32
:108CA00096E360E040E00E94987E8BEE96E36AE9EE
:108CB00079E00E946C878091EF01E82FF0E0EE0FE1
:108CC000FF1FE555FD4F659174918E010F5F1F4F9A
:108CD000C8010E941E08E091EF01F0E0E25DFE4F46
:108CE0008BEE96E3608140E00E94987E8BEE96E3E7
:108CF000B8010E9494888091BB0380934101109237
:108D00002D011092EC018E0109541E4FE091B10229
:108D1000F0E0E15AF44D608170E06F5F7F4FC80171
:108D20004AE00E94588BCE0182549E4FB8010E94A7
:108D30000F8C80913A2B882311F460E201C06EE71A
:108D40009EEBC92E91E0D92ECC0EDD1EC6010E94ED
:108D5000928A8C0185ECE82E81E0F82EEC0EFD1E47
:108D6000E091B102F0E0E25BF44D608170E06F5F92
:108D70007F4FC7014AE00E94588BC801B7010E948B
:108D8000A38ABC018E0104531E4FC8010E94048CAB
:108D900082E192E0B8010E94ED8BC8010E941A8C1A
:108DA000C7010E941A8CC6010E94208CCE018954F2
:108DB0009E4F0E941A8C2091352B30E080914C02FE
:108DC00090E0FC01EE0FFF1FE80FF91FA5E2CA2E8D
:108DD000ADE0DA2E2C9DD0012D9DB00D3C9DB00D47
:108DE0001124EA0FFB1FE95DFF4E90819F70A15E89
:108DF000BF4EEC918CE0E89FF0011124E90FF11DCA
:108E0000E355FC4FE491F0E0EE0FFF1FE159FC4FFA
:108E1000659174917E010894E11CF11CC7010E94C8
:108E20001E088E010D521E4FC801B7010E94DA8A3A
:108E300089E192E0B8010E94ED8BC8010E941A8C72
:108E400080914C0290E02091352B30E0FC01EE0F38
:108E5000FF1FE80FF91F2C9DC0012D9D900D3C9D1B
:108E6000900D1124E80FF91FE95DFF4E8081829576
:108E70008770E82FF0E0EE0FFF1FEF59FC4F659170
:108E80007491C7010E941E088E0106521E4FC80130
:108E9000B7010E94DA8A80E292E0B8010E94ED8B6D
:108EA000C8010E941A8C2091352B30E080914C0231
:108EB00090E0FC01EE0FFF1FE80FF91F2C9DD00181
:108EC0002D9DB00D3C9DB00D1124EA0FFB1FEB5DF5
:108ED000FF4E608166956F71262F2F5FA05EBF4E9B
:108EE000AC91A03619F4220F220F03C0A03309F46D
:108EF000220FCE018F519E4F2A1729F462E171E0B3
:108F00000E94DA8A06C070E06F5F7F4F4AE00E94DD
:108F1000588B8E010F511E4F87E292E0B8010E94DC
:108F2000ED8BC8010E941A8C28EEA22E21E0B22EF1
:108F3000AC0EBD1EC50162E172E00E94048C9FEE82
:108F4000C92E91E0D92ECC0EDD1EC60169E172E07A
:108F50000E94048C86EFE82E81E0F82EEC0EFD1EB8
:108F6000C70160E272E00E94048C8E0103501E4F24
:108F7000C80167E272E00E94048CC501B601A70136
:108F800098010E94C73AC8010E941A8CC7010E942A
:108F90001A8CC6010E941A8CC5010E941A8C8BEE95
:108FA00096E36FE041E00E94987E80914C0290E051
:108FB0002091352B30E0FC01EE0FFF1FE80FF91F69
:108FC00085E29DE0AC01249FC001259F900D349F58
:108FD000900D1124E80FF91FE95DFF4E808187FF96
:108FE00007C08BEE96E368E979E00E946C8716C1B2
:108FF0008BEE96E366E171E00E9494880FC1809148
:10900000AE029091AF02079721F480914101813027
:10901000A9F08BE092E066E071E00E940E8BBC014B
:1090200084E092E00E94ED8BBC018DEF91E00E9404
:10903000ED8BBC0186EF91E00E94ED8B8091AE023A
:109040009091AF02079771F49091BB038091410119
:10905000981741F480912D01882321F48091EC012F
:109060008823A1F18BEE96E360E040E00E94987EB9
:109070008BEE96E367E879E00E946C878091EF01C0
:10908000E82FF0E0EE0FFF1FED51FD4F6591749159
:109090008E010F5F1F4FC8010E941E08E091EF0173
:1090A000F0E0E25DFE4F8BEE96E3608140E00E94CF
:1090B000987E8BEE96E3B8010E9494888091BB0362
:1090C0008093410110922D011092EC018091352B7B
:1090D00090E025E23DE0829FF001839FF00D929F9A
:1090E000F00D1124E15EFF4E8081E82FF0E0EE0FDD
:1090F000FF1FED50FD4F659174917E010894E11CB6
:10910000F11CC7010E941E088E010C5F1D4FC80193
:10911000B7010E94DA8A82E192E0B8010E94ED8BE9
:10912000C8010E941A8C8091F535E82FF0E0EE0F0F
:10913000FF1FEF58FC4F65917491C7010E941E08F4
:109140008E01055F1D4FC801B7010E94DA8A89E1CF
:1091500092E0B8010E94ED8BC8010E941A8C8E012A
:109160000E5E1D4F60915E0170E063507040C8015B
:109170004AE00E94588B80E292E0B8010E94ED8B99
:10918000C8010E941A8C8E01075E1D4FC80160E065
:1091900071E00E94DA8A87E292E0B8010E94ED8BCA
:1091A000C8010E941A8CF0E2AF2EF2E0BF2EAC0E86
:1091B000BD1EC50162E172E00E94048CE7E2CE2E82
:1091C000E2E0DE2ECC0EDD1EC60169E172E00E94F7
:1091D000048C7EE2E72E72E0F72EEC0EFD1EC70136
:1091E00060E272E00E94048C8E010B5C1D4FC8018E
:1091F00067E272E00E94048CC501B601A7019801E4
:109200000E94C73AC8010E941A8CC7010E941A8C9A
:10921000C6010E941A8CC5010E941A8C87E090E05A
:109220000C9445518091AE029091AF020697A9F03F
:109230008BE092E066E071E00E940E8BBC0184E05E
:1092400092E00E94ED8BBC018DEF91E00E94ED8BCE
:10925000BC0186EF91E00E94ED8BE091E636F0E0F4
:10926000E854F94C928980911137981771F084E095
:1092700092E066E071E00E940E8BE091E636F0E04D
:10928000E854F94C8289809311378091AE02909115
:10929000AF02069741F480912D01882321F480913B
:1092A000EC018823B1F18BEE96E360E040E00E9490
:1092B000987E8BEE96E366E779E00E946C8780915A
:1092C000EF01E82FF0E0EE0FFF1FED55FD4F659128
:1092D00074918E010F5F1F4FC8010E941E08E0911C
:1092E000EF01F0E0E25DFE4F8BEE96E3608140E03F
:1092F0000E94987E8BEE96E3B8010E94948886E0E7
:1093000090E09093AF028093AE0210922D011092E4
:10931000EC01E091E636F0E0E854F94C8081E82F6A
:10932000F0E0EE0FFF1FEB5DFC4F659174917E0145
:109330000894E11CF11CC7010E941E088E01045C08
:109340001D4F6091E63670E06F5F7F4FC8014AE0C5
:109350000E94588B82E192E0B8010E94ED8BC80117
:109360000E941A8C8E010D5B1D4FC801B7010E942F
:10937000DA8A89E192E0B8010E94ED8BC8010E946F
:109380001A8C8091E636E82FF0E0E854F94C828997
:109390009E01265B3D4F882331F0C90160E070E0FB
:1093A0000E94DA8A08C0628170E06F5F7F4FC90156
:1093B0004AE00E94588B8E01065B1D4F80E292E0CE
:1093C000B8010E94ED8BC8010E941A8C8E010F5AC1
:1093D0001D4FE091E636F0E0EE0FFF1FEE0FFF1F8E
:1093E000E454F94C608171818281938120E030E006
:1093F00048EC52E40E94DE8D0E94FC8C9B01AC0183
:10940000C801622F4AE00E94898B87E292E0B8018E
:109410000E94ED8BC8010E941A8C38E5A32E32E021
:10942000B32EAC0EBD1EC50162E172E00E94048C39
:109430002FE5C22E22E0D22ECC0EDD1EC60169E140
:1094400072E00E94048C96E6E92E92E0F92EEC0E72
:10945000FD1EC70160E272E00E94048C8E01035978
:109460001D4FC80167E272E00E94048CC501B6017D
:10947000A70198010E94C73AC8010E941A8CC7012F
:109480000E941A8CC6010E941A8CC5010E941A8C77
:10949000E091E636F0E0E854F94C8289882309F43B
:1094A000F8C60E94DF39F5C68091AE029091AF02F6
:1094B0000997A9F08BE092E066E071E00E940E8BC4
:1094C000BC0184E092E00E94ED8BBC018DEF91E045
:1094D0000E94ED8BBC0186EF91E00E94ED8B8BEE3C
:1094E00096E360E040E00E94987E8091B102209176
:1094F000AE023091AF02803109F044C0293031050D
:1095000069F480912D01882349F480910F378031CF
:1095100029F48091EC01882309F475C08BEE96E361
:1095200065E679E00E946C878091EF01E82FF0E01A
:10953000EE0FFF1FED53FD4F659174918E010F5F8C
:109540001F4FC8010E941E08E091EF01F0E0E25DAC
:10955000FE4F8BEE96E3608140E00E94987E8BEE9A
:1095600096E3B8010E94948889E090E09093AF025E
:109570008093AE021092EC0110922D0180E1809355
:109580000F3741C02930310561F480912D018823C6
:1095900041F480910F37803121F08091EC018823D4
:1095A00091F18BEE96E364E579E00E946C878091FF
:1095B000EF01E82FF0E0EE0FFF1FE554FD4F65913E
:1095C00074918E010F5F1F4FC8010E941E08E09129
:1095D000EF01F0E0E25DFE4F8BEE96E3608140E04C
:1095E0000E94987E8BEE96E3B8010E94948889E0F1
:1095F00090E09093AF028093AE021092EC01109233
:109600002D0110920F372091352B30E04091B1029F
:10961000C42EDD2480914C0290E0DC01AA0FBB1F18
:10962000A80FB91F84EC90E0C89EB001C99E700DD0
:10963000D89E700D11246A0F7B1F85E29DE0289F44
:109640007001299FF00C389FF00C11246E0D7F1DC6
:10965000FB01E352FC4F80808694869486944031CF
:10966000F1F4FD01EE0DFF1DDF01AB5DBF4E9C91DE
:10967000929596959695937011968C918770880F18
:10968000880F892BA82EBB2460EF7FEFA60EB71E94
:10969000EA5DFF4E908096949694969419C0FB01D3
:1096A000E452FC4F2081922F929596959695937057
:1096B00081818770880F880F892BA82EBB2480EFAB
:1096C0009FEFA80EB91E922E969496949FE0992231
:1096D0008E010C581D4FEFE5FBE2CE0EDF1EF601AA
:1096E000608170E06F5F7F4FC8014AE00E94588B35
:1096F000CE0185589D4FB8010E940F8C80913A2B66
:10970000882311F460E201C06EE7ABE7CA2EA2E045
:10971000DA2ECC0EDD1EC6010E94928A8C01F2E880
:10972000EF2EF2E0FF2EEC0EFD1EE091B102F0E014
:10973000E25BF44D608170E06F5F7F4FC7014AE0EC
:109740000E94588BC801B7010E94A38ABC018E01F8
:1097500007571D4FC8010E94048C82E192E0B801B6
:109760000E94ED8BC8010E941A8CC7010E941A8CBE
:10977000C6010E94208CCE018C589D4F0E941A8CED
:10978000B7FC30C0E7E9CE2EE2E0DE2ECC0EDD1EC7
:10979000C60168E171E00E94F48A70E9E72E72E088
:1097A000F72EEC0EFD1EC701B5014AE00E94588B52
:1097B000C601B7010E94A38ABC018E0102561D4F4B
:1097C000C8010E94048C89E192E0B8010E94ED8BEF
:1097D000C8010E941A8CC7010E941A8CC6010E94FF
:1097E000208C10C08E010B551D4FC801B5014AE0F9
:1097F0000E94588B89E192E0B8010E94ED8BC8016C
:109800000E941A8CE92DF0E0EE0FFF1FEB5FFC4F7A
:10981000659174918E010F5F1F4FC8010E941E0851
:1098200080E292E0B8010E940E8B2091352B30E04F
:1098300080914C0290E0FC01EE0FFF1FE80FF91F32
:1098400085E29DE0289FD001299FB00D389FB00D83
:109850001124EA0FFB1FEB5DFF4E608166956F716F
:10986000262F2F5FA05EBF4EAC91A03619F4220FB9
:10987000220F03C0A03309F4220F8091B10280317E
:10988000E1F4CE0184559D4F2A1729F462E171E07D
:109890000E94DA8A06C070E06F5F7F4F4AE00E9444
:1098A000588B8E0104551D4F87E292E0B8010E944B
:1098B000ED8BC8010E941A8C51C041ECC42E42E0CD
:1098C000D42ECC0EDD1E882041F4C6016AE171E081
:1098D0000E94DA8AEE24FF2428C03AEBE32E32E01D
:1098E000F32EEC0EFD1EC7016EE171E00E94F48ABA
:1098F0008E010D541D4FE82DF0E0EC5CFE4F6081B1
:1099000080E891E070E00E94808EC8014AE00E94E9
:10991000588BC701B8010E94A38ABC01C6010E94EE
:10992000048CEE24E394FF24F3948E010F531D4F17
:1099300087E292E0B8010E94ED8BC8010E941A8C68
:10994000FF2029F0CE018D549D4F0E941A8CEE20ED
:1099500029F0CE0186549D4F0E94208C28ECA22E27
:1099600022E0B22EAC0EBD1EC50162E172E00E9483
:10997000048C9FECC92E92E0D92ECC0EDD1EC601C0
:1099800069E172E00E94048C86EDE82E82E0F82EF8
:10999000EC0EFD1EC70160E272E00E94048C8E0195
:1099A00003521D4FC80167E272E00E94048CC5019A
:1099B000B601A70198010E94C73AC8010E941A8CFB
:1099C000C7010E941A8CC6010E941A8CC5010E9410
:1099D0001A8C8091B102803109F05BC48BEE96E362
:1099E0006FE041E00E94987E80914C0290E02091CF
:1099F000352B30E0FC01EE0FFF1FE80FF91F85E269
:109A00009DE0AC01249FC001259F900D349F900DD7
:109A10001124E80FF91FE95DFF4E808187FF05C023
:109A20008BEE96E362E579E049C08BEE96E366E162
:109A300071E00E9494882DC485E090E09093AF027D
:109A40008093AE028BEE96E360E040E00E94987E49
:109A50008BEE96E361E479E00E946C878BEE96E3EF
:109A600060E041E00E94987E0E947D398BEE96E393
:109A700062E041E00E94987E8091CE36882329F0F2
:109A80008BEE96E36DE379E004C08BEE96E36AE338
:109A900079E00E946C878BEE96E36AE041E00E94D9
:109AA000987E8091F202882329F08BEE96E366E39C
:109AB00079E004C08BEE96E363E379E00E946C8763
:109AC000E8C38091AE029091AF020197A9F08BE0BC
:109AD00092E066E071E00E940E8BBC0184E092E0AF
:109AE0000E94ED8BBC018DEF91E00E94ED8BBC01DB
:109AF00086EF91E00E94ED8B8091AE029091AF02D3
:109B0000019741F480912D01882321F48091EC018B
:109B1000882381F18BEE96E360E040E00E94987E1E
:109B20008BEE96E362E279E00E946C878091EF0110
:109B3000E82FF0E0EE0FFF1FED52FD4F659174919D
:109B40008E010F5F1F4FC8010E941E08E091EF01B8
:109B5000F0E0E25DFE4F8BEE96E3608140E00E9414
:109B6000987E8BEE96E3B8010E94948810922D01A6
:109B70001092EC018E010C511D4F6091F53370E095
:109B80006F5F7F4FC8014AE00E94588B82E192E0EC
:109B9000B8010E94ED8BC8010E941A8C8E010551FC
:109BA0001D4F6091F6337091F7336F5F7F4FC8019F
:109BB0004AE00E94588B89E192E0B8010E94ED8B47
:109BC000C8010E941A8CB2EFCB2EB2E0DB2ECC0E75
:109BD000DD1EE091F633F091F733EC50FC4C6185DB
:109BE00062956F706F5BC6010E94BB8BE12CA3E096
:109BF000FA2EEC0EFD1EC701B6010E940F8CE091FB
:109C0000F633F091F733EC50FC4C21858E01075070
:109C10001D4F622F70E06F5F7F4F822F82958F7094
:109C200090E0F4E0880F991FFA95E1F7681B790B33
:109C3000C8014AE00E94588BC701B8010E94A38A5C
:109C4000BC0180E292E00E94ED8BC8010E941A8C58
:109C5000C7010E94208CC6010E941A8C8EE292E0FD
:109C600060E272E00E94ED8B88E08093F0018E014B
:109C7000095F1C4F6091FA337091FB336F5F7F4F28
:109C8000C8014AE00E94278B87E292E0B8010E9457
:109C9000ED8BC8010E941A8CEEE0AE2EE3E0BE2EE2
:109CA000AC0EBD1EC50162E172E00E94048C75E13C
:109CB000C72E73E0D72ECC0EDD1EC60169E172E01F
:109CC0000E94048C6CE1E62E63E0F62EEC0EFD1E85
:109CD000C70160E272E00E94048C8E010D5D1C4F92
:109CE000C80167E272E00E94048CC501B601A701B9
:109CF00098010E94C73AC8010E941A8CC7010E94AD
:109D00001A8CC6010E941A8CC5010E941A8C81E02F
:109D100090E0BBC28091AE029091AF02892BC9F452
:109D200080912D018823A9F48091EC01882389F486
:109D30008091143790E02091F6333091F7338217F9
:109D4000930739F4909113378091F533981709F4FC
:109D5000ADC08BEE96E360E040E00E94987E0E94EA
:109D60007D398BEE96E360E040E00E94987E8BEEBA
:109D700096E365E179E00E946C876091F53370E0CD
:109D80006F5F7F4F8BEE96E34AE050E00E94818840
:109D90008091F533809313378BEE96E360E041E0DA
:109DA0000E94987E0E947D398BEE96E360E041E050
:109DB0000E94987E8BEE96E360E179E00E946C87CA
:109DC0008091F633809314376091F6337091F733B6
:109DD00077FF02C060E070E06F5F7F4F8BEE96E32D
:109DE0004AE050E00E9481888BEE96E368E041E013
:109DF0000E94987E8BEE96E36AE079E00E946C8781
:109E00005AE2C52E53E0D52ECC0EDD1EE091F6337E
:109E1000F091F733EC50FC4C618562956F706F5B8D
:109E2000C6010E94BB8B48E3E42E43E0F42EEC0E07
:109E3000FD1EC701B6010E940F8CE091F633F09130
:109E4000F733EC50FC4C21858E010F5C1C4F622FC8
:109E500070E06F5F7F4F822F82958F7090E034E0CB
:109E6000880F991F3A95E1F7681B790BC8014AE002
:109E70000E94588BC701B8010E94A38ABC0180E2EE
:109E800092E00E94ED8BC8010E941A8CC7010E94CB
:109E9000208CC6010E941A8C8BEE96E360E272E081
:109EA0000E94358910922D011092EC011092AF02A0
:109EB0001092AE02EEC18091AE029091AF020D976A
:109EC000A9F08BE092E066E071E00E940E8BBC018D
:109ED00084E092E00E94ED8BBC018DEF91E00E9446
:109EE000ED8BBC0186EF91E00E94ED8B8091AE027C
:109EF0009091AF020D9741F480912D01882321F4B8
:109F00008091EC01882381F110922D011092EC01D7
:109F10008BEE96E360E040E00E94987E8BEE96E345
:109F200069EF78E00E946C878091EF01E82FF0E004
:109F3000EE0FFF1FE552FD4F659174918E010F5F8B
:109F40001F4FC8010E941E08E091EF01F0E0E25DA2
:109F5000FE4F8BEE96E3608140E00E94987E8BEE90
:109F600096E3B8010E9494888E01015C1C4FC801E1
:109F7000609139364AE00E94898B82E192E0B80113
:109F80000E94ED8BC8010E941A8C8E010A5B1C4F47
:109F9000C80160913A364AE00E94898B89E192E0DB
:109FA000B8010E94ED8BC8010E941A8C8E01035BE0
:109FB0001C4FC80160913B364AE00E94898B80E2C9
:109FC00092E0B8010E94ED8BC8010E941A8C8E01AC
:109FD0000C5A1C4FC80160913C364AE00E94898BA4
:109FE00087E292E0B8010E94ED8BC8010E941A8CB2
:109FF0009BE5A92E93E0B92EAC0EBD1EC50162E112
:10A0000072E00E94048C82E6C82E83E0D82ECC0E2B
:10A01000DD1EC60169E172E00E94048C09E6E02EB3
:10A0200003E0F02EEC0EFD1EC70160E272E00E941C
:10A03000048C8E0100591C4FC80167E272E00E9437
:10A04000048CC501B601A70198010E94C73AC80156
:10A050000E941A8CC7010E941A8CC6010E941A8C99
:10A06000C5010E941A8C8DE090E00FC18091AE0274
:10A070009091AF020E9729F48091EC01882309F4A6
:10A080006CC01092EC018BEE96E360E040E00E9421
:10A09000987E8BEE96E368EE78E00E946C878BEEFC
:10A0A00096E360E041E00E94987E0E947D398BEE4D
:10A0B00096E362E041E00E94987E60914C0270E07D
:10A0C0006F5F7F4F8BEE96E34AE050E00E948188FD
:10A0D0008BEE96E36AE041E00E94987E80914C020C
:10A0E00090E02091B10230E04091352B50E0FC012E
:10A0F000EE0FFF1FE80FF91F84EC90E0BC01269FD4
:10A10000C001279F900D369F900D1124E80FF91F75
:10A1100085E29DE09C01429FC001439F900D529FAC
:10A12000900D1124E80FF91FE252FC4F60816F7708
:10A1300070E0882777FD8095982F0E942A8D2AE06D
:10A1400037ED43E25DE30E94DE8DAB01BC018BEE97
:10A1500096E322E030E00E94328980914C0290E048
:10A160002091B10230E04091352B50E0FC01EE0F20
:10A17000FF1FE80FF91FA4ECEA2EF12C2E9DC00161
:10A180002F9D900D3E9D900D1124E80FF91F05E2C3
:10A190001DE0409FC001419F900D509F900D1124E4
:10A1A000E80FF91FE252FC4F20812F7730E08091B9
:10A1B000103790E02817390709F465C08BEE96E355
:10A1C0006AE041E00E94987E80914C0290E02091EC
:10A1D000B10230E04091352B50E0FC01EE0FFF1F43
:10A1E000E80FF91F2E9DC0012F9D900D3E9D900DF3
:10A1F0001124E80FF91F409FC001419F900D509F0F
:10A20000900D1124E80FF91FE252FC4F60816F7727
:10A2100070E0882777FD8095982F0E942A8D2AE08C
:10A2200037ED43E25DE30E94DE8DAB01BC018BEEB6
:10A2300096E322E030E00E94328980914C0290E067
:10A240002091B10230E04091352B50E0FC01EE0F3F
:10A25000FF1FE80FF91F2E9DC0012F9D900D3E9D01
:10A26000900D1124E80FF91F409FC001419F900DF0
:10A27000509F900D1124E80FF91FE252FC4F80818E
:10A280008F77809310378EE090E09093AF028093A9
:10A29000AE02C158DC4F0FB6F894DEBF0FBECDBF83
:10A2A000CF91DF911F910F91FF90EF90DF90CF90B2
:10A2B000BF90AF909F908F9008959F92AF92BF9262
:10A2C000CF92DF92EF92FF920F931F93DF93CF9382
:10A2D00000D000D00F92CDB7DEB7809146029091AA
:10A2E00047028230910561F10C9751F18091EF01A5
:10A2F00090E061E070E00E946F10282F809146028C
:10A3000090914702049749F48091B102803129F479
:10A31000822F233030F082E004C0822F243008F0F6
:10A3200083E08093EF019091EF0180913D37981782
:10A3300039F090933D3781E080932D0180932C017B
:10A340008091F501882309F4B6C00091B1024091D3
:10A35000352B0031A1F4842F90E025E23DE08C0103
:10A36000029FC001039F900D129F900D11248E5DDE
:10A370009F4E61E041E027E009EB13E01FC010E0D1
:10A3800084EC90E09C01029FC001039F900D129FFE
:10A39000900D112450E025E23DE0B901469F900167
:10A3A000479F300D569F300D1124820F931F055C7F
:10A3B000144D81569B4F61E041E027E00E94CB1095
:10A3C00080918B3682FD07C08091460290914702B2
:10A3D000029709F070C05091B1024091352B503175
:10A3E000A1F4242F30E085E29DE0289FF001299F11
:10A3F000F00D389FF00D1124EE53FC4FE05AF34F4F
:10A400008081E056FC4083831FC0242F30E085E22A
:10A410009DE0289FD001299FB00D389FB00D1124D9
:10A42000252F30E084EC90E0289FF001299FF00D6B
:10A43000389FF00D1124EA0FFB1FE156FB4F80817E
:10A44000AE53BC4F13968C9320E030E004EC10E048
:10A4500065E27DE0FF24F3948091352B90E0209F0E
:10A46000F001219FF00D309FF00D1124DC01A69F1B
:10A47000C001A79F900DB69F900D1124E80FF91F02
:10A48000E156FB4FDC01AE53BC4FAD014D5F5F4F5A
:10A4900013968C9113978083F901E55CF44DF0825B
:10A4A0002F5F3F4F20313105B9F6FD01E05AF34FE0
:10A4B000DA018C9180838091F401882309F4B8C07B
:10A4C0000091B1024091352B0031A1F4842F90E02E
:10A4D00025E23DE0FC01E29FC001E39F900DF29F69
:10A4E000900D11248D5D9F4E61E040E023E009EB6B
:10A4F00013E01FC010E084EC90E09C01029FC001BB
:10A50000039F900D129F900D112450E025E23DE035
:10A51000B901469F9001479F300D569F300D112481
:10A52000820F931F055C144D82569B4F61E040E003
:10A5300023E00E94CB1080918B3682FD07C0809172
:10A54000460290914702029709F072C02091B10231
:10A550004091352B203169F450E085E29DE0489F21
:10A56000F001499FF00D589FF00D1124ED5DFF4E55
:10A5700019C050E030E084EC90E0289FF001299F62
:10A58000F00D389FF00D112485E29DE0DC014A9F1B
:10A59000C0014B9F900D5A9F900D1124E80FF91F99
:10A5A000E256FB4F208185E29DE0489FF001499FE4
:10A5B000F00D589FF00D1124EE53FC4F228320E044
:10A5C00030E004EC10E065E27DE0FF24F39480913C
:10A5D000352B90E0209FF001219FF00D309FF00D72
:10A5E0001124AC01469FC001479F900D569F900DCE
:10A5F0001124E80FF91FE256FB4FDC01AE53BC4FAC
:10A60000AD014E5F5F4F12968C9112978083F901D6
:10A61000E55CF44DF0822F5F3F4F20313105B9F6F4
:10A62000FD01EF59F34FDA018C918083F092B90369
:10A6300080914602909147028630910509F48AC7BD
:10A6400087309105A4F48230910571F18330910532
:10A650002CF4019711F00C940C62C2C58330910563
:10A6600009F4D5C0049711F00C940C6225C389300D
:10A67000910511F40C94195E8A30910554F48730D9
:10A68000910511F40C94C95B089711F00C940C62BD
:10A6900021C68C30910511F40C94D8610D9711F0FE
:10A6A0000C940C620C94EF618091913682FF6AC029
:10A6B0008091352B90E015E2E12E1DE0F12E8E9D6C
:10A6C000F0018F9DF00D9E9DF00D1124EE53FC4F77
:10A6D000D080CF0161E040E02FE308E31BE20E945D
:10A6E000CB108091352B90E08E9DF0018F9DF00D69
:10A6F0009E9DF00D1124EE53FC4F80818D1591F13C
:10A7000020E030E064EC70E045E25DE011E0809133
:10A71000352B90E0269FF001279FF00D369FF00D1E
:10A720001124DC01A49FC001A59F900DB49F900D42
:10A730001124E80FF91FE456FB4FDC01AE53BC4F68
:10A740008C918083F901E55CF44D10832F5F3F4FBE
:10A7500020313105E1F6FD01E15AF34F8C91808300
:10A760001093B9038091B102082F10E0025B144DE1
:10A77000F801F0808F2D90E061E070E00E946F1092
:10A780000C94D05E80914802837059F480913E020F
:10A7900090913F0261E00E94511190933F0280939B
:10A7A0003E0280913E0290913F024F9730F48EE13D
:10A7B00090E090933F0280933E0280913E02909100
:10A7C0003F028A3F910530F08AEF90E090933F027C
:10A7D00080933E0220913E0230913F0280913A37B1
:10A7E00090913B372817390711F40C940C62309381
:10A7F0003B3720933A370E943D2681E080932C011D
:10A8000080914802837009F4D3C50C940C62809146
:10A81000EF018130C1F0813040F0823009F49BC0FB
:10A82000833011F00C940C62FEC180919F3683FD41
:10A8300002C00C94BF5E80918D3682FF02C00C94E2
:10A84000BF5E0C94A85E0091B1024091352B00319F
:10A8500099F5842F90E0B5E2EB2EBDE0FB2EFC01D4
:10A86000EE9DC001EF9D900DFE9D900D1124FC0109
:10A87000EF5DFF4ED080CF0161E040E02FE309EBB8
:10A8800013E00E94CB108091352B90E08E9DF0015B
:10A890008F9DF00D9E9DF00D1124EF5DFF4E4081C8
:10A8A000D41608F0C4C280913602813009F0BFC2CC
:10A8B0008091B1026D2D4CC0242F30E010E0A4EC4B
:10A8C000CA2ED12C0C9DC0010D9D900D1C9D900D8C
:10A8D0001124F5E2EF2EFDE0FF2EA9014E9D90011F
:10A8E0004F9D300D5E9D300D1124820F931FFC0192
:10A8F000E456FB4FB080055C144DCF0161E040E0B1
:10A900002FE30E94CB105091B102252F30E08091AF
:10A91000352B90E02C9DF0012D9DF00D3C9DF00D10
:10A920001124BC016E9DC0016F9D900D7E9D900D08
:10A930001124E80FF91FE456FB4F4081B41608F0CC
:10A9400076C280913602813009F071C2852F6B2D5D
:10A950000E945A1F6CC22091B1024091352B2031C8
:10A9600071F4242F30E085E29DE0289FF001299FBB
:10A97000F00D389FF00D1124E05EFF4E19C030E05D
:10A9800050E084EC90E0289FF001299FF00D389F63
:10A99000F00D112485E29DE0DC014A9FC0014B9F30
:10A9A000900D5A9F900D1124E80FF91FE356FB4FAD
:10A9B00010811831A9F0193128F41C30A9F0103198
:10A9C000B1F410C0103341F0103619F0103279F4A0
:10A9D00005C01092A8360BC081E007C082E005C018
:10A9E00083E003C084E001C085E08093A8368091B5
:10A9F000A83661E00E94A010863008F085E08093C0
:10AA0000A83680911C37882371F48CE197E30E946B
:10AA10003487892B41F08091A836809339378CE1B7
:10AA200097E30E943E879091A83680913937981716
:10AA300011F40C940C629093393781E080932C01CF
:10AA4000E091B102E03119F48093B90304C0F0E061
:10AA5000E55CF44D80838091A8368230B1F083307C
:10AA600028F4882351F0813021F50AC08430B1F0F8
:10AA7000843070F08530E9F417C0EE2410E602C08F
:10AA8000EE2410E3EFE1FE2E14C0EE2410E2FACF24
:10AA900074E0E72E18E16BE1F62E0BC058E0E52ECE
:10AAA00010E147E1F42E05C03AE0E32E1CE025E179
:10AAB000F22E8091B1026E2D4F2D0E94A212809134
:10AAC000B102803191F48091352B90E025E23DE098
:10AAD000829FF001839FF00D929FF00D1124E05EA4
:10AAE000FF4E812F60810E94F30B2091B1024091B3
:10AAF000352B203171F4242F30E085E29DE0289F32
:10AB0000F001299FF00D389FF00D1124E05EFF4EFB
:10AB100019C030E050E084EC90E0289FF001299FBC
:10AB2000F00D389FF00D112485E29DE09C01429FBD
:10AB3000C001439F900D529F900D1124E80FF91F03
:10AB4000E356FB4F10838091953682FF70C1509180
:10AB5000B1024091352B5031A1F4242F30E085E231
:10AB60009DE0289FF001299FF00D389FF00D1124E2
:10AB7000EE53FC4FE25AF34F8081EE55FC40818347
:10AB80001FC0242F30E085E29DE0289FD001299F3F
:10AB9000B00D389FB00D1124252F30E084EC90E0EB
:10ABA000289FF001299FF00D389FF00D1124EA0F26
:10ABB000FB1FE356FB4F8081AE53BC4F11968C9325
:10ABC00000E010E094ECA92EB12C85E2C82E8DE0B7
:10ABD000D82E992493948091352B90E00A9DD00132
:10ABE0000B9DB00D1A9DB00D11248C9DF0018D9D13
:10ABF000F00D9C9DF00D1124AE0FBF1FA356BB4F4F
:10AC0000EE53FC4F81818C93802F6E2D4F2D0E942F
:10AC1000A212F801E55CF44D90820F5F1F4F0031E6
:10AC20001105C9F65CC280919F3683FFD2C2409164
:10AC3000B1028091352B90E025E23DE0829FF0014A
:10AC4000839FF00D929FF00D1124EE53FC4FE40F03
:10AC5000F11D8781882309F4A1C240E050E0A4ECF3
:10AC6000B0E065E27DE08091B10290E02091352B6B
:10AC700030E0FA01EE0FFF1FE40FF51F8C010A9F71
:10AC8000C0010B9F900D1A9F900D1124E80FF91F22
:10AC9000269FC001279F900D369F900D1124E80F2D
:10ACA000F91FE452FC4F8081826080834F5F5F4FC9
:10ACB00040345105C1F672C20091B1026091EF01BA
:10ACC000003109F065C08091352B90E025E23DE030
:10ACD000829FF001839FF00D929FF00D1124E15EA1
:10ACE000FF4E8081613051F1613028F0623011F007
:10ACF0000C940C6238C061E00E94A010482F89308B
:10AD000008F048E080913837481739F040933837D9
:10AD100081E08093B90380932C018091352B90E0E2
:10AD200025E23DE0829FF001839FF00D929FF00DA0
:10AD30001124E15EFF4E40830C940C628091F53546
:10AD400061E00E94A010982F8C3008F09BE0909357
:10AD5000F53580913737981711F40C940C62909365
:10AD600037370C94EB6180915E0161E00E94A01086
:10AD7000982F883008F097E090935E0180913637E5
:10AD8000981711F40C940C62909336370C94EB6185
:10AD9000613051F1613040F0623009F44CC06330F1
:10ADA00011F00C940C62B5C180919F3683FF85C56C
:10ADB00080918D3682FD81C590E080913A2B882369
:10ADC00009F491E090933A2B992351F0E091B1026C
:10ADD000F0E0DF01A15AB44D8C91E25BF44D808329
:10ADE00081E080932C0169C510E084EC90E09C0127
:10ADF000029FC001039F900D129F900D112420917E
:10AE0000352B30E045E25DE0B901649F9001659F1C
:10AE1000300D749F300D1124820F931F055C144D6B
:10AE200084569B4F61E040E02FE30E94CB100E94CC
:10AE300027250C940C62402F50E02091352B30E0F8
:10AE400084EC90E0489FF001499FF00D589FF00D71
:10AE5000112485E29DE0DC012A9FC0012B9F900D0B
:10AE60003A9F900D1124E80FF91FE356FB4F108114
:10AE70001831A9F0193128F41C30A9F01031B1F4BF
:10AE800010C0103341F0103619F0103279F405C0BB
:10AE90001092A8360BC081E007C082E005C083E0B5
:10AEA00003C084E001C085E08093A8368091A83675
:10AEB00061E00E94A010863008F085E08093A836FB
:10AEC00080912437882371F484E297E30E943487C9
:10AED000892B41F08091A8368093353784E297E33F
:10AEE0000E943E879091A83680913537981711F4CB
:10AEF0000C940C629093353781E080932C01E091A3
:10AF0000B102E03119F48093B90304C0F0E0E55CCC
:10AF1000F44D80838091A8368230A9F0833028F4E4
:10AF2000882351F0813011F509C08430A1F08430BC
:10AF300060F08530D9F415C010E601C010E3EE24AE
:10AF4000EFE1FE2E13C010E2FACF18E174E0E72E15
:10AF50006BE1F62E0BC010E158E0E52E47E1F42E30
:10AF600005C01CE03AE0E32E25E1F22E8091B1020B
:10AF70006E2D4F2D0E94A2128091B102803191F46A
:10AF80008091352B90E025E23DE0829FF001839F88
:10AF9000F00D929FF00D1124E05EFF4E812F608135
:10AFA0000E94F30B2091B1024091352B203171F4B6
:10AFB000242F30E085E29DE0289FF001299FF00DCD
:10AFC000389FF00D1124E05EFF4E19C030E050E0D4
:10AFD00084EC90E0289FF001299FF00D389FF00D40
:10AFE000112485E29DE09C01429FC001439F900D8A
:10AFF000529F900D1124E80FF91FE356FB4F108369
:10B000008091953682FF13CF5091B1024091352B3C
:10B010005031A1F4242F30E085E29DE0289FF0011B
:10B02000299FF00D389FF00D1124EE53FC4FE25A8A
:10B03000F34F8081EE55FC4081831FC0242F30E008
:10B0400085E29DE0289FD001299FB00D389FB00D6B
:10B050001124252F30E084EC90E0289FF001299FF7
:10B06000F00D389FF00D1124EA0FFB1FE356FB4F44
:10B070008081AE53BC4F11968C9300E010E094ECAD
:10B08000A92EB12C85E2C82E8DE0D82E9924939458
:10B090008091352B90E00A9DD0010B9DB00D1A9D3B
:10B0A000B00D11248C9DF0018D9DF00D9C9DF00D37
:10B0B0001124AE0FBF1FA356BB4FEE53FC4F81812F
:10B0C0008C93802F6E2D4F2D0E94A212F801E55C0B
:10B0D000F44D90820F5F1F4F00311105C9F680E1DA
:10B0E0006E2D4F2D0E94A2128091352B90E025E20B
:10B0F0003DE0829FF001839FF00D929FF00D11249F
:10B10000EE53FC4F8181E25AF34F80839092B90352
:10B110008ECE80919F3683FF5CC08091352B90E06E
:10B1200025E23DE0829FF001839FF00D929FF00D9C
:10B130001124EE53FC4FE00FF11D8781882371F13C
:10B1400040E050E0A4ECB0E065E27DE08091B10227
:10B1500090E02091352B30E0FA01EE0FFF1FE40F55
:10B16000F51F8C010A9FC0010B9F900D1A9F900D37
:10B170001124E80FF91F269FC001279F900D369FCD
:10B18000900D1124E80FF91FE452FC4F808182607A
:10B1900080834F5F5F4F40345105C1F68091352B5E
:10B1A00090E04091B10225E23DE0829FF001839F53
:10B1B000F00D929FF00D1124EE53FC4FE40FF11DA2
:10B1C00090E08781882309F491E0978381E0809360
:10B1D0002C0181EB92E061E040E020E10C940862F8
:10B1E0008091B302E091F633F091F733EC50FC4CD0
:10B1F0009185981741F081E08093ED01809146029E
:10B200008093EE0102C01092ED018091EF01813038
:10B2100091F0813038F0823029F1833011F00C94B4
:10B220000C6241C085EF93E361E040E02FE000EF66
:10B2300015E30C940A6280919F3682FF05C086EF69
:10B2400093E36AE070E004C086EF93E361E070E0AE
:10B2500040E050E023EF31E000E010E00E940312F4
:10B260000C940C628091F6339091F73383509C4C90
:10B2700061E040E02FE701EF15E30E94CB108091E1
:10B280009F3682FD02C00C940C62E091F633F0917F
:10B29000F733EC50FC4C81858093B50281E08093BC
:10B2A000362B0C940C6280919F3682FF05C08AEF8A
:10B2B00093E36AE070E004C08AEF93E361E070E03A
:10B2C00040E050E023EF31E000E010E00E948E11FA
:10B2D0000C940C628091F101813029F0823011F0E0
:10B2E0000C940C6295C08091EF01813089F181301E
:10B2F00040F0823009F46BC0833011F00C940C6282
:10B300006CC080914802837061E00E94A010582FA9
:10B310005370533009F452E0852F837040914802F6
:10B320004C7F482B40934802252F30E080913437E2
:10B3300090E02817390711F40C940C6250933437BD
:10B3400044604093480281E0809337020C94EC61A2
:10B35000809140029091410261E00E9451119C0154
:10B360008E31910518F42EE130E005C08B3F910538
:10B3700010F02AEF30E03093410220934002809198
:10B38000333790E02817390711F40C940C6220939E
:10B3900033370E943D268091400290914102909364
:10B3A0003F0280933E0281E08093370280932C011C
:10B3B0008091CA36882319F080E00E942D16809172
:10B3C000CB36882311F40C940C6281E02AC18DE302
:10B3D00092E061E042E02AE02DC08AE392E061E081
:10B3E00040E026E007E312E00E94CB108091480283
:10B3F0008370813011F00C940C6280913A02853098
:10B4000010F40C940C6284E080933A020C940C6269
:10B410008091EF01813089F0813038F0823081F005
:10B42000833011F00C940C6250C086E392E061E02E
:10B4300040E021E007E312E0EDC785E392E0F7CFBB
:10B4400080914402909145020090B40202C096950A
:10B4500087950A94E2F781708983CE01019661E0B5
:10B4600040E021E007E312E00E94CB108981409187
:10B47000B4022091440230914502882391F081E08A
:10B4800090E0A0E0B0E004C0880F991FAA1FBB1F86
:10B490004A95D2F7282B392B30934502209344024A
:10B4A000BBC781E090E0A0E0B0E004C0880F991F26
:10B4B000AA1FBB1F4A95D2F78095909582239323AC
:10B4C0009093450280934402A7C7809142029091D5
:10B4D00043020090B40202C0969587950A94E2F761
:10B4E00081708983CE01019661E040E021E007E3AD
:10B4F00012E00E94CB1089814091B4022091420257
:10B5000030914302882391F081E090E0A0E0B0E028
:10B5100004C0880F991FAA1FBB1F4A95D2F7282B7A
:10B52000392B309343022093420276C781E090E0AA
:10B53000A0E0B0E004C0880F991FAA1FBB1F4A9566
:10B54000D2F7809590958223932390934302809322
:10B55000420262C78091EF01813071F0813030F09A
:10B56000823099F0833009F057C75EC086EE96E3CB
:10B5700061E040E021E04CC78091E63690E08854DD
:10B58000994C61E040E024E030C080919F3683FF19
:10B5900011C08091E636E82FF0E0E854F94C90E0D5
:10B5A0008289882309F491E0928B81E08093E736C9
:10B5B00080932C018091E636282F30E0F901E85481
:10B5C000F94C82898823A1F480918B362E5F3F4FFE
:10B5D00082FF05C0C9018854994C6AE004C0C901C2
:10B5E0008854994C61E040E02EEF07EE16E312C755
:10B5F000813009F011C7F488C9018453994C61E086
:10B6000040E027E007EE16E30E94CB109091E6366B
:10B61000E92FF0E0E854F94C84898F1509F4FCC651
:10B62000892F0E942D16F8C680918B360091E63640
:10B6300082FF11C010E0000F111F000F111F0454F2
:10B64000194CD8016D917D918D919C912DEC3CEC24
:10B650004CEC5DE310C010E0000F111F000F111F34
:10B660000454194CD8016D917D918D919C912AE0E3
:10B6700037ED43E25CE30E944112F801608371837D
:10B68000828393838091E636C82EDD24F601EE0F87
:10B69000FF1FEE0FFF1FE454F94CE080F1800281A0
:10B6A0001381C801B70120E030E040E050E00E9483
:10B6B0008B8C88235CF40F2EF0E0EF2EF0E0FF2E51
:10B6C000F0E00F2FF0E01F2FF02D14C0C801B701DC
:10B6D00020E030E040E85FE30E94DA8D181654F471
:10B6E0000F2EF0E0EF2EF0E0FF2EF0E80F2FFFE33B
:10B6F0001F2FF02DCC0CDD1CCC0CDD1C2CEB36E30D
:10B70000C20ED31ED601ED92FD920D931C9313979A
:10B71000E091E636F0E0EE0FFF1FEE0FFF1FE20FA5
:10B72000F31FE080F18002811381C801B7012091ED
:10B730002F373091303740913137509132370E9456
:10B740008B8C882369F0E0922F37F092303700938A
:10B7500031371093323781E08093E73680932C01A4
:10B7600080919F3683FF58C6E091E636F0E0EE0FF9
:10B77000FF1FEE0FFF1FE454F94C80E090E0A0E8BB
:10B78000BFE380839183A283B38381E08093E73614
:10B7900023C62091352B30E080914C0290E0DC01F3
:10B7A000AA0FBB1FA80FB91F85E29DE0F901E89F12
:10B7B0009001E99F300DF89F300D1124A20FB31FA7
:10B7C000FD01E95DFF4E8081F82FFF70FD838295BA
:10B7D00087708983215E3F4EF9011081AB5DBF4EBA
:10B7E0000C9106950F718091BB03813009F053C015
:10B7F0008091EF01813049F1813020F0823009F0F1
:10B800004AC035C0812F61E00E94A010182F8930F6
:10B8100008F018E080912E37181739F010932E3762
:10B8200081E08093B90380932C018091352B90E0C7
:10B8300025E23DE0829FF001839FF00D929FF00D85
:10B840001124E15EFF4E108326C08091F53561E042
:10B850000E94A010982F8C3008F09BE09093F53553
:10B8600080912D379817B9F090932D3711C08091A2
:10B870005E0161E00E94A010982F883008F097E0E8
:10B8800090935E0180912C37981729F090932C3774
:10B8900081E080932C018091BB03882309F0BCC513
:10B8A0008091EF018130E9F0813038F0823009F485
:10B8B0001CC1833009F0B0C599C180913A2B88230F
:10B8C00009F0AAC58091B102082F10E0025B144D67
:10B8D000D801FC908F2D61E00E94A010F8018083B8
:10B8E00061C223B122702093FE3593B19170909381
:10B8F000FF35222371F480910036882351F099237B
:10B9000021F4EE24EA94FE2C06C071E0E72EF12C1F
:10B9100002C0EE24FF2420930036E114F10409F460
:10B920007BC580918B3682FFAFC08091352B90E034
:10B9300025E23DE0829FF001839FF00D929FF00D84
:10B940001124EF5DFF4E008180918D3682FD02C093
:10B9500040E02EC080915E2B813061F0813028F074
:10B96000823079F08330D9F413C00031C0F040E068
:10B970000FE016C0003218F040E10FE111C040E1C5
:10B980000FC0003318F040E20FE20AC040E208C0E6
:10B99000003418F040E30FE303C040E301C040E08F
:10B9A00080914C02841710F0081710F440934C0259
:10B9B0002091352B30E0812F90E0FC01EE0FFF1F2E
:10B9C000E80FF91FEE0FFF1FEE0FFF1FBF016854B6
:10B9D0007C4F542FAA24A394BB24B39485E29DE00A
:10B9E000289FD001299FB00D389FB00D1124E35539
:10B9F000FC4FE491CE2EDD24FB018491682F70E092
:10BA000029C0252F30E0F901EE0FFF1FE20FF31FD1
:10BA1000EA0FFB1FE95DFF4EE0818E2F8F7090E0F3
:10BA20008C159D0521F4E295E77009F4AA24861788
:10BA3000970779F4F901EE0FFF1FE20FF31FEA0FEA
:10BA4000FB1FE95DFF4E808182958770873009F486
:10BA5000BB245F5F0517A8F6142F13C0F1E0EF16A3
:10BA6000F10419F4BB2041F40BC02FEFE2162FEFC5
:10BA7000F20631F4AA2021F0812FB7010E94D40CE4
:10BA80001F5F011758F72DC08091953683FF24C0A2
:10BA900020E030E065E27DE04D814F708091352BF4
:10BAA00090E0F901EE0FFF1FE20FF31FDC01A69FEC
:10BAB000C001A79F900DB69F900D1124E80FF91FAC
:10BAC000E95DFF4E8081807F842B80832F5F3F4F15
:10BAD0002034310519F705C080914C02B7010E944E
:10BAE000D40C81E08093B90377C48091953683FFAD
:10BAF0004EC023B122702093FE3593B19170909384
:10BB0000FF35222361F480910036882341F0992388
:10BB100019F48FEF9FEF05C081E090E002C080E054
:10BB200090E0209300368093EC028823C9F140E036
:10BB300050E065E27DE08091352B90E0FA01EE0F58
:10BB4000FF1FE40FF51F8C01069FC001079F900D9A
:10BB5000169F900D1124E80FF91FE95DFF4E20811B
:10BB6000822F82958F709091EC02890F8770829559
:10BB7000807F2F78282B20834F5F5F4F4034510503
:10BB8000D1F681E08093B90380932C0109C0CE01E6
:10BB9000019661E040E027E009EB13E00E94CB1042
:10BBA00080919F3683FF02C083E0898380914C029D
:10BBB00090E02091352B30E0FC01EE0FFF1FE80FE5
:10BBC000F91F85E29DE0AC01249FC001259F900DE7
:10BBD000349F900D1124E80FF91FE95DFF4E998104
:10BBE00097709295907F80818F78DFC3802F0E941D
:10BBF000F81020914C0230E04091352B50E0F901D3
:10BC0000EE0FFF1FE20FF31F25E23DE0B901469F53
:10BC10009001479F300D569F300D1124E20FF31F06
:10BC2000EB5DFF4E8F71880F9081917C982B9083F4
:10BC3000F3C31C822091B1024091352B80914C02BC
:10BC4000203199F590E0242F30E0FC01EE0FFF1F2A
:10BC5000E80FF91F85E29DE0D901A89F9001A99FF7
:10BC6000300DB89F300D1124E20FF31FDF01AB5DE3
:10BC7000BF4E4C91942F92959695969593701196F0
:10BC80008C918770880F880F892B8983205E3F4EA7
:10BC9000D9013C91EA5DFF4E808186958695869517
:10BCA0008A83842F86958F7141C090E030E050E008
:10BCB000FC01EE0FFF1FE80FF91F84EC90E08901F3
:10BCC000089F9001099F300D189F300D1124E20F3D
:10BCD000F31F85E29DE0BA01689FA001699F500DA6
:10BCE000789F500D1124E40FF51FDF01A452BC4FC3
:10BCF0009C91692F629566956695637011968C91FB
:10BD00008770880F880F862B8983240F351F235651
:10BD10003B4FD9013C91969596959F709A83E3523B
:10BD2000FC4F80818695869586958B839091EF0157
:10BD3000913009F44CC0913038F0923009F478C158
:10BD4000933009F069C361C280919F3683FF17C0A9
:10BD500090E080913A2B882309F491E090933A2B5C
:10BD6000992351F0E091B102F0E0DF01A15AB44D06
:10BD70008C91E25BF44D808381E080932C01809173
:10BD80003A2B882309F048C38091B102082F10E0B4
:10BD9000025B144DF801F0808F2D61E00E94A0102D
:10BDA000D8018C938091B102E82FF0E0E25BF44D72
:10BDB0008081843008F083E08083E091B102F0E07C
:10BDC000E25BF44D8081F81609F005C325C33831D4
:10BDD00099F0393128F43C30D9F0303119F512C0DE
:10BDE000303321F0303611F03032E1F4CE010196DB
:10BDF00061E040E02FE111C0CE01019661E044E036
:10BE00002BE10BC0CE01019661E048E027E105C0BF
:10BE1000CE01019661E04AE025E18E010C5F1F4FE3
:10BE20000E94CB1080919F3683FF06C080E18983FA
:10BE300081E08C8380932C018C81882309F46AC073
:10BE4000A091B1024091352B80914C026981A031C3
:10BE500051F590E0242F30E0FC01EE0FFF1FE80FBA
:10BE6000F91F85E29DE08C01209FC001219F900D6C
:10BE7000309F900D1124E80FF91FEB5DFF4E962FB8
:10BE80009295990F990F907C80818F73892B808375
:10BE90006695669567708181887F862B818381E0B6
:10BEA0008093B90337C090E0B0E0242F30E0FC016C
:10BEB000EE0FFF1FE80FF91F84EC90E0AC01A49F88
:10BEC000C001A59F900DB49F900D1124E80FF91F9C
:10BED00085E29DE08C01209FC001219F900D309F45
:10BEE000900D1124E80FF91FE452FC4F962F929504
:10BEF000990F990F907C80818F73892B8083669531
:10BF0000669567708181887F862B8183A55CB44D9F
:10BF100081E08C938091953683FF7EC28091352B92
:10BF200090E025E23DE0829FF001839FF00D929F1B
:10BF3000F00D1124EE53FC4F898185838091B1026D
:10BF4000803199F520E030E045E25DE08091352BCD
:10BF500090E0F901EE0FFF1FE20FF31F849FD00165
:10BF6000859FB00D949FB00D1124EA0FFB1FEB5D70
:10BF7000FF4EAE53BC4F15969C9115979295990F15
:10BF8000990F907C80818F73892B808315969C916B
:10BF90009695969597708181887F892B81832F5FF5
:10BFA0003F4F2034310591F6F0C040E050E014ECF2
:10BFB000E12EF12C05E21DE02091352B30E080913F
:10BFC000B102682F70E0FA01EE0FFF1FE40FF51FBA
:10BFD0006E9DC0016F9D900D7E9D900D1124E80F08
:10BFE000F91F209FD001219FB00D309FB00D11246B
:10BFF000EA0FFB1FE452FC4FAE53BC4F15969C91C9
:10C0000015979295990F990F907C80818F73892B4A
:10C01000808315969C919695969597708181887FDF
:10C02000892B81834F5F5F4F4034510529F6E7C06C
:10C03000CE01029661E040E02FE08E010C5F1F4FC1
:10C040000E94CB1080919F3683FF05C01A8281E049
:10C050008C8380932C018C81882309F458C0A09193
:10C06000B1024091352B80914C026A81A03109F5D3
:10C0700090E0242F30E0FC01EE0FFF1FE80FF91FC6
:10C0800085E29DE08C01209FC001219F900D309F93
:10C09000900D1124E80FF91FEA5DFF4E660F660F41
:10C0A000660F80818770862B808381E08093B9033F
:10C0B0002EC090E0B0E0242F30E0FC01EE0FFF1F17
:10C0C000E80FF91F84EC90E0AC01A49FC001A59F8C
:10C0D000900DB49F900D1124E80FF91F85E29DE0AB
:10C0E0008C01209FC001219F900D309F900D112445
:10C0F000E80FF91FE452FC4F6F70660F660F8081E6
:10C10000837C862B8083A55CB44D81E08C938091E9
:10C11000953683FF81C18091352B90E025E23DE08B
:10C12000829FF001839FF00D929FF00D1124EE533A
:10C13000FC4F8A8184838091B102803151F520E0E7
:10C1400030E045E25DE08091352B90E0D901AA0F07
:10C15000BB1FA20FB31F849FF001859FF00D949F1A
:10C16000F00D1124AE0FBF1FAA5DBF4EEE53FC4F62
:10C170009481990F990F990F8C918770892B8C93CB
:10C180002F5F3F4F20343105F1F681E08093B903F2
:10C1900043C140E050E094ECE92EF12C05E21DE0B3
:10C1A0002091352B30E08091B102682F70E0DA01E8
:10C1B000AA0FBB1FA40FB51F6E9DC0016F9D900DF0
:10C1C0007E9D900D1124A80FB91F209FF001219F83
:10C1D000F00D309FF00D1124AE0FBF1FA452BC4FC5
:10C1E000EE53FC4F94819F70990F990F8C91837C33
:10C1F000892B8C934F5F5F4F4034510589F6655C06
:10C20000744D81E0DB018C9307C10091B1020031D4
:10C2100061F50E94F810482F80919F3683FF06C079
:10C2200081E08093B90380932C014CE080914C0213
:10C2300090E02091352B30E0FC01EE0FFF1FE80F5E
:10C24000F91F85E29DE08C01209FC001219F900D88
:10C25000309F900D1124E80FF91FEB5DFF4E4F71D9
:10C26000440F8081817C842BA1C0E0E4F1E02CE0CC
:10C270008081381721F0215031972223C9F72150AE
:10C2800010E0055C144DCE01039661E040E00E9491
:10C29000CB1080919F3683FF0AC01B82E091B102D0
:10C2A000F0E0E55CF44D81E0808380932C01809187
:10C2B000953683FF4CC08091352B90E025E23DE020
:10C2C000829FF001839FF00D929FF00D1124EE5399
:10C2D000FC4F8B81868340E050E0B4ECEB2EF12CD8
:10C2E00005E21DE02091352B30E08091B102682FEE
:10C2F00070E0FA01EE0FFF1FE40FF51F6E9DC00105
:10C300006F9D900D7E9D900D1124E80FF91F209FC9
:10C31000D001219FB00D309FB00D1124EA0FFB1FFB
:10C32000E352FC4FAE53BC4F16969C91990F990F58
:10C33000990F80818770892B80834F5F5F4F4034D6
:10C34000510581F6655C744D81E0DB018C93809131
:10C350004C0290E02091B10230E04091352B50E04A
:10C36000FC01EE0FFF1FE80FF91F84EC90E08C0139
:10C37000209FC001219F900D309F900D1124E80F48
:10C38000F91F85E29DE09C01429FC001439F900DF3
:10C39000529F900D1124E80FF91FE352FC4F9B812F
:10C3A000990F990F990F80818770892B808334C0F2
:10C3B0008091363690E061E070E00E946F10982F17
:10C3C000873008F096E09093363680913C37981786
:10C3D00019F190933C3781E080932C011DC080912E
:10C3E000EF01813051F0813028F0823049F0833004
:10C3F00099F409C089E396E308C08AE396E305C08F
:10C400008BE396E302C08CE396E369E140E024E627
:10C4100000E010E00E94CB100F900F900F900F9053
:10C420000F90CF91DF911F910F91FF90EF90DF90D0
:10C43000CF90BF90AF909F900895CF92DF92EF92F0
:10C44000FF920F931F937B018C0127E8C22E28E3F4
:10C45000D22E980144275527205BC601622F0E94E7
:10C46000F47F5527412F302F2F2DC601622F0E94B8
:10C470008080C6016E2D0E9480801F910F91FF90D9
:10C48000EF90DF90CF9008953F924F925F926F921E
:10C490007F928F929F92AF92BF92CF92DF92EF9254
:10C4A000FF920F931F932091FA333091FB33220FA9
:10C4B000232F221F330B3195322EE82EFF2400E06C
:10C4C00010E030E040E050E0E1E8AE2EE9E0BE2EC2
:10C4D000C12CD12CA20EB31EC41ED51ED801C7017B
:10C4E00072E0880F991FAA1FBB1F7A95D1F7A80E7B
:10C4F000B91ECA1EDB1E67E0AA0CBB1CCC1CDD1CCF
:10C500006A95D1F729013A0147E0440C551C661C95
:10C51000771C4A95D1F78824C601B5010E941D6297
:10C52000831401F599240AC0E92DF0E0EC50FC4C8D
:10C5300087E898E361850E9480809394292D30E0FC
:10C5400040E050E08091FA339091FB33A0E0B0E0FE
:10C5500084199509A609B709281739074A075B07FF
:10C5600018F30EC09924E92DF0E0EC50FC4C87E85C
:10C5700098E361850E948080939480E8981699F7EB
:10C5800087E898E30E94C3806AE070E080E090E072
:10C590000E94C1858394381408F0BECF39E0EE0CB8
:10C5A000FF1C001F111F3A95D1F783E792ECA4E01E
:10C5B000B0E0E80EF91E0A1F1B1FC801B7010E9458
:10C5C0001D6287E898E36091FA330E948080609151
:10C5D000FB3387E898E30E94808087E898E30E9415
:10C5E000C3806AE070E080E090E00E94C1851F9106
:10C5F0000F91FF90EF90DF90CF90BF90AF909F9002
:10C600008F907F906F905F904F903F900895CF9262
:10C61000DF92EF92FF920F931F9360E070EC84E043
:10C6200090E00E941D6207E818E360914802637081
:10C63000C8010E948080C801609140020E948080F1
:10C64000C801609139020E948080C801609138025F
:10C650000E948080C80160913A020E948080C801D7
:10C6600060913D020E948080C801609136020E9464
:10C670008080B8E4EB2EB2E0FB2EC8016091350259
:10C680000E948080AAEFCA2EAFEFDA2ECE0CDF1CFC
:10C69000C801F60160810E948080F6016181C801B5
:10C6A0000E9480808CEF9FEFE80EF91EC801F70111
:10C6B00060810E948080F7016181C8010E948080B2
:10C6C000C8010E94C3806AE070E080E090E00E94B0
:10C6D000C1851F910F91FF90EF90DF90CF9008954B
:10C6E0009F92AF92BF92CF92DF92EF92FF920F9301
:10C6F0001F938091480282FF48C0837090E0813090
:10C70000910509F18230910559F1892BC9F5809184
:10C7100040029091410290933F0280933E028091AB
:10C72000CA36882319F080E00E942D168091CB36FE
:10C73000882319F081E00E942D160E94702681E066
:10C74000809371011DC00E94702681E08093710169
:10C7500080913A028530A0F084E080933A0210C0C4
:10C7600080E293E0A0E0B0E08093680190936901DB
:10C77000A0936A01B0936B010E9470261092710120
:10C78000809148028B7F80934802809137028823F2
:10C7900051F080918F3683FF06C00E94076310928C
:10C7A00037020E94693980914602909147020897AA
:10C7B00011F01092370280914802837009F4B2C0E0
:10C7C0009090033793E6991508F459C0823009F523
:10C7D000E0906801F090690100916A0110916B018D
:10C7E0006091043770910537809106379091073733
:10C7F0000E94288D5B016C0189E690E0A0E0B0E02A
:10C80000E80EF91E0A1F1B1F60E67AEE80E090E03A
:10C810001AC0813081F5E0906801F09069010091C3
:10C820006A0110916B016091043770910537809116
:10C830000637909107370E94288D5B016C0160E1FB
:10C8400077E280E090E0A80197010E94938ECA01F0
:10C85000B9010E94288D9B01AC01C601B5010E945F
:10C86000278C0E94FC8C609304377093053780936B
:10C870000637909307379394909203372BC06091BB
:10C88000043770910537809106379091073724E679
:10C8900030E040E050E00E94938E30933F022093BE
:10C8A0003E022B3F310518F08AEF90E005C02E3193
:10C8B000310530F48EE190E090933F0280933E0288
:10C8C00010920337109204371092053710920637F2
:10C8D0001092073720913E0230913F02809101373C
:10C8E00090910237281B390B37FF03C030952195F3
:10C8F0003F4F25313105B4F08091CA36882319F0B5
:10C9000080E00E942D168091CB36882319F081E0BB
:10C910000E942D1680913E0290913F029093023723
:10C92000809301371F910F91FF90EF90DF90CF9090
:10C93000BF90AF909F9008952F923F924F925F9239
:10C940007F928F929F92AF92BF92CF92DF92EF929F
:10C95000FF920F931F93DF93CF9300D000D0CDB7FA
:10C96000DEB7062FC82EDD24EE24FF24603109F443
:10C970001EC1262E332444245524C701B60123E1C9
:10C9800030E040E050E00E94418E620D731D841D36
:10C99000951DE7E0660F771F881F991FEA95D1F76D
:10C9A0000E941D627724802E99249A82898284ECC9
:10C9B00090E0889E5001899EB00C989EB00C112486
:10C9C0004CC0872D90E0FC01EE0FFF1FE80FF91F10
:10C9D000EA0DFB1DE20FF31FDF01A452BC4F2C91A7
:10C9E000022F0695017010E0000F111F822F86950F
:10C9F00086958F7090E0880F991F880F991F082BDC
:10CA0000192B822F817090E0082B192B22952695E7
:10CA10002695237011968C918770880F880F822B32
:10CA200090E0A6E0880F991FAA95E1F7082B192B33
:10CA3000E352FC4F8081887F8C831B822B813C8159
:10CA4000022B132B87E898E3602F0E94808087E8F1
:10CA500098E3612F0E94808073948091352B90E041
:10CA6000F5E28F2EFDE09F2E889D9001899D300D6F
:10CA7000989D300D1124F501E20FF31FE456FB4F92
:10CA80008081871508F09DCF87E898E30E94C380D6
:10CA90006AE070E080E090E00E94C185C701B601C5
:10CAA00020E839E040E050E00E94418E7B018C019B
:10CAB00080E098E0A0E0B0E0E80EF91E0A1F1B1F1E
:10CAC000C201B10126E030E040E050E00E94418E1A
:10CAD000E60EF71E081F191FC801B7010E941D624C
:10CAE00087E898E360E00E9480808091352B90E099
:10CAF000889DF001899DF00D989DF00D1124EA0D9F
:10CB0000FB1DE456FB4F87E898E360810E9480801C
:10CB10008091352B90E0889DF001899DF00D989DC6
:10CB2000F00D1124EA0DFB1DE356FB4F87E898E357
:10CB300060810E9480808091352B90E0889DF0017B
:10CB4000899DF00D989DF00D1124EA0DFB1DE15615
:10CB5000FB4F87E898E360810E9480808091352BAD
:10CB600090E0889DF001899DF00D989DF00D1124B5
:10CB7000EA0DFB1DE256FB4F87E898E360810E94B7
:10CB800080808091352B90E0889DF001899DF00D8B
:10CB9000989DF00D1124EE53FC4FA981BA81EA0F44
:10CBA000FB1F87E898E367810E948080F5C0C7017A
:10CBB000B60120E839E040E050E00E94418E6B0170
:10CBC0007C016058774F8F4F9F4F0E941D6280916C
:10CBD000352B90E005E21DE0809FF001819FF00D74
:10CBE000909FF00D1124EF5DFF4E87E898E3608180
:10CBF0000E9480808091352B90E0809FF001819F82
:10CC0000F00D909FF00D1124E05EFF4E87E898E351
:10CC100060810E9480808091352B90E0809FF001A0
:10CC2000819FF00D909FF00D1124EE5DFF4E87E87F
:10CC300098E360810E9480808091352B90E0809FF6
:10CC4000F001819FF00D909FF00D1124ED5DFF4EDE
:10CC500087E898E360810E9480808091352B90E086
:10CC6000809FF001819FF00D909FF00D1124E15EF7
:10CC7000FF4E87E898E360810E94808000E0E5E253
:10CC8000AE2EEDE0BE2E11C0802F90E0FC01EE0F25
:10CC9000FF1FE80FF91FE20FF31FE95DFF4E6081F0
:10CCA00087E898E30E9480800F5F8091352B90E0A9
:10CCB0008A9D90018B9D300D9A9D300D1124F901B4
:10CCC000EF5DFF4E80818017F8F687E898E30E94B9
:10CCD000C3806AE070E080E090E00E94C185C701F7
:10CCE000B6016050774F8F4F9F4F0E941D62FF2407
:10CCF00065E2C62E6DE0D62E3EC08F2D90E0FC0181
:10CD0000EE0FFF1FE80FF91FE20FF31FDF01AB5D0E
:10CD1000BF4E2C91022F06950F7110E0000F111FCE
:10CD2000422F429546954695437011968C91877097
:10CD3000880F880F842B90E036E0880F991F3A9572
:10CD4000E1F7082B192B217030E0022B132BEA5D41
:10CD5000FF4E808198EF992E98228824082919295E
:10CD600087E898E3602F0E94808087E898E3612F2E
:10CD70000E948080F3948091352B90E08C9D9001EF
:10CD80008D9D300D9C9D300D1124F901EF5DFF4EFE
:10CD900080818F1508F0B1CF87E898E30E94C380A7
:10CDA0006AE070E080E090E00E94C1850F900F90F3
:10CDB0000F900F90CF91DF911F910F91FF90EF9007
:10CDC000DF90CF90BF90AF909F908F907F905F90BB
:10CDD0004F903F902F9008952F923F924F925F92E5
:10CDE0007F928F929F92AF92BF92CF92DF92EF92FB
:10CDF000FF920F931F93DF93CF9300D000D0CDB756
:10CE0000DEB77724C8C0003109F43FC0C701B601BE
:10CE10000E941D6210E087E898E362E00E94808033
:10CE200087E898E364E00E9480801F5F103499F7E0
:10CE300087E898E30E94C3806AE070E080E090E0B9
:10CE40000E94C185C501B4010E941D6287E898E374
:10CE500061E00E94808087E898E36FE00E94808014
:10CE600087E898E368E10E94808087E898E361E0C2
:10CE70000E94808087E898E360E00E94808087E8D5
:10CE800098E360E00E94808044C069817A818B8150
:10CE90009C810E941D6287E898E36FE00E94808079
:10CEA00087E898E368E10E94808087E898E361E082
:10CEB0000E94808087E898E360E00E94808087E895
:10CEC00098E360E00E94808010E087E898E360E3E8
:10CED0000E9480801F5F1034C1F787E898E30E94AA
:10CEE000C3806AE070E080E090E00E94C185C201EA
:10CEF000B1010E941D6210E087E898E368E10E949A
:10CF0000808087E898E364E00E9480801F5F10348F
:10CF100099F787E898E30E94C3806AE070E080E0B8
:10CF200090E00E94C1850F5F86E090E0A0E0B0E055
:10CF3000880E991EAA1EBB1E80E890E0A0E0B0E01B
:10CF4000C80ED91EEA1EFB1E013109F05CCF272D49
:10CF500026952695269581E090E0A0E0B0E004C0FB
:10CF6000880F991FAA1FBB1F2A95D2F79C01AD01FC
:10CF700080913E3790913F37822B932B90933F3790
:10CF800080933E3760E070E040E00E94960E73941C
:10CF900090E8791651F1672D70E080E090E020E88C
:10CFA00039E040E050E00E94418E6B017C01812C11
:10CFB000A8E09A2EA12CB12C860E971EA81EB91E91
:10CFC000DC01CB018058974FAF4FBF4F89839A83C5
:10CFD000AB83BC83212CF9E03F2E412C512C2C0C2F
:10CFE0003D1C4E1C5F1C00E00ECF60E070EC84E046
:10CFF00090E00E941D6287E898E360E00E948080D4
:10D0000087E898E368E70E94808087E898E361E01A
:10D010000E94808087E898E361E00E94808087E832
:10D0200098E361E00E94808087E898E30E94C380D3
:10D030006AE070E080E090E00E94C18587E898E3B4
:10D0400067E570E00E94FE7F87E898E36FEF0E943B
:10D05000808087E898E36DEF0E94808087E898E3FE
:10D0600060E00E94808087E898E361E00E94808011
:10D0700087E898E363E00E94808087E898E30E9455
:10D08000C3806AE070E080E090E00E94C1850F906C
:10D090000F900F900F90CF91DF911F910F91FF9004
:10D0A000EF90DF90CF90BF90AF909F908F907F9048
:10D0B0005F904F903F902F9008953F924F925F92D4
:10D0C0006F927F928F929F92AF92BF92CF92DF9298
:10D0D000EF92FF920F931F93A82EBB24CC24DD2444
:10D0E00086017501F9E0EE0CFF1C001F111FFA9577
:10D0F000D1F783E792ECA4E0B0E0E80EF91E0A1F36
:10D100001B1FC801B7010E941D6287E898E30E94B7
:10D11000C38078010027112790E5E90E87E898E39E
:10D120006E2D42E00E94D88087E898E30E9411802B
:10D130008C0187E898E30E941180382F20E010705E
:10D14000022B132B1093FB330093FA33045F11402F
:10D1500020F01092FB331092FA338091FA339091C1
:10D16000FB33880F892F881F990B9195582E282FF4
:10D1700030E040E050E061E8662E69E0762E812CD8
:10D18000912C620E731E841E951E92E0AA0CBB1C8D
:10D19000CC1CDD1C9A95D1F76A0C7B1C8C1C9D1C49
:10D1A00087E0660C771C881C991C8A95D1F7C4010E
:10D1B000AA27BB2710E5412E480E59016A01B7E0A6
:10D1C000AA0CBB1CCC1CDD1CBA95D1F73A2CFF2451
:10D1D000C401B3010E941D6287E898E30E94C380E6
:10D1E000F51461F54091FA33431987E898E3642D0B
:10D1F0000E94D880EE240EC00E2D10E087E898E340
:10D200000E941180F801EC50FC4C8187813808F0B5
:10D210001186E3942E2D30E040E050E08091FA3307
:10D220009091FB33A0E0B0E08A199B09AC09BD09DD
:10D23000281739074A075B07F8F218C087E898E310
:10D24000642D40E80E94D880EE240E2D10E087E87F
:10D2500098E30E941180F801EC50FC4C81878138E2
:10D2600008F01186E394B0E8EB1679F7F3945F14B5
:10D2700008F0AECF1F910F91FF90EF90DF90CF900D
:10D28000BF90AF909F908F907F906F905F904F90E6
:10D290003F9008950F931F9360E070EC84E090E05E
:10D2A0000E941D6287E898E30E94C38087E898E3A4
:10D2B00064E540E80E94D88087E898E30E941180E6
:10D2C000982F9370933009F492E093708091480204
:10D2D0008C7F892B8093480287E898E30E94118015
:10D2E00090E08E31910518F48EE190E005C08B3FFF
:10D2F000910510F08AEF90E09093410280934002F4
:10D3000087E898E30E941180882311F481E003C02C
:10D31000813108F080E18093390287E898E30E9428
:10D320001180882311F481E003C0813108F080E18D
:10D330008093380287E898E30E941180873008F0D4
:10D3400086E080933A0287E898E30E941180823059
:10D3500010F482E003C08B3008F08AE080933D0235
:10D3600087E898E30E941180811181E08093360262
:10D3700087E898E30E941180811181E08093350253
:10D3800087E898E30E9411808C0187E898E30E9467
:10D390001180382F20E01070022B132B10934302C2
:10D3A000009342020050104130F08FEF9FE09093C5
:10D3B00043028093420287E898E30E9411808C0127
:10D3C00087E898E30E941180382F20E01070022B2C
:10D3D000132B10934502009344020050104130F08B
:10D3E0008FEF9FE090934502809344021F910F912D
:10D3F00008950E944A6910924E02109233011092D1
:10D4000032011092F10183E090E090934702809303
:10D41000460280E00E946C860E94A8898091680084
:10D42000816080936800D89A80916B0083608093BC
:10D430006B001092CD008FE18093CC008091CA00E8
:10D4400086608093CA008091C90088698093C90072
:10D450001092F202809140029091410290933F021B
:10D4600080933E0280914802837090E08130910564
:10D4700029F08230910541F0892B51F40E947026E9
:10D4800081E08093710104C00E94702610927101A6
:10D49000809148028B7F80934802809149028823C3
:10D4A00011F02C9A01C02C988091352B90E025E248
:10D4B0003DE0829FF001839FF00D929FF00D1124BB
:10D4C000DF01A95DBF4E4C91942F9F70E15EFF4E2E
:10D4D000E0818CE0E89FF0011124E90FF11DE35594
:10D4E000FC4FE491E150F0E0EE0FFF1FE75EFB4FD1
:10D4F00085919491469546954695342F3E7020E04F
:10D50000820F931F0E94480F08952F923F924F92CF
:10D510005F926F927F928F929F92AF92BF92CF92C3
:10D52000DF92EF92FF920F931F93DF93CF93CDB7CC
:10D53000DEB76E970FB6F894DEBF0FBECDBF062FD5
:10D5400010921D3690E0A0E0B0E0BC01CD0120E8D3
:10D5500039E040E050E00E94418E5B016C01612C9B
:10D5600078E0772E812C912C6A0C7B1C8C1C9D1CE6
:10D57000A60195012058374F4F4F5F4F29873A87B3
:10D580004B875C87CA01AA27BB27382F305B3E83B5
:10D59000D601C5018050974FAF4FBF4F8A839B8301
:10D5A000AC83BD83CD01AA27BB27E82FE05BE983CD
:10D5B00010E085E29DE09C01029FC001039F900D59
:10D5C000129F900D1124AC0144565B4F5E8F4D8F1E
:10D5D000DC01A753BC4FB887AF83222433242C012E
:10D5E0008E539C4FFC01E15AF34FFC8BEB8B9C015B
:10D5F000225A334F3E8B2D8BAC01405A534F588FDC
:10D600004F8BDC01AF59B34FBA8FA98FFC01E35A9E
:10D61000F34FFC8FEB8FF0E12F16310409F4D5C0E6
:10D62000C401B3010E941D6287E898E30E94C38091
:10D63000940144275527205B87E898E3622F46E052
:10D640000E94D88087E898E30E94118087E898E3D9
:10D650000E941180AD8DBE8D8C9387E898E30E9467
:10D660001180ED8DFE8D818387E898E30E94118003
:10D67000AD8DBE8D13968C9387E898E30E94118040
:10D68000ED8DFE8D828387E898E30E941180AF8143
:10D69000B8858C93ED8DFE8DE080FF240894E11C0D
:10D6A000F11CEE0CFF1C0027F7FC0095102FC601A3
:10D6B000B5010E941D6287E898E30E94C38096012D
:10D6C00044275527205B87E898E3622F4E2D0E9460
:10D6D000D880EE2444EC50E0249E9001259E300D2D
:10D6E000349E300D11243A8B298B68C087E898E36B
:10D6F0000E9411808C0187E898E30E9411808E8738
:10D700001D86A80150708D859E85482B592B6E2D46
:10D7100070E0FB01EE0FFF1FE60FF71FA989BA8922
:10D72000EA0FFB1FE40DF51DE452FC4F242F21707E
:10D7300030813C7FCA018270907096958795817088
:10D74000880F322B382BCA018C7390709695879571
:10D75000969587958F70282F220F220F337C322BBE
:10D760003083882311F4337C3083FB01EE0FFF1FDD
:10D77000E60FF71F29893A89E20FF31FE40DF51D23
:10D78000DF01A452BC4FCA01807C977076E0969569
:10D7900087957A95E1F7382F3295330F330F307C28
:10D7A0002C912F73232B2C9386958695E352FC4F57
:10D7B000252F287F8770822B8083E394AD8DBE8DCB
:10D7C0008C918E1508F092CFD0C069857A858B85B3
:10D7D0009C850E941D6287E898E30E94C38087E8C9
:10D7E00098E36E8140E80E94D88087E898E30E9421
:10D7F0001180EB89FC89808387E898E30E9411807F
:10D80000AD89BE898C9387E898E30E941180EF89E7
:10D81000F88D808387E898E30E941180A98DBA8DE6
:10D820008C9387E898E30E941180EB8DFC8D8083B8
:10D83000893008F088E0AB8DBC8D8C9300E022C06D
:10D8400087E898E30E941180202F30E0F901EE0F65
:10D85000FF1FE20FF31FE40DF51DE95DFF4E282FBA
:10D8600030E02077307054E0359527955A95E1F7F0
:10D8700027702295207F982F90788F70282B292B46
:10D8800020830F5FEB89FC89E080E016C8F66A818F
:10D890007B818C819D810E941D6287E898E30E94B4
:10D8A000C3802E2D30E02F5F3F4F220F331F4427C0
:10D8B00037FD4095542F87E898E36981422F0E94F5
:10D8C000D880EE244CC087E898E30E9411808C0138
:10D8D00087E898E30E941180888B1F8610702F853F
:10D8E0003889022B132B8E2D90E0AC01440F551F6D
:10D8F000480F591F440D551DFA01EB5DFF4E702F67
:10D900007170C8018E739070969587958F71880F8E
:10D910009801207C3770B6E036952795BA95E1F7E7
:10D92000622F6295660F660F607C872B862B808343
:10D9300026952695812F869586958695FA01EA5D2E
:10D94000FF4E982F990F990F990F2770292B20833D
:10D95000815E8F71803110F027702083E394AB8952
:10D96000BC898C918E1508F0AECF0894211C311C17
:10D97000ED8DFE8DEC53FF4FFE8FED8F26E030E0F6
:10D9800040E050E0620E731E841E951E4F81588544
:10D990004F5F5F4F58874F8380E890E0A0E0B0E092
:10D9A000A80EB91ECA1EDB1E91E12916310409F02A
:10D9B00032CE81E080931D366E960FB6F894DEBFAE
:10D9C0000FBECDBFCF91DF911F910F91FF90EF90D0
:10D9D000DF90CF90BF90AF909F908F907F906F908F
:10D9E0005F904F903F902F90089580ED84B982EF23
:10D9F0008AB98CEF81B989E061E00E948E8612B805
:10DA00005F980E94C17D8FEF0E949F7D87E898E319
:10DA10000E94DC800895FF920F931F93CF93DF93B2
:10DA200000E0C5E2DDE06CE0F62E7EC16CE070E067
:10DA300080E090E00E946889162F80913936823309
:10DA400081F1833320F4893109F097C007C08B340A
:10DA500009F44AC0843609F090C069C067E070E0FC
:10DA600080E090E00E946889613071058105910530
:10DA700009F083C08091352B90E08C9F90018D9FA1
:10DA8000300D9C9F300D1124F901E15EFF4EE081C5
:10DA9000EF9DF0011124E10FF11DE355FC4F44917E
:10DAA0005CC064E070E080E090E00E9468896130D2
:10DAB00071058105910509F060C08091352B90E0DA
:10DAC0008C9F90018D9F300D9C9F300D1124F9018A
:10DAD000E15EFF4EE081EF9DF0011124E10FF11DA9
:10DAE000E355FC4F449139C063E070E080E090E082
:10DAF0000E946889613071058105910509F03DC07A
:10DB00008091352B90E08C9F90018D9F300D9C9FD4
:10DB1000300D1124F901E15EFF4EE081EF9DF0012F
:10DB20001124E10FF11DE355FC4F449116C0809183
:10DB3000352B90E08C9F90018D9F300D9C9F300D78
:10DB40001124F901E15EFF4EE081EF9DF001112407
:10DB5000E10FF11DE355FC4F4491802F90E0FC0153
:10DB6000EE0FFF1FE80FF91FE20FF31FE95DFF4EF5
:10DB70004F708081807F842B808368E070E080E03C
:10DB800090E00E946889162F80913A36823379F0AE
:10DB9000833318F48931C1F505C08B3469F08436BC
:10DBA00099F515C067E070E080E090E009C064E09E
:10DBB00070E080E090E004C063E070E080E090E01E
:10DBC0000E9468896130710581059105E9F4202F73
:10DBD00030E08091352B90E0F901EE0FFF1FE20F4E
:10DBE000F31F9C012C9FC0012D9F900D3C9F900D19
:10DBF0001124E80FF91FE95DFF4E17701295107F91
:10DC000080818F78812B808362E070E080E090E0FB
:10DC10000E946889162F80913B36823379F08333D6
:10DC200018F48931B1F505C08B3469F0843689F573
:10DC300015C067E070E080E090E009C064E070E04B
:10DC400080E090E004C063E070E080E090E00E943B
:10DC500068896130710581059105D9F4202F30E084
:10DC60008091352B90E0F901EE0FFF1FE20FF31FBB
:10DC70009C012C9FC0012D9F900D3C9F900D112465
:10DC8000E80FF91FEB5DFF4E117080818E7F812BB5
:10DC900080836AE070E080E090E028E130E040E0DE
:10DCA00050E00E948A89162F80913C36823379F0A9
:10DCB000833318F48931B9F505C08B3469F08436A3
:10DCC00091F515C067E070E080E090E009C064E085
:10DCD00070E080E090E004C063E070E080E090E0FD
:10DCE0000E9468896130710581059105E1F4202F5A
:10DCF00030E08091352B90E0F901EE0FFF1FE20F2D
:10DD0000F31F9C012C9FC0012D9F900D3C9F900DF7
:10DD10001124E80FF91FEB5DFF4E1F71110F808179
:10DD2000817C812B80830F5F8091352B90E08C9FCD
:10DD3000F0018D9FF00D9C9FF00D1124EF5DFF4EC3
:10DD40008081801708F072CEDF91CF911F910F91E3
:10DD5000FF9008958F929F92AF92BF92CF92DF92E1
:10DD6000EF92FF920F931F93CF93DF9381E060E0D8
:10DD700070E00E9485089093B7368093B636809104
:10DD8000AB02882379F08091460290914702089770
:10DD900049F483E090E0909347028093460281E04B
:10DDA00080932C0180914602909147028430910526
:10DDB00031F00C9721F01092B0021092F43580915E
:10DDC0002D36882379F00E94B38560932F367093A7
:10DDD0003036809331369093323681E080932E3600
:10DDE00010922D3680912E368823F1F08091AB026F
:10DDF0008823D1F00E94B38520912F3630913036A0
:10DE00004091313650913236621B730B840B950B67
:10DE1000615971408040904038F081E080932C3609
:10DE20001092710110922E3680919D3682FF21C092
:10DE300080919F3683FF1DC08091460290914702DA
:10DE40000597B9F08091B3026091352B0E94856AE5
:10DE50000E9490258091B3020E94AD2BEBE3FBE280
:10DE600011923BE2EB34F307D9F71092B903109209
:10DE7000E7368091AD3683FF0CC080918B3682FDF2
:10DE800008C080917101882321F08091480283703D
:10DE900029F080912B36882309F44AC081E08093D1
:10DEA000AB02109240011092353610922B36109230
:10DEB000043610924E021092B4031092B3031092E3
:10DEC000AA021092E8362C982C9A109249021092CD
:10DED000B036109233011092320180E090E021E0E0
:10DEE000FC01E05AFD4F1082FC01E752FD4F108209
:10DEF000FC01EA54FD4F2083FC01EE57FD4F1082D8
:10DF0000FC01E45FF94C2083FC01ED56FD4F2083BA
:10DF100001968131910521F78091CA36882311F04D
:10DF20001092C6368091CB36882311F01092C736F6
:10DF300080913536882341F08091AB02882321F00F
:10DF4000109235361092B0368091AF3683FF0CC0F8
:10DF500080918B3682FD08C080917101882321F069
:10DF600080914802837049F080910536882329F416
:10DF700080912C36882309F454C05F981092EA02ED
:10DF8000109249021092B0021092B6031092B5039B
:10DF90008091312B882359F091E09093332B80911D
:10DFA000322B8093B5028093B3029093362B8091ED
:10DFB0000536882311F01092B03680912C368823D4
:10DFC00011F01092B03610922C3610920536109146
:10DFD000B0361F5F1093B036113019F0123009F5CA
:10DFE00017C0109340011092AB020E94A3290E9417
:10DFF000A3290E94A3290E94A32980913502882386
:10E0000081F080E090E80E94DE0E10934A0209C081
:10E010001092400181E08093AB021092B0361092D2
:10E020004E0280918B3682FF36C08091993683FFF5
:10E0300004C08091B1020E94712080919B3683FFC1
:10E0400004C08091B1020E9470228091AB3683FFA0
:10E0500009C08CE090E0909347028093460281E0F3
:10E0600080932C018091953683FFFBC080914602FE
:10E0700090914702019739F081E090E09093470238
:10E080008093460204C0109247021092460281E03B
:10E0900080932C01E6C08091460290914702823025
:10E0A0009105A9F48091993683FF02C00E94B61EA3
:10E0B00080919B3683FF03C00E94001F3FC082FFF8
:10E0C00003C00E9441393AC084FF38C034C0833055
:10E0D0009105B9F48091993683FF08C08091B1020F
:10E0E0000E94FB1B8091B10280934C2B80919B3648
:10E0F00083FF24C08091B10260914C2B0E94F91CD7
:10E100001DC00997D9F48091993683FF08C080918A
:10E110004C0280934D028091B10280934C2B8091F0
:10E120009B3683FF0BC080914C2B60914D02409138
:10E130004C020E94FC1A81E080932C018091A13650
:10E1400083FF12C08091460290914702039719F015
:10E1500083E090E002C082E090E0909347028093D9
:10E16000460281E080932C018091AB3683FF1CC076
:10E170008091460290914702049719F084E090E064
:10E1800002C083E090E09093470280934602809122
:10E19000B102803121F481E08093F43502C0109205
:10E1A000F43581E080932C012091933623FF17C032
:10E1B00080914602909147028530910581F09093BD
:10E1C000AD028093AC0285E090E09093470280938B
:10E1D000460220642093933681E080932C012091A5
:10E1E000933624FF23C026FF0AC0809146029091F7
:10E1F00047020597D9F42F7B2093933617C080915F
:10E20000460290914702059789F48091F2339091EC
:10E21000F333892B59F48091AC029091AD02909325
:10E2200047028093460281E080932C018091460250
:10E2300090914702059721F01092F3331092F23338
:10E240008091460290914702089711F01092F101D7
:10E2500080914602909147020797029710F0109222
:10E26000F1018091AD3683FF1DC080918B3682FF16
:10E2700019C08091AB028823A9F488E090E09093C4
:10E280004702809346028091F1018F5F8093F101F4
:10E29000833018F081E08093F1011092EF0181E06A
:10E2A00080932C019091A5369695969596959170B0
:10E2B00041F080918B3682FD04C081E08093F501AE
:10E2C00007C08091A53684FF06C01092F50181E059
:10E2D00080932C0110C0992371F080918B3682FFBE
:10E2E0000AC08091B102803131F48DE090E09093CA
:10E2F0004702809346028091A93683FF04C081E0E3
:10E300008093F40105C084FF05C01092F40181E000
:10E3100080932C012091460230914702C901039756
:10E32000029768F02730310551F02930310539F076
:10E330002630310521F02C30310509F0E5C58091FA
:10E34000B6369091B736892B11F41092B53680917C
:10E350008D3682FF3EC08091973683FF0DC083E0EB
:10E3600090E090934702809346020E94B30B809303
:10E37000B10281E080932C0180918F3683FF0CC025
:10E3800087E090E0909347028093460280E180937B
:10E39000B10281E080932C0180919F3683FF0CC0F5
:10E3A00083E090E0909347028093460280E180935F
:10E3B000B10281E080932C0180919D3683FF09C0DA
:10E3C00086E090E0909347028093460281E080933C
:10E3D0002C0180919D3683FF1CC08091B102803159
:10E3E000C1F480918D3682FD14C087E090E0909357
:10E3F000470280934602809101368093BB0391E0EF
:10E4000090932C018F5F80930136823010F0109230
:10E4100001368091460290914702079711F01092C1
:10E42000013680919F3683FF11C080914602909102
:10E430004702079759F41092013683E090E09093D9
:10E4400047028093460281E080932C018091A3369D
:10E4500082FF91C08091AB02882309F48CC0209187
:10E46000B1024091352B203109F043C080915F0209
:10E4700090E0242F30E0FC01EE0FFF1FE80FF91FA2
:10E4800085E29DE0A901489F9001499F300D589F6A
:10E49000300D1124E20FF31FEB5DFF4E80818E7F64
:10E4A000808380915F0290E0FC01EE0FFF1FE80F78
:10E4B000F91FE20FF31FDF01AB5DBF4E8C918E7F22
:10E4C0008C93EA5DFF4E8081877080839C911196CA
:10E4D0008C911197887F846011968C93119791701D
:10E4E00098619C9381E08093B9035F981092EA024F
:10E4F00042C030E0D901A15BBD4F8C9190E050E06B
:10E50000FC01EE0FFF1FE80FF91F84EC90E0289F3D
:10E51000B001299F700D389F700D1124E60FF71F71
:10E5200085E29DE0EA01C89FA001C99F500DD89FD8
:10E53000500D1124E40FF51FE452FC4F80818E7FB3
:10E5400080838C9190E0FC01EE0FFF1FE80FF91F14
:10E55000E60FF71FE40FF51FDF01A452BC4F8C91AB
:10E5600083708C93E352FC4F84E08083255C344DB0
:10E5700081E0F901808380918B3682FF0DC080910C
:10E58000A33683FF09C08091B102803119F00E9447
:10E59000171E02C00E94621E8091913682FF0BC13D
:10E5A0008091973683FF07C180918B3682FF6EC0C2
:10E5B0008091352B90E025E23DE0829F8001839F92
:10E5C000100D929F100D11240E531C4FD801FC907A
:10E5D0000E94B30BE091B102F0E0E25BF44D908158
:10E5E0009295907F980FE801988320E030E064ECEA
:10E5F00070E045E25DE011E08091352B90E0269FD0
:10E60000F001279FF00D369FF00D1124DC01A49F2F
:10E61000C001A59F900DB49F900D1124E80FF91F24
:10E62000E456FB4FDC01AE53BC4F8C918083F90163
:10E63000E55CF44D10832F5F3F4F20313105E1F64B
:10E64000FD01E15AF34F8C9180831093B9038091BF
:10E650003602813009F0ACC010E0C5E2DDE0809107
:10E66000352B90E08C9FF0018D9FF00D9C9FF00D5D
:10E670001124EE53FC4F4081F41620F4812F6F2DAE
:10E680000E945A1F1F5F113151F792C08091B10251
:10E690004091352B8031C1F5842F90E0C5E2DDE05B
:10E6A0008C9F80018D9F100D9C9F100D11240F5D7C
:10E6B0001F4EF801F0800E94B30B2091B102E22FAF
:10E6C000F0E0E25BF44D90819295907F980FD80135
:10E6D0009C9381E08093B90380913602813009F0E8
:10E6E00065C08091352B90E08C9FF0018D9FF00DDF
:10E6F0009C9FF00D1124EF5DFF4E4081F41608F051
:10E7000055C0822F6F2D50C0242F30E090E004ECD4
:10E71000E02EF12C8E9DF0018F9DF00D9E9DF00D51
:10E720001124C5E2DDE02C9F80012D9F100D3C9F40
:10E73000100D1124E00FF11FE456FB4FD0800E9412
:10E74000B30B5091B102A52FB0E0AE9D9001AF9DEB
:10E75000300DBE9D300D1124020F131F04561B4FA8
:10E76000FD01E25BF44D90819295907F980FF80146
:10E770009083A55CB44D81E08C938091360281300A
:10E78000A9F48091352B90E08C9FF0018D9FF00DC6
:10E790009C9FF00D1124E20FF31FE456FB4F4081C4
:10E7A000D41620F4852F6D2D0E945A1F0E94272514
:10E7B00081E080932C0180918B3682FF5DC0809137
:10E7C0008D3683FF59C04091B1024E3009F454C0D8
:10E7D0004F3009F451C0403109F44EC08091352BBF
:10E7E00090E025E23DE0829FF001839FF00D929F33
:10E7F000F00D1124EE53FC4FE40FF11D87818823A7
:10E8000081F1178240E050E0A4ECB0E065E27DE0E9
:10E810008091B10290E02091352B30E0FA01EE0FAB
:10E82000FF1FE40FF51FEC01CA9FC001CB9F900DA5
:10E83000DA9F900D1124E80FF91F269FC001279F32
:10E84000900D369F900D1124E80FF91FE452FC4FF4
:10E850008081826080834F5F5F4F40345105C1F6F5
:10E8600002C081E0878381E080932C01E091B102B6
:10E87000F0E0E55CF44D8083809146029091470280
:10E880008330910539F08730910521F08930910569
:10E8900009F061C18091973684FF04C01092B536AB
:10E8A00010920A378091913682FD2EC380918D3669
:10E8B00082FD2AC380918B3682FD15C0809146026D
:10E8C00090914702039779F48091B1022091B63676
:10E8D0003091B736803121F4C9010E94420A03C049
:10E8E000C9010E94EF088091973683FFA2C0209152
:10E8F0004602309147022930310521F02730310599
:10E9000009F097C080918B3682FF83C02930310592
:10E9100009F07FC0A0E0B0E005E21DE0C4ECD0E06B
:10E920008091B6369091B7360A2E02C0969587959B
:10E930000A94E2F780FF67C02091B1024091352B25
:10E940002031A1F4842F90E0FD01EE0FFF1FEA0FAC
:10E95000FB1F9C01209FC001219F900D309F900DB7
:10E960001124E80FF91FEB5DFF4E45C0842F90E0A6
:10E97000622F70E0809FA001819F500D909F500DED
:10E980001124FA01EE53FC4FE60FF71F87819D011A
:10E99000220F331F8823F9F0F901EA0FFB1F6C9F48
:10E9A000C0016D9F900D7C9F900D1124E80FF91F01
:10E9B000E40FF51FE452FC4F8081982F969580FD5F
:10E9C00005C090FF20C08D7F81601CC0826090FFD9
:10E9D00019C08E7F17C0F901EA0FFB1F6C9FC001A1
:10E9E0006D9F900D7C9F900D1124E80FF91FE40F8F
:10E9F000F51FE452FC4F90E0808180FF91E0808120
:10EA00008E7F892B80831196A031B10509F088CFC4
:10EA10000DC00E94B30BE091B102F0E0E25BF44D57
:10EA200090819295907F980F90934C0281E0809313
:10EA30002C0180914602909147028930910541F066
:10EA4000079709F062C08091B102803109F05DC082
:10EA50000E94D10B082F0E94B30B10E0081B110974
:10EA60000130110509F0ACC680910A37882309F0FE
:10EA7000A7C62091352B30E080914C0290E0FC013C
:10EA8000EE0FFF1FE80FF91F85E29DE0AC01249F08
:10EA9000C001259F900D349F900D1124E80FF91FA0
:10EAA00022C00E94D10B682F8091352B90E025E287
:10EAB0003DE0829FA001839F500D929F500D112435
:10EAC000FA01EF5DFF4E80816817F9F480910A37F3
:10EAD0008823D9F4862F90E0FC01EE0FFF1FE80F8A
:10EAE000F91FE40FF51FE95DFF4E90E0808187FF7D
:10EAF00091E097959927979580818F77892B8083CF
:10EB000081E080930A3780932C0180918B3682FFBD
:10EB1000FBC18091973683FFF7C1809146029091A7
:10EB20004702099709F4F0C189E090E09093470209
:10EB3000809346020E94B30BE091B102F0E0E25BE9
:10EB4000F44D90819295907F980F90934C0281E0C4
:10EB500080932C01D9C18430910509F045C1809181
:10EB6000B102803139F48091F435882319F481E0C1
:10EB70008093F4358091AB02882361F080918F36C9
:10EB800083FF08C090E08091B002882309F491E0EF
:10EB90009093B0028091A33682FF53C0A091B1023E
:10EBA0004091352BA031F9F480915F0290E0242F41
:10EBB00030E0FC01EE0FFF1FE80FF91F85E29DE03A
:10EBC000DC012A9FC0012B9F900D3A9F900D1124CC
:10EBD000E80FF91FEB5DFF4E80818E7F808381E01F
:10EBE0008093B9032EC0B0E0FD01E15BFD4F808151
:10EBF00090E0242F30E0FC01EE0FFF1FE80FF91F1B
:10EC000084EC90E0EC01AC9FC001AD9F900DBC9FE7
:10EC1000900D1124E80FF91F85E29DE0AC01249FBF
:10EC2000C001259F900D349F900D1124E80FF91F0E
:10EC3000E452FC4F80818E7F8083A55CB44D81E0DF
:10EC40008C938091913682FD0AC080918D3682FD31
:10EC500006C08091F435882369F00E94651340E076
:10EC600050E0A4EC8A2E912CF5E2AF2EFDE0BF2EF1
:10EC700001E064C0C0E0D0E0E1E0EE2EF12C809134
:10EC8000B6369091B7360C2E02C0969587950A94A9
:10EC9000E2F7282F2170FE01EE0FFF1FE559F94C16
:10ECA00090819E7F922B9083892F86958170281763
:10ECB00099F192FD31C0213079F587010C2E02C007
:10ECC000000F111F0A94E2F7C8010E940E2AC80122
:10ECD0000E94DE0E80ED97E00E941A8680E090E0B0
:10ECE0000E94DE0E8091AB028823B1F08091B002C9
:10ECF000813091F4FE01EF58FD4F8081FE0166E006
:10ED0000EE0FFF1F6A95E1F7E80FF11DEE0FFF1FF1
:10ED1000E059F44DF182E082FE01EE0FFF1FE5594C
:10ED2000F94C8081982F9170990F8D7F892B80836A
:10ED30002196C031D10509F0A2CF91CFFA01E05A56
:10ED4000FD4F8081882309F048C010E0489DE00114
:10ED5000499DD00D589DD00D11246A0136E0CC0C90
:10ED6000DD1C3A95E1F72BE3E22E2BE2F22EE40EC6
:10ED7000F51E21C0212F30E0D601A20FB31FAA0F2C
:10ED8000BB1FA059B44D8D919C911197892B91F087
:10ED9000F901EE0FFF1FE20FF31FEC0FFD1FE60F4F
:10EDA000F71FE452FC4F808183608083F70100836A
:10EDB0001D921C921F5F8091352B90E08A9DB001BF
:10EDC0008B9D700D9A9D700D1124FE01E60FF71FAB
:10EDD000E456FB4F8081181768F24F5F5F4F403158
:10EDE000510509F0ABCF90C00C9709F08DC0809110
:10EDF000B6369091B73690933836809337368091F7
:10EE0000AB02882309F480C080918F3683FF08C04D
:10EE100090E08091B002882309F491E09093B002D1
:10EE20008091B002882309F46FC040E050E0E4EC28
:10EE3000EE2EF12C05E21DE0CC24C39477E0D72E12
:10EE40008091373690913836042E02C0969587957A
:10EE50000A94E2F780FF52C0DA01A15BBD4F8C91AA
:10EE600090E02091352B30E0FC01EE0FFF1FE80F02
:10EE7000F91F4E9DB0014F9D700D5E9D700D1124C8
:10EE8000E60FF71F209FE001219FD00D309FD00D8E
:10EE90001124EC0FFD1FE452FC4F808181608083C0
:10EEA000209136362223B1F08C9190E0FC01EE0FD8
:10EEB000FF1FE80FF91FE60FF71FEC0FFD1FE352CE
:10EEC000FC4F9D2D921B990F990F990F8081877090
:10EED000892B0FC08C9190E0FC01EE0FFF1FE80F13
:10EEE000F91FE60FF71FEC0FFD1FE352FC4F808167
:10EEF00087708083FA01E55CF44DC0824F5F5F4FFD
:10EF00004031510509F09CCF809146029091470213
:10EF1000029709F083C180918D3682FF3EC08091B7
:10EF2000973683FF0DC083E090E090934702809373
:10EF300046020E94B30B8093B10281E080932C01C2
:10EF400080918F3683FF0CC087E090E0909347025A
:10EF50008093460280E18093B10281E080932C018E
:10EF600080919F3683FF0CC083E090E0909347022E
:10EF70008093460280E18093B10281E080932C016E
:10EF800080919D3683FF09C086E090E09093470210
:10EF90008093460281E080932C018091913682FF1C
:10EFA00054C08091973683FF50C00091352B10E0FC
:10EFB0000E94B30B25E23DE0029FD001039FB00DFC
:10EFC000129FB00D1124AE53BC4FE091B102F0E09E
:10EFD000E25BF44D90819295907F980F9C9320E096
:10EFE00030E0C4ECD0E065E27DE041E08091352B7B
:10EFF00090E02C9FF0012D9FF00D3C9FF00D11240F
:10F00000DC01A69FC001A79F900DB69F900D112413
:10F01000E80FF91FE456FB4FDC01AE53BC4F8C9157
:10F020008083E091B102F0E0E55CF44D40832F5F16
:10F030003F4F20313105D1F6FD01E15AF34F8C915C
:10F0400080834093B90340932C018091913683FFD4
:10F0500004C081E08093F20105C084FF05C01092D6
:10F06000F20181E080932C018091A33683FF0CC0D4
:10F070008091973682FF08C09091B3028091B502CB
:10F08000981711F40E944E1F8091993682FF1BC081
:10F090008091973683FF17C00E94B30B0091B20294
:10F0A0000295007F080F0E94553910E0802F612FD4
:10F0B0000E949C64802F0E94472B1F5F1131B1F783
:10F0C00081E080932C018091973684FF0AC0809163
:10F0D000913682FD06C01092B53610920937109213
:10F0E00008372091B6363091B7362115310509F42D
:10F0F00075C08091913682FD71C0809108379091E2
:10F1000009372817390709F469C030930937209364
:10F1100008378091953682FF1AC00E94B30B873062
:10F1200010F087E002C00E94B30B8093B20280917E
:10F13000B3029091B2029295907F8F70980F909346
:10F14000B5028091B302891709F045C047C080918C
:10F150008D3682FD43C08091993682FD3FC00E946A
:10F16000D10B882309F10E94D10B182F0E94B30BF9
:10F17000181B1093312B0E94B30B9091B202929501
:10F18000907F980F9093322B9093B50221E02093BB
:10F19000B5368091B3028917B1F48091AB02882310
:10F1A00091F02093332B11C08091B536882369F4F8
:10F1B0000E94B30B9091B2029295907F980F90931A
:10F1C000B5021092312B1092332B9091B3028091A3
:10F1D000B502981719F081E08093362B9091B30215
:10F1E0008091B5028917D1F42091312B2223B1F0FF
:10F1F0008091AB02882391F08091332B9091322B38
:10F20000980F9093B50291E09093362B8F5F809387
:10F21000332B8150821710F01092332B80914602CD
:10F22000909147028130910519F40E9427268CC0E5
:10F23000892B09F087C00E9427268091F235882308
:10F24000C1F48091AB028823A1F41092F73310929D
:10F25000F6339091FD339093B5028091B3028917F4
:10F2600019F081E08093362B81E080932C0180930C
:10F27000F2358091D802882309F443C02091FA33F3
:10F280003091FB3321153105E1F11092D8028091C4
:10F29000F335882391F01092F7331092F633909162
:10F2A000FD339093B5028091B302891719F081E084
:10F2B0008093362B1092F33521C08091F6339091D4
:10F2C000F73301969093F7338093F63301978217C3
:10F2D000930720F01092F7331092F633E091F63353
:10F2E000F091F733EC50FC4C91859093B5028091EE
:10F2F000B302891719F081E08093362B81E0809367
:10F300002C018091A33683FF1FC08091AB0288231C
:10F3100021F081E08093F33517C01092F7331092FB
:10F32000F6339091FD339093B5028091B302891723
:10F3300019F081E08093362B81E080932C0180933B
:10F34000F23502C01092F235809146029091470248
:10F350000897D9F48091F1018230B9F48091EF01DE
:10F360008250823090F48091973683FF07C00E94CC
:10F37000B30B8093B40281E080932C018091B4029E
:10F380008B3018F08BE08093B4028091460290910C
:10F3900047020D9709F04BC08091953683FF05C059
:10F3A0000E940B6D81E08093B90380918D3682FFBE
:10F3B0003EC08091973683FF0DC083E090E090932C
:10F3C0004702809346020E94B30B8093B10281E012
:10F3D00080932C0180918F3683FF0CC087E090E0F2
:10F3E000909347028093460280E18093B10281E0CE
:10F3F00080932C0180919F3683FF0CC083E090E0C6
:10F40000909347028093460280E18093B10281E0AD
:10F4100080932C0180919D3683FF09C086E090E0A7
:10F42000909347028093460281E080932C01809163
:10F430004602909147020E9769F48091973684FFB7
:10F4400009C083E090E0909347028093460281E0F8
:10F4500080932C018091F035882349F08091F53319
:10F460000E945D681092F03581E080932C018091BC
:10F47000362B882399F11092362B81E080932C0152
:10F48000EBE3FBE21192BBE2EB34FB07D9F71092FE
:10F49000382B1092B90380918B3682FD04C0809185
:10F4A000AB02882371F481E080931E3660E0809186
:10F4B000352B882309F461E08091B5020E94856AAA
:10F4C0000DC060E08091352B882309F461E08091C4
:10F4D000B5020E94856A81E08093372B80911E36A9
:10F4E0008823C1F080911D368823A1F090E080919F
:10F4F000352B882309F491E09093352B8091B50248
:10F500008093B3020E9490258091B3020E94AD2B9C
:10F5100010921E368091372B8823A1F08091AB0288
:10F52000882381F41092372B90E08091352B88232B
:10F5300009F491E09093352B0E9490258091B302BD
:10F540000E94AD2B8091EA36882331F08091B3027E
:10F550000E94AD2B1092EA3680918F3683FF16C041
:10F5600080918D3682FD12C0CBE3DBE210E0888112
:10F57000882341F018828091B302612F0E949C641D
:10F580000E9469391F5F2196103189F78091B90374
:10F590008823B9F080918F3683FF13C080918D3618
:10F5A00082FD0FC08091460290914702049749F076
:10F5B0001092B9038091B30260E10E949C640E94A2
:10F5C00069398091E7368823A1F080918F3683FFD7
:10F5D00010C080918D3682FD0CC0809146029091C2
:10F5E0004702049731F01092E7368091B3020E94EF
:10F5F000472B8091F1358823A1F080918F3683FFCE
:10F6000010C080918D3682FD0CC080914602909191
:10F610004702049731F01092F1358091F5330E9442
:10F62000446280918F3684FF03C081E080932C0177
:10F630008091460290914702059709F0C7C08091DA
:10F640008D3682FD63C08091933682FD06C0809125
:10F65000B6369091B7360E94FE0A80918B3682FFB3
:10F6600035C08091933683FD04C08091A33683FF1B
:10F6700007C01092F1331092F0331092CE3615C0BD
:10F6800080919F3683FF22C08091392B882381F09F
:10F690008091F202882349F41092F1331092F033F2
:10F6A0001092F2021092392B0EC01092F2020BC08F
:10F6B0001092F20281E08093392B8FEF9FEF9093AD
:10F6C000F1338093F03381E080932C0180919D365B
:10F6D00083FF0BC090E08091CE36882309F491E03F
:10F6E0009093CE3681E080932C0180919F3683FFEA
:10F6F0001EC080918B3682FD1AC090E08091F2028C
:10F70000882309F491E09093F2020EC0809197361D
:10F7100083FF0DC083E090E0909347028093460200
:10F720000E94B30B8093B10281E080932C019091F1
:10F73000B3028091B5028917D1F42091312B222395
:10F74000B1F08091AB02882391F08091332B90919E
:10F75000322B980F9093B50291E09093362B8F5FE8
:10F760008093332B8150821710F01092332B8091AD
:10F77000933684FF15C02091F2333091F333211575
:10F78000310571F08091F0339091F1338227932706
:10F790009093F1338093F0331092F3331092F2335D
:10F7A0008091933682FF12C06091F2337091F333EF
:10F7B00080E00E9485089093F3338093F23306C073
:10F7C0000E94B30B882309F0A0C96BC9DF91CF91C8
:10F7D0001F910F91FF90EF90DF90CF90BF90AF906F
:10F7E0009F908F9008958091AB02882311F410921E
:10F7F00005360E943D280E945D510E9464160E94B9
:10F8000070630E94AA6E0E94813B0895FF920F933D
:10F810001F930E94F56CECE6F6E31082329686E3C5
:10F82000EC38F807D1F71092B0361092A836109243
:10F830009E361092943687E898E367E570E00E9460
:10F84000FE7F87E898E36FEF0E94808087E898E367
:10F850006DEF0E94808087E898E30E94C38087E86C
:10F8600098E367E570E043E050E00E94D48087E8C9
:10F8700098E30E941180082F87E898E30E94118086
:10F88000F82E87E898E30E94118010E00F0D111DFB
:10F89000080F111D0430110531F00E94A6390E9495
:10F8A000EC660E94142B0E9425108091093684304A
:10F8B00051F40E9484398FE70E947D0F80E094E02C
:10F8C0000E94480FF8CF80910836833041F40E949F
:10F8D000A6390E94EC660E94142B0E949C2B0E9469
:10F8E000282C80910A36803F51F490E080910B36AD
:10F8F000882309F491E090930B360E94A42B0E9478
:10F90000F96980916800816080936800D89A80913D
:10F910006B00836080936B0080E06091352B0E94C8
:10F92000856A0E94902580E090E00E94DE0E0E9491
:10F93000B61E80E00E945D681092B1008091B10017
:10F940008093B0008091B00082608093B00080917D
:10F95000B10082608093B1008FE78093B300809103
:10F9600070008260809370000E941A2C78948BEE55
:10F9700096E360E045E75AE00E94CE7E8BEE96E388
:10F9800061E04DE75AE00E94CE7E8BEE96E362E0A6
:10F9900045E85AE00E94CE7E8BEE96E363E04DE8A8
:10F9A0005AE00E94CE7E8BEE96E364E045E95AE091
:10F9B0000E94CE7E8BEE96E365E04DE95AE00E9410
:10F9C000CE7E8BEE96E360E142E020E00E94FE7E78
:10F9D0008BEE96E360E00E948E7E8BEE96E361E014
:10F9E0000E948E7E8BEE96E362E00E948E7E8BEE0E
:10F9F00096E364E040E00E94987E8BEE96E364EC30
:10FA00000E948F878BEE96E36EED0E948F878BEEC0
:10FA100096E367ED0E948F878BEE96E361ED0E947F
:10FA20008F878BEE96E369E040E00E94987E8BEE34
:10FA300096E36CEB0E948F878BEE96E360EB0E945F
:10FA40008F878BEE96E369EB0E948F878BEE96E3B0
:10FA50006FEB0E948F878BEE96E36BEB0E948F8794
:10FA60008BEE96E360EB0E948F878BEE96E360E06F
:10FA700041E00E94987E8BEE96E363E00E948E7ECA
:10FA80008BEE96E364E00E948E7E8BEE96E365E05B
:10FA90000E948E7E8BEE96E366E041E00E94987EA7
:10FAA0008BEE96E365EE7AE00E946C8760ED77E07E
:10FAB00080E090E00E94C1858BEE96E360E045EA2D
:10FAC0005AE00E94CE7E8BEE96E361E04DEA5AE06A
:10FAD0000E94CE7E8BEE96E362E045EB5AE00E94F8
:10FAE000CE7E8BEE96E363E04DEB5AE00E94CE7E35
:10FAF0008BEE96E364E045EC5AE00E94CE7E8BEEFE
:10FB000096E365E04DEC5AE00E94CE7E8BEE96E3E4
:10FB100066E045ED5AE00E94CE7E8BEE96E367E00C
:10FB20004DED5AE00E94CE7E8BEE96E360E142E01E
:10FB300020E00E94FE7E1F910F91FF900895982F64
:10FB400080917A378230E0F42FB7F894913029F021
:10FB5000913060F0923029F402C092E008C094E045
:10FB600006C082E080937A372FBF089591E081E04C
:10FB700080937A3780917B37892B80937B372FBF97
:10FB8000089584E061E00E94F28684E061E00E94D2
:10FB90008E868CB580618CBD8CB580648CBD87E011
:10FBA00061E00E948E8685E061E00E948E86089565
:10FBB0000F931F938C01FC01868160E00E94F28606
:10FBC00081E090E00E941A86F801868161E00E943F
:10FBD000F28681E090E00E941A86F801868160E05A
:10FBE0000E94F28684E690E00E941A861F910F918F
:10FBF0000895CF92DF92EF92FF920F931F93CF93CE
:10FC0000DF93D82EC92E282F392FC9018C01C0E0CF
:10FC1000D0E0E62EFF24F801878161E00E948E8605
:10FC2000B7010C2E02C0759567950A94E2F76170D2
:10FC3000F80187810E94F28621960F5F1F4FC8301E
:10FC4000D10549F78D2D9C2D0E94D87DDF91CF9154
:10FC50001F910F91FF90EF90DF90CF900895CF927A
:10FC6000DF92EF92FF920F931F93CF93DF93D82EE3
:10FC7000C92E282F392FC9018C01C0E0D0E0E62E13
:10FC8000FF24F801878161E00E948E86B7010C2E67
:10FC900002C0759567950A94E2F76170F801878153
:10FCA0000E94F28621960F5F1F4FC430D10549F79D
:10FCB0008D2D9C2D0E94D87DDF91CF911F910F91AA
:10FCC000FF90EF90DF90CF9008951F93CF93DF9335
:10FCD000EC01162F8C81642F0E94F2868D818F3F5C
:10FCE00019F060E00E94F2868F8584FF05C0CE0186
:10FCF000612F0E94F97D0EC0612F70E084E0759540
:10FD000067958A95E1F7CE010E942F7ECE01612F83
:10FD10000E942F7EDF91CF911F91089541E00E94B4
:10FD2000657E81E090E0089540E00E94657E089540
:10FD3000DF93CF93CDB7DEB728970FB6F894DEBF29
:10FD40000FBECDBF9C01FE013196A4ECB1E088E06E
:10FD50000D9001928150E1F7F9018389481708F06D
:10FD600040E0E42FF0E0EE0FFF1FEC0FFD1F81815C
:10FD7000680F6068C9010E94947E28960FB6F894B7
:10FD8000DEBF0FBECDBFCF91DF91089562E00E942C
:10FD9000947E80ED97E00E941A860895EF92FF927C
:10FDA0000F931F93CF93DF938C017A0170E06770FC
:10FDB000707023E0660F771F2A95E1F760640E9458
:10FDC000947EC0E0D0E0F701EC0FFD1F4491F801F4
:10FDD000A081B1812D913C91C801642FF901099551
:10FDE0002196C830D10579F7C8010E94C67EDF91FF
:10FDF000CF911F910F91FF90EF900895CF93DF93D4
:10FE0000EC01423018F08F8588608F874B8B1C8AFD
:10FE1000222329F0413019F48F8584608F8780E593
:10FE200093EC0E941A868C8160E00E94F2868E819B
:10FE300060E00E94F2868D818F3F19F060E00E94A1
:10FE4000F286CE0163E00E942F7E88E893E10E9453
:10FE50001A86CE0168E00E942F7E88E893E10E9416
:10FE60001A86CE0162E00E942F7E88E893E10E940C
:10FE70001A86CE0162E00E942F7E88E893E10E94FC
:10FE80001A86CE0168E00E942F7E88E893E10E94E6
:10FE90001A86CE0168E00E94947E88E893E10E9471
:10FEA0001A86CE0161E00E94947E88E893E10E9468
:10FEB0001A86CE0166E00E94947E88E893E10E9453
:10FEC0001A86CE0162E00E94947E88E893E10E9447
:10FED0001A86CE016CE00E94947E88E893E10E942D
:10FEE0001A86DF91CF9108956F927F928F92AF9291
:10FEF000CF92EF920F931F93DF93CF93CDB7DEB7DF
:10FF00003C01162F842FF301448325830683E78267
:10FF1000C086A18682869D8593879E8594879F85CE
:10FF200095879889968761E00E948E86F301858186
:10FF30008F3F19F061E00E948E86F301868161E0B7
:10FF40000E948E86112319F0F301178603C080E109
:10FF5000F3018787C30160E141E020E00E94FE7E5B
:10FF6000CF91DF911F910F91EF90CF90AF908F9035
:10FF70007F906F9008958F92AF92CF92EF920F93F0
:10FF80001F93CF93DF93DC01362F542F722F102F46
:10FF9000AE2C8C2C13961C921E92129780EC91E042
:10FFA00011969C938E9300D000D0EDB7FEB731969A
:10FFB000CDB7DEB71982118212821382CD0161E0C2
:10FFC000432F2FEF052FE72EC12E0E94747F0F9035
:10FFD0000F900F900F90DF91CF911F910F91EF90A5
:10FFE000CF90AF908F90089581E080938638609392
:10FFF00001381092843810928538089581E08093FA
:020000021000EC
:1000000086386093013810928438109285380895AC
:100010002091003830E08091FF37281B3109C90159
:1000200008954091FF3780910038481718F02FEF5E
:100030003FEF0AC0E42FF0E0E358F84C8081282F0E
:1000400030E04F5F4093FF37C9010895E091FF37DB
:1000500080910038E81718F0EFEFFFEF06C0F0E0EE
:10006000E358F84C8081E82FF0E0CF01089508951F
:1000700010928A381092893888EE93E0A0E0B0E0C0
:1000800080938B3890938C38A0938D38B0938E38B2
:1000900080ED91E090938838809387380895CF92CF
:1000A000DF92EF92FF920F931F93CF93DF937C0128
:1000B0006B018A01809186388823A1F0C0E0D0E0EE
:1000C0000DC0D701ED91FC91D601AC0FBD1F019081
:1000D000F081E02DC7016C9109952196C017D107D9
:1000E00080F304C0CB01642F0E948581C801DF9199
:1000F000CF911F910F91FF90EF90DF90CF900895D7
:10010000DF93CF930F92CDB7DEB7FC016983809167
:1001100086388823C9F080918538823838F081E0AC
:1001200090E09383828320E030E015C08091843892
:10013000E82FF0E0EE5FF74C998190838F5F80931A
:1001400084388093853805C0CE01019661E00E9415
:10015000858121E030E0C9010F90CF91DF910895B2
:100160000F93062F8091013862E078E34091853843
:1001700021E00E94308110928438109285381092CC
:1001800086380F91089561E00E94B0800895433849
:1001900008F042E8862F6DE777E30E94E78010922F
:1001A000FF3780930038089521E00E94C7800895AA
:1001B00021E00E94C78008951092FF371092003806
:1001C00010928438109285380E9435830895382F14
:1001D000433810F040E042C0809193388823E1F723
:1001E00091E090939338209395388FEF8093263A3F
:1001F00010921D39415040931E394F5F90939438AF
:1002000080919438330F832B809394388091963863
:10021000813041F410929638809194388093BB00DD
:1002200085EC01C085EE8093BC00809193388130CD
:10023000E1F380911D39841710F440911D3920E0BD
:1002400030E00AC0FB01E20FF31FD901A556B74CFD
:100250008C9180832F5F3F4F2417A0F3842F089544
:100260000F931F93582F122F433810F081E04AC08C
:10027000809193388823E1F782E08093933800934C
:1002800095388FEF8093263A10921D3940931E398E
:10029000ABE9B8E3FB0102C081918D938E2F861BE1
:1002A0008417D0F31092943880919438550F852B91
:1002B0008093943880919638813041F4109296382A
:1002C000809194388093BB0085EC01C085EE8093CB
:1002D000BC00112321F0809193388230E1F38091AA
:1002E000263A8F3F11F480E00DC08091263A80328B
:1002F00011F482E007C08091263A803311F084E047
:1003000001C083E01F910F910895482F633810F0CA
:1003100081E0089580919338843011F082E008954F
:100320006093A239AFE1B9E3842F9C01F90102C0C7
:1003300081918D938E2F841B8617D0F380E00895D2
:100340001F920F920FB60F920BB60F9211242F939C
:100350003F934F935F936F937F938F939F93AF934D
:10036000BF93EF93FF938091B90090E0887F9070E6
:100370008036910509F4F2C081369105CCF58832BA
:10038000910509F47BC089329105B4F4803191055F
:1003900009F46FC0813191053CF4009709F447C11D
:1003A000089709F04FC165C08831910509F466C00E
:1003B000809709F047C182C08034910509F4A4C038
:1003C0008134910544F48033910509F482C0C897C3
:1003D00009F038C189C08035910509F489C0883594
:1003E000910509F496C08834910509F02BC1AEC07F
:1003F0008839910509F413C189399105ECF48837DE
:10040000910509F4ABC0893791054CF48836910504
:1004100009F4A4C08037910509F014C19FC0883841
:10042000910509F4FCC08039910509F49DC080381C
:10043000910509F007C198C0803B910509F4C6C039
:10044000813B91054CF4803A910509F49FC0883AAC
:10045000910509F0F7C0BAC0803C910509F4E3C0EA
:10046000883C910509F4DFC0883B910509F0EAC09A
:10047000C2C0809194388093BB00CFC090911D3949
:1004800080911E39981768F490911D39E92FF0E09A
:10049000E556F74C80818093BB009F5F90931D3998
:1004A000BCC080919538882309F44BC085ED8093BA
:1004B000BC008091BC0084FDFCCFC2C080E2809370
:1004C000263A85ED8093BC008091BC0084FDFCCF72
:1004D000B7C080E38093263A85ED8093BC0080917D
:1004E000BC0084FDFCCFACC088E38093263A9BC05F
:1004F00080911D399091BB00E82FF0E0E556F74C54
:1005000090838F5F80931D3990911D3980911E39A2
:1005100082C080911D399091BB00E82FF0E0E55634
:10052000F74C90838F5F80931D3980919538882395
:1005300041F085ED8093BC008091BC0084FDFCCF30
:100540007FC081E08093963884EA6EC085ED809309
:10055000BC008091BC0084FDFCCF72C083E080931E
:1005600093381092253A59C08091253A823808F084
:1005700056C08091253A9091BB00E82FF0E0ED55F0
:10058000F64C90838F5F8093253A47C08091253A3F
:10059000823830F4E091253AF0E0ED55F64C1082C7
:1005A00085ED8093BC008091BC0084FDFCCF10924F
:1005B00093386091253AE0919938F0919A3883EA1E
:1005C00099E370E009951092253A2DC084E080935C
:1005D00093381092A1391092A239E0919738F09196
:1005E000983809958091A239882329F481E0809375
:1005F000A23910921F399091A139E92FF0E0E15E04
:10060000F64C80818093BB009F5F9093A1399091BD
:10061000A1398091A239981710F485EC01C085E8C2
:100620008093BC000FC085EC8093BC0009C0109281
:10063000263A85ED8093BC008091BC0084FDFCCF00
:1006400010929338FF91EF91BF91AF919F918F914D
:100650007F916F915F914F913F912F910F900BBEC2
:100660000F900FBE0F901F9018951092933881E055
:10067000809395381092963881E161E00E94F2866D
:1006800080E161E00E94F286E9EBF0E080818E7FFC
:10069000808380818D7F808388E48093B80085E4A7
:1006A0008093BC000895F999FECF72BD61BDF89AA0
:1006B00080B50895F999FECF1FBA72BD61BD40BDE6
:1006C0000FB6F894FA9AF99A0FBE089508951F92FA
:1006D0000F920FB60F920BB60F9211242F933F93E8
:1006E0004F938F939F93EF93FF934091C600209178
:1006F000683A3091693A2F5F3F4F2F733070809185
:100700006A3A90916B3A2817390759F0E091683AA4
:10071000F091693AE85DF54C40833093693A209353
:10072000683AFF91EF919F918F914F913F912F9157
:100730000F900BBE0F900FBE0F901F901895E09179
:10074000443BF091453BE05CFF4F819191912081CA
:100750003181821B930B8F739070892B11F00E9453
:10076000668308951F920F920FB60F920BB60F92E9
:1007700011242F933F938F939F93EF93FF93209197
:10078000AC3A3091AD3A8091AE3A9091AF3A281799
:10079000390731F48091C1008F7D8093C10014C06E
:1007A000E091AE3AF091AF3AE459F54C2081809156
:1007B000AE3A9091AF3A01968F7390709093AF3AA2
:1007C0008093AE3A2093C600FF91EF919F918F9155
:1007D0003F912F910F900BBE0F900FBE0F901F9067
:1007E00018951F920F920FB60F920BB60F9211240D
:1007F0002F933F938F939F93EF93FF932091343BDD
:100800003091353B8091363B9091373B2817390723
:1008100031F48091C9008F7D8093C90014C0E091AC
:10082000363BF091373BEC50F54C20818091363BC4
:100830009091373B01968F7390709093373B8093E4
:10084000363B2093CE00FF91EF919F918F913F9186
:100850002F910F900BBE0F900FBE0F901F90189509
:10086000DC011C96ED91FC911D97E05CFF4F2191FE
:10087000319180819181281B390B2F733070C90110
:100880000895DC011C96ED91FC911D97E05CFF4FF3
:1008900020813181E054F040DF01AE5BBF4F8D918C
:1008A0009C9111972817390719F42FEF3FEF07C0D4
:1008B0008D919C91E80FF91F8081282F30E0C901AC
:1008C0000895DC011C96ED91FC911D97E05CFF4FB3
:1008D00020813181E054F040DF01AE5BBF4F8D914C
:1008E0009C9111972817390719F42FEF3FEF10C08B
:1008F0008D919C911197E80FF91F20818D919C910A
:10090000119701968F73907011969C938E9330E09F
:10091000C9010895FC0186859785DC01A05CBF4F65
:10092000FC01EE5BFF4F2D913C91119780819181ED
:1009300028173907C1F70895CF93DF93EC01EE85AF
:10094000FF85E05CFF4F20813181E054F0402F5F54
:100950003F4F2F733070DF01AE5BBF4F8D919C9185
:10096000119728173907D1F3E05CFF4F80819181FF
:10097000E054F040E80FF91F6083EE85FF85E05CEE
:10098000FF4F31832083EE89FF89208181E090E051
:100990000D8C02C0880F991F0A94E2F7282B208340
:1009A00081E090E0DF91CF9108951F9310923B3B3F
:1009B00010923A3B28EE33E040E050E020933C3B7D
:1009C00030933D3B40933E3B50933F3B60EE71E0A4
:1009D0007093393B6093383B88E29AE39093453BB0
:1009E0008093443B8CE69AE39093473B8093463B4D
:1009F00085EC90E09093493B8093483B84EC90E0F9
:100A000090934B3B80934A3B80EC90E090934D3B1E
:100A100080934C3B81EC90E090934F3B80934E3B16
:100A200086EC90E09093513B8093503B14E0109300
:100A3000523BB3E0B093533BA7E0A093543BF5E0A7
:100A4000F093553BE1E0E093563B10925A3B1092F5
:100A5000593B20935B3B30935C3B40935D3B509311
:100A60005E3B7093583B6093573B80EB9AE39093C7
:100A7000643B8093633B84EF9AE39093663B80935F
:100A8000653B8DEC90E09093683B8093673B8CECEA
:100A900090E090936A3B8093693B88EC90E0909360
:100AA0006C3B80936B3B89EC90E090936E3B809322
:100AB0006D3B8EEC90E09093703B80936F3B109376
:100AC000713BB093723BA093733BF093743BE09304
:100AD000753B1F9108951F920F920FB60F9211242C
:100AE0002F933F938F939F93AF93BF9380917A3BC4
:100AF00090917B3BA0917C3BB0917D3B30917E3BC4
:100B00000196A11DB11D232F2D5F2D3720F02D57EC
:100B10000196A11DB11D20937E3B80937A3B90935B
:100B20007B3BA0937C3BB0937D3B8091763B909147
:100B3000773BA091783BB091793B0196A11DB11D07
:100B40008093763B9093773BA093783BB093793B2F
:100B5000BF91AF919F918F913F912F910F900FBEB9
:100B60000F901F9018958FB7F89420917A3B309191
:100B70007B3B40917C3B50917D3B8FBFB901CA01CB
:100B800008959B01AC017FB7F8948091763B9091DA
:100B9000773BA091783BB091793B66B5A89B05C0A7
:100BA0006F3F19F00196A11DB11D7FBFBA2FA92F6C
:100BB000982F8827860F911DA11DB11D62E0880F17
:100BC000991FAA1FBB1F6A95D1F7BC012DC0FFB7A3
:100BD000F8948091763B9091773BA091783BB091CF
:100BE000793BE6B5A89B05C0EF3F19F00196A11D22
:100BF000B11DFFBFBA2FA92F982F88278E0F911DE7
:100C0000A11DB11DE2E0880F991FAA1FBB1FEA9525
:100C1000D1F7861B970B885E9340C8F22150304075
:100C20004040504068517C4F211531054105510528
:100C300071F60895019739F0880F991F880F991F51
:100C400002970197F1F70895789484B5826084BD86
:100C500084B5816084BD85B5826085BD85B58160C0
:100C600085BDEEE6F0E0808181608083E1E8F0E020
:100C70001082808182608083808181608083E0E84F
:100C8000F0E0808181608083E1EBF0E0808184602E
:100C90008083E0EBF0E0808181608083E1E9F0E037
:100CA000808182608083808181608083E0E9F0E0E0
:100CB000808181608083EAE7F0E0808184608083C6
:100CC0008081826080838081816080838081806870
:100CD00080831092C1000895982F883108F09851B0
:100CE00097708091AB018295880F880F807C892B4B
:100CF00080937C0080917A00806480937A00809158
:100D00007A0086FDFCCF2091780040917900942FE5
:100D100080E030E0282B392BC9010895482F50E09E
:100D2000CA01865D944FFC012491465F544FFA013D
:100D300084918823C1F0E82FF0E0EE0FFF1FE4510B
:100D4000F54FA591B491662341F49FB7F8948C9127
:100D5000209582238C939FBF08959FB7F8948C9120
:100D6000822B8C939FBF08958430C9F0853038F46E
:100D70008230F1F0833078F4813099F516C08730F5
:100D8000F9F0883018F4863061F516C08830F1F03B
:100D9000893039F521C0809180008F7703C0809120
:100DA00080008F7D80938000089584B58F7702C086
:100DB00084B58F7D84BD08958091B0008F7703C086
:100DC0008091B0008F7D8093B00008958091900055
:100DD0008F77809390000895809190008F7D80930D
:100DE00090000895FF920F931F93F62E482F50E026
:100DF000CA01865B944FFC012491CA01865D944F21
:100E0000FC011491465F544FFA0104910023C9F08C
:100E1000222319F0822F0E94B486E02FF0E0EE0F1B
:100E2000FF1FEA50F54FA591B4919FB7F894FF20AA
:100E300021F48C911095812302C08C91812B8C938D
:100E40009FBF1F910F91FF900895CF93DF930E9452
:100E500024860E94067CCFE9D3E80E94F37B20978A
:100E6000E1F30E949F83F9CFFC0120E030E0808114
:100E7000882311F421E030E0C9010895FC0181E0EC
:100E800080830895CF92DF92EF92FF920F931F938A
:100E9000CF93DF937C016B018A01C0E0D0E00FC0EB
:100EA000D6016D916D01D701ED91FC910190F0811A
:100EB000E02DC7010995C80FD91F01501040011539
:100EC000110571F7CE01DF91CF911F910F91FF9026
:100ED000EF90DF90CF900895EF92FF920F931F93C2
:100EE000CF93DF937C018B01C0E0D0E0F8010F5F6E
:100EF0001F4F6491662359F0D701ED91FC91019049
:100F0000F081E02DC7010995C80FD91FEFCFCE01A1
:100F1000DF91CF911F910F91FF90EF900895DC0129
:100F2000ED91FC910190F081E02D09950895CF930A
:100F3000DF93DB010D900020E9F71197A61BB70B9B
:100F4000EC01E881F9810280F381E02DAD01099582
:100F5000DF91CF9108954F925F927F928F929F92EF
:100F6000AF92BF92CF92DF92EF92FF920F931F93B7
:100F7000DF93CF93CDB7DEB7A1970FB6F894DEBF5E
:100F80000FBECDBF2C01742ECB01223008F42AE015
:100F900019A231E2C32ED12CCC0EDD1E822E992453
:100FA000AA24BB24672D752FA50194010E94938E5E
:100FB00079018A01C801B701A50194010E94418EFF
:100FC000472D461B0894C108D1084A3014F4405DEF
:100FD00001C0495CF6014083E114F10401051105EB
:100FE00021F07E2C5F2DC801DDCFC201B6010E9429
:100FF0009787A1960FB6F894DEBF0FBECDBFCF91F5
:10100000DF911F910F91FF90EF90DF90CF90BF90F5
:10101000AF909F908F907F905F904F900895DC01EC
:101020002115310541F4ED91FC910190F081E02D05
:10103000642F099508950E94AB870895EF92FF925F
:101040000F931F939A017B0100E010E0B801A70104
:101050000E940F881F910F91FF90EF900895EF92DB
:10106000FF920F931F939A01E62EFF2400E010E0F9
:10107000B801A7010E940F881F910F91FF90EF9078
:101080000895CF92DF92EF92FF920F931F93CF9329
:10109000DF93EC016A017B012115310541F4E88100
:1010A000F9810190F081E02D642F09951FC02A304D
:1010B0003105D1F477FF17C0E881F9810190F08103
:1010C000E02D6DE209958C0144275527BA014C1992
:1010D0005D096E097F09CE012AE00E94AB87980165
:1010E000280F391F04C02AE00E94AB879C01C90168
:1010F000DF91CF911F910F91FF90EF90DF90CF90F4
:101100000895EF92FF920F931F937B019A0100279E
:10111000F7FC0095102FB801A7010E9441881F918C
:101120000F91FF90EF9008950E94978708957F9206
:101130008F929F92AF92BF92CF92DF92EF92FF92E7
:101140000F931F93CF93DF934C017A018B01722E83
:10115000CB01BA0120E030E040E050E00E948B8CEF
:1011600087FD03C0C0E0D0E00EC0D401ED91FC913A
:101170000190F081E02DC4016DE20995EC0117FBAF
:10118000109517F9109520E030E040E05FE3AA24C5
:101190000BC0CA01B90120E030E040E251E40E94F6
:1011A0008F8C9B01AC01A394A71498F3C801B701DD
:1011B0000E94278C5B016C010E94FC8C7B018C01DE
:1011C000C401B801A7012AE030E00E940F88C80FCF
:1011D000D91F772039F0C40160E271E00E9497873F
:1011E000C80FD91FC801B7010E94288D9B01AC010F
:1011F000C601B5010E94268C24C020E030E040E208
:1012000051E40E94DE8D7B018C010E94F78C5B0112
:101210006C01CC24B7FCC094DC2CC401B601A50140
:101220002AE030E00E944188C80FD91FC601B501ED
:101230000E942A8D9B01AC01C801B7010E94268C37
:101240007A947720D1F6CE01DF91CF911F910F9143
:10125000FF90EF90DF90CF90BF90AF909F908F90D6
:101260007F9008950E9497880895AF92BF92CF9281
:10127000DF92EF92FF920F931F93CF93DF935C0166
:101280006B01EE24FF24C0E0D0E010C0D501ED9149
:10129000FC9100811181C601BE010E94B089682FB6
:1012A000C501F8010995E80EF91E2196F601848121
:1012B0009581C817D90750F3C701DF91CF911F91CE
:1012C0000F91FF90EF90DF90CF90BF90AF90089577
:1012D000EF92FF920F931F937B018C0161157105B3
:1012E0008105910529F420E030E040E050E00BC09A
:1012F0000E943B07A80197010E94B58EAC01CB016B
:10130000DA019C01AD01B901CA011F910F91FF9053
:10131000EF900895EF92FF920F931F937B018C0142
:10132000621773078407950764F4261B370B480B75
:10133000590BCA01B9010E946889E60EF71E081F01
:10134000191FB701C8011F910F91FF90EF900895E9
:10135000009729F0BC0180E090E00E9440070895CA
:10136000FC01848195816817790748F40190F08128
:10137000E02D309721F0E60FF71F8081089580E07F
:101380000895CF93DF939C01FB01EC01A881B98103
:10139000109729F06081718161157105D1F4C081C8
:1013A000D181209759F084819581892B39F08881EA
:1013B00090E022273327281B390B12C0109771F0B9
:1013C000F90184819581892B49F08C91282F30E097
:1013D00007C0CD010E942E089C0102C020E030E031
:1013E000C901DF91CF910895FC01DB012481358192
:1013F00014968D919C9115972817390711F020E0CC
:1014000007C0CF010E94C18920E0892B09F421E0A7
:10141000822F08950F931F93CF93DF93EC018B01DD
:101420006F5F7F4F888199810E944907009711F46F
:1014300080E005C0998388831B830A8381E0DF9164
:10144000CF911F910F910895CF93DF93EC01888185
:101450009981892B29F08A819B818617970760F4EF
:10146000CE010E940A8A882341F08C819D81892BBC
:1014700019F4E881F981108281E0DF91CF9108951C
:10148000EF92FF920F931F93CF93DF93EC017B01B9
:101490006C817D81E114F104C1F04115510599F091
:1014A0008A01060F171FB8010E94248A882369F059
:1014B000888199812C813D81820F931FB7010E9401
:1014C00037081D830C8381E001C080E0DF91CF915C
:1014D0001F910F91FF90EF900895DF93CF9300D06D
:1014E000CDB7DEB769831A82BE016F5F7F4F41E0DF
:1014F00050E00E94408A0F900F90CF91DF910895A5
:10150000CF93DF93EC0188819981009711F00E94BD
:101510009006198218821D821C821B821A82DF911A
:10152000CF9108950F931F93182F092F0E946D8A52
:10153000882321F4812F902F0E94808A812F902F61
:101540001F910F9108950F931F93182F092FFB01DF
:1015500060817181448155810E94408A882321F4F1
:10156000812F902F0E94808A812F902F1F910F91A1
:101570000895EF92FF920F931F93CF93DF93EC01A7
:101580007B018A01BA010E94248A882321F4CE01BA
:101590000E94808A07C01D830C8388819981B701CE
:1015A0000E943708CE01DF91CF911F910F91FF90DC
:1015B000EF900895CF93DF93EC01198218821B827C
:1015C0001A821D821C821E826115710551F0DB0199
:1015D0000D900020E9F71197A61BB70BAD010E94F3
:1015E000B98ADF91CF910895CF93DF93EC011982EF
:1015F00018821B821A821D821C821E82611571054F
:1016000051F0DB010D900020E9F71197A61BB70BF5
:10161000AD010E94B98ADF91CF9108950F931F9376
:10162000182F092F6115710559F0DB010D9000206D
:10163000E9F71197A61BB70BAD010E94B98A02C04A
:101640000E94808A812F902F1F910F910895EF9211
:10165000FF920F931F93DF93CF93CDB7DEB76197C0
:101660000FB6F894DEBF0FBECDBF8C01CB01F801E1
:1016700011821082138212821582148216827E01D8
:101680000894E11CF11CB70150E00E945F08C801FA
:10169000B7010E940E8B61960FB6F894DEBF0FBEA5
:1016A000CDBFCF91DF911F910F91FF90EF900895E3
:1016B000EF92FF920F931F93DF93CF93CDB7DEB7D7
:1016C00062970FB6F894DEBF0FBECDBF8C01CB0181
:1016D000F8011182108213821282158214821682FE
:1016E0007E010894E11CF11CB70150E00E943E0805
:1016F000C801B7010E940E8B62960FB6F894DEBF48
:101700000FBECDBFCF91DF911F910F91FF90EF9052
:101710000895EF92FF920F931F93DF93CF93CDB76E
:10172000DEB729970FB6F894DEBF0FBECDBF8C0190
:10173000862FF80111821082138212821582148280
:10174000168290E07E010894E11CF11CB70150E084
:101750000E945F08C801B7010E940E8B29960FB640
:10176000F894DEBF0FBECDBFCF91DF911F910F91D7
:10177000FF90EF900895DF93CF9300D0CDB7DEB701
:10178000FC01118210821382128215821482168249
:1017900069831A82BE016F5F7F4F0E940E8B0F908C
:1017A0000F90CF91DF910895DF93CF9300D0CDB705
:1017B000DEB7FC011182108213821282158214821C
:1017C000168269831A82BE016F5F7F4F0E940E8B63
:1017D0000F900F90CF91DF910895CF93DF93EC019D
:1017E000FB018617970761F06081718161157105B2
:1017F00029F0448155810E94B98A02C00E94808AE2
:10180000CE01DF91CF910895FC01118210821382E5
:1018100012821582148216820E94ED8B0895FC01BB
:1018200011821082138212821582148216820E9403
:10183000ED8B0895FC01808191810E9490060895AE
:10184000FC01808191810E94900608955058BB2729
:10185000AA270ED075C166D130F06BD120F031F4DB
:101860009F3F11F41EF45BC10EF4E095E7FB51C1FC
:10187000E92F77D180F3BA176207730784079507BA
:1018800018F071F49EF58FC10EF4E0950B2EBA2F6F
:10189000A02D0B01B90190010C01CA01A001112476
:1018A000FF27591B99F0593F50F4503E68F11A1622
:1018B000F040A22F232F342F4427585FF3CF4695B3
:1018C00037952795A795F0405395C9F77EF41F16D5
:1018D000BA0B620B730B840BBAF09150A1F0FF0F9F
:1018E000BB1F661F771F881FC2F70EC0BA0F621F8B
:1018F000731F841F48F4879577956795B795F7957B
:101900009E3F08F0B3CF9395880F08F09927EE0F0C
:10191000979587950895D9D008F481E008950CD063
:101920000FC107D140F0FED030F021F45F3F19F035
:10193000F0C0511139C1F3C014D198F39923C9F300
:101940005523B1F3951B550BBB27AA2762177307C5
:10195000840738F09F5F5F4F220F331F441FAA1F79
:10196000A9F333D00E2E3AF0E0E830D09150504039
:10197000E695001CCAF729D0FE2F27D0660F771FE7
:10198000881FBB1F261737074807AB07B0E809F0C9
:10199000BB0B802DBF01FF2793585F4F2AF09E3F5E
:1019A000510568F0B6C000C15F3FECF3983EDCF330
:1019B000869577956795B795F7959F5FC9F7880FD7
:1019C000911D9695879597F90895E1E0660F771F29
:1019D000881FBB1F621773078407BA0720F0621BBA
:1019E000730B840BBA0BEE1F88F7E095089504D0B3
:1019F0006894B111D9C00895BCD088F09F5790F079
:101A0000B92F9927B751A0F0D1F0660F771F881F23
:101A1000991F1AF0BA95C9F712C0B13081F0C3D03E
:101A2000B1E00895C0C0672F782F8827B85F39F0DC
:101A3000B93FCCF3869577956795B395D9F73EF482
:101A400090958095709561957F4F8F4F9F4F08952A
:101A5000E89409C097FB3EF4909580957095619548
:101A60007F4F8F4F9F4F9923A9F0F92F96E9BB27FE
:101A70009395F695879577956795B795F111F8CF7A
:101A8000FAF4BB0F11F460FF1BC06F5F7F4F8F4FE5
:101A90009F4F16C0882311F096E911C0772321F0DB
:101AA0009EE8872F762F05C0662371F096E8862F73
:101AB00070E060E02AF09A95660F771F881FDAF7CA
:101AC000880F9695879597F90895990F0008550FF7
:101AD000AA0BE0E8FEEF16161706E807F907C0F0B4
:101AE00012161306E407F50798F0621B730B840BBC
:101AF000950B39F40A2661F0232B242B252B21F496
:101B000008950A2609F4A140A6958FEF811D811D35
:101B1000089597F99F6780E870E060E008959FEF6F
:101B200080EC089500240A94161617061806090674
:101B3000089500240A941216130614060506089543
:101B4000092E0394000C11F4882352F0BB0F40F4CB
:101B5000BF2B11F460FF04C06F5F7F4F8F4F9F4F0B
:101B6000089557FD9058440F551F59F05F3F71F08D
:101B70004795880F97FB991F61F09F3F79F08795F4
:101B80000895121613061406551FF2CF4695F1DF7D
:101B900008C0161617061806991FF1CF869571050D
:101BA000610508940895E894BB2766277727CB0141
:101BB00097F908958ADF08F48FEF08950BD0C0CF0E
:101BC000B1DF28F0B6DF18F0952309F0A2CFA7CF38
:101BD0001124EACFC6DFA0F3959FD1F3950F50E013
:101BE000551F629FF001729FBB27F00DB11D639FCF
:101BF000AA27F00DB11DAA1F649F6627B00DA11D75
:101C0000661F829F2227B00DA11D621F739FB00D1A
